:020000040800F2
:10000000F8FF0120F9F00A0895F10A0839BC050843
:1000100095F10A0895F10A0895F10A080000000018
:1000200000000000000000000000000095F10A0838
:1000300095F10A080000000095F10A081D6B0408FC
:1000400095F10A0895F10A0895F10A0895F10A0850
:1000500095F10A0895F10A08A5210408CD210408A4
:10006000F52104081D22040845220408BD030000F0
:10007000D1030000E5030000F90300000D040000B7
:10008000210400003504000095F10A0895F10A08E2
:1000900095F10A0895F10A0895F10A086D220408FD
:1000A00095F10A08514C040895F10A08414C0408DE
:1000B000614C0408714C0408814C0408AD16040816
:1000C000A1160408E1160408D516040895F10A08DB
:1000D00095F10A08DD3D0000A53F000089410000C0
:1000E000AD22040895F10A08000000003D4D040807
:1000F000154D04084D4D0408054D04084904000041
:1001000095F10A0845320408914C040895F10A0853
:100110007143000059450000A14C0408A50F0A08CE
:100120005D040000710400008504000099040000D3
:10013000AD04000095F10A0895F10A0895F10A0846
:1001400000000000000000000000000000000000AF
:10015000C1040000D5040000E9040000414700008C
:10016000151704080917040895F10A0895F10A08FB
:1001700095F10A0895F10A0895F10A0800000000B7
:1001800095F10A0895F10A0829490000114B000071
:1001900095F10A0895F10A0895F10A0895F10A08FF
:1001A00095F10A0895F10A0895F10A0895F10A08EF
:1001B00095F10A0895F10A0895F10A08491704080B
:1001C0003D17040895F10A0895F10A0895F10A0807
:1001D00095F10A08E5050A0895F10A0895F10A085B
:1001E00095F10A0895F10A0895F10A0895F10A08AF
:1001F00095F10A0895F10A0895F10A0895F10A089F
:1002000095F10A0895F10A0895F10A0895F10A088E
:100210005D4D04086D4D04087D4D040895F10A08F4
:1002200095F10A0895F10A0895F10A080000000006
:100230004932040895F10A080000000095F10A0807
:1002400095F10A0895F10A0895F10A0895F10A084E
:1002500095F10A0895F10A0895F10A0895F10A083E
:1002600095F10A0895F10A0895F10A0895F10A082E
:1002700095F10A0895F10A08F94C00000000000009
:1002800095F10A080000000095F10A08000000003E
:080290000000000095F10A08CE
:020000040804EE
:10000000114A037A0168D35C10B4CC58CA1824F0A2
:100010000104CC501368DB07FCD4037D1F2B09D9E6
:10002000203B20225DF8044B02FA03F343F018034F
:10003000CB60704720225DF8044B02FA03F343F0D3
:1000400018038B60704700BF18F40B084368426DBB
:1000500030B49A61EFF31182502383F31288416820
:10006000D2B2856C0B68046D23EA050323430B6051
:1000700082F31188436981681A68096822F00102D5
:10008000D0E908541A60826A1D605C615A60D0E948
:100090000B429C60DA600023B0F86C2030BCCA626E
:1000A00003777047002A4FEA014C034630B508BF7A
:1000B000E64600F1C00514BF8E468C460024196840
:1000C0000C3353F8042C43F8084C41EA0C0142EA83
:1000D0000E02AB4243F80C1C43F8042CEFD1D0F8CD
:1000E000C03043EA0E03C0E93144C0F8C03030BD2F
:1000F00010B40C4C6368002B11DD002004F1080CD7
:100100000146DCF8AC3003F1C00259600C33934275
:10011000FBD1013063680CF5867C8342F1DC5DF82D
:10012000044B704704000020F0B5404C04EB401332
:1001300093F8543403B9F0BD3D4B42011D7893F858
:1001400001C065450CD00CEB4C0E03EBCE0E9EF8B7
:1001500004604FEA4C0E771E012F5AD9032E52D05D
:100160002244A2F83814EFF31181902383F312880C
:1001700092F83A34C9B2B2F8380443EA4003002096
:100180009BB282F83A0481F311881909207881EA38
:1001900013215940D8B1C9431B01D2F8505401244E
:1001A000D2F83C049BB201F00F01D5F8AC2084409A
:1001B0000B4302F1C000590013F4004F8BB202D17F
:1001C0005168214351600C329042F4D1F0BDD2F815
:1001D0003C041B01D2F8502401F00F0110309BB2F7
:1001E0000124D2F8AC200B43844002F1C000590036
:1001F00013F4004F8BB202D15168214351600C328D
:100200009042F4D1F0BD0CF1010606F00306AE42B7
:10021000A6D0E64403EBCE030344597C00299FD0CB
:10022000A318012083F83A049AE700BF04000020D5
:10023000401E0024704700BF024B03EB401393F8AD
:100240005504704704000020D0E90920131A5842D1
:100250005841704790F8573830B53BB990F8551869
:10026000012490F85638DAB2914200D830BD04FA31
:1002700003F2B0F85E5801332A43A0F85E28F2E793
:100280000379024613F0010006D0D2E90731D268A3
:100290005B1A013A03EA0200704710B5037904467D
:1002A00013F001030ED0FFF7EBFF034650B1226AB3
:1002B0006369E1689B5C0132B2FBF1F0DBB201FBE8
:1002C00010222262184610BD03799B070AD5436AA3
:1002D0008269D154436A02690133B3FBF2F102FB34
:1002E00011334362704770470171704703790146CB
:1002F00013F0020007D00B69D1E90921013B521A22
:100300001A40D2B2981A70470C4B4FF0E02C10B440
:100310005A6EDCF81800596E8A42F9D1996E8842FB
:10032000F6D8DC6E4FF47A7101FB04F31B1AB3FBB1
:10033000F4F35DF8044B01FB02307047401E0024CB
:1003400010B584464FEA810E102312F4004F4FEA95
:10035000420214BF0E240724013B92B2CCF80040A5
:10036000F444F2D100EB81128C010351122042F8C7
:10037000213010BD10B584464FEA810E0424130BC2
:10038000013C4FEA021203EB430392B203F118035C
:10039000CCF80030F444F2D100EB01130A01845090
:1003A000062043F8214010BD704700BF704700BFD2
:1003B00000EB4000024B03EBC00393F84905704784
:1003C00004000020064B93F8F825824206D900EB82
:1003D000400003EBC003D3F84C0570470020704782
:1003E000040000201D4B93F8FC25AAB3D3F8381560
:1003F00009B100200860012A2ED0D3F8501509B1A8
:1004000000200860022A27D0D3F8681509B100201F
:100410000860032A20D0D3F8801509B100200860B5
:10042000042A19D0D3F8981509B100200860052ACC
:1004300012D0D3F8B01509B100200860062A0BD0FD
:10044000D3F8C81509B100200860072A04D0D3F8F2
:10045000E0350BB100221A60704700BF0400002095
:100460001D4B93F8FC25AAB3D3F8381509B1002029
:100470000860012A2ED0D3F8501509B10020086079
:10048000022A27D0D3F8681509B100200860032A92
:1004900020D0D3F8801509B100200860042A19D0B3
:1004A000D3F8981509B100200860052A12D0D3F8B6
:1004B000B01509B100200860062A0BD0D3F8C81582
:1004C00009B100200860072A04D0D3F8E0350BB149
:1004D00000221A60704700BF04000020C34B1B7845
:1004E000002B40F04D81C24B93F8FC25002A00F010
:1004F000478193F8481530B500294ED1D3F8381507
:100500000020012A086047D993F86015002966D1B8
:10051000D3F850150020022A08603DD993F87815C9
:10052000002940F0C980D3F868150020032A08602C
:1005300032D993F89015002940F0E080D3F8801567
:100540000020042A086027D993F8A815002940F054
:10055000F680D3F898150020052A08601CD993F876
:10056000C015002940F00D81D3F8B0150020062AEF
:10057000086011D993F8D815002959D1D3F8C815B6
:100580000020072A086007D993F8F025002A72D1C5
:10059000D3F8E03500221A6030BDD3F83C25910A2B
:1005A000A1F58011522940F20D814FF0FE0CEFF3BE
:1005B0001181502080F312888E4C4FF02C0E556A1A
:1005C000C9B250690EFB0C4C013540F00100CCF86B
:1005D0009850506181F3118893F8FC258EE7D3F889
:1005E0005425910AA1F58011522940F2EF804FF075
:1005F000FE0CEFF31181502080F312884FF02C0E87
:10060000556A7C4CC9B2506901350EFB0C4440F070
:100610000100C4F89850506181F3118893F8FC25CB
:100620000020D3F85015022A08603FF677AFB3E7F1
:10063000D3F8CC25910AA1F58011522900F2E2806D
:100640006D4810F801C0EFF31181502080F312883B
:100650004FF02C0E556A674CC9B2506901350EFB3C
:100660000C4440F00100C4F89850506181F31188A7
:1006700093F8FC2582E7D3F8E425910AA1F58011CF
:10068000522900F2C2805C4810F801C0EFF31181DA
:10069000502080F312884FF02C0E556A554CC9B289
:1006A000506901350EFB0C4440F00100C4F898502D
:1006B000506181F311886BE7D3F86C25910AA1F59D
:1006C0008011522940F286804FF0FE0EEFF3118127
:1006D000502080F312884FF02C0C556A454CC9B25B
:1006E000506901350CFB0E4440F00100C4F89850ED
:1006F000506181F3118893F8FC2514E7D3F8842521
:10070000910AA1F58011522968D94FF0FE0CEFF340
:100710001181502080F312884FF02C0E556A354C11
:10072000C9B2506901350EFB0C4440F00100C4F819
:100730009850506181F3118893F8FC25FEE6D3F8B8
:100740009C25910AA1F5801152294BD94FF0FE0C3E
:10075000EFF31181502080F312884FF02C0E556A70
:10076000244CC9B2506901350EFB0C4440F0010025
:10077000C4F89850506181F3118893F8FC25E8E69D
:100780007047D3F8B425910AA1F58011522935D9C3
:100790004FF0FE0CEFF31181502080F312884FF0E0
:1007A0002C0E556A134CC9B2506901350EFB0C442E
:1007B00040F00100C4F89850506181F3118893F81B
:1007C000FC25D1E60C4810F801C0F0E60A4810F804
:1007D00001C00EE7084810F801E077E7064810F876
:1007E00001C094E7044810F801C0B1E700000024FC
:1007F00004000020401E002490200B08044810F83C
:1008000001C0C7E74FF0FE0C1DE74FF0FE0C3DE7BF
:1008100090200B0800EE100AB8EE400A704700BFA7
:10082000BCEEC00A10EE103A98B2704707280AD8FA
:100830004FF4B472054B02FB0033B3F80006B0FA74
:1008400080F0400970470020704700BF040000207E
:10085000072807D8044B4FF4B471012201FB003381
:1008600083F80226704700BF04000020072808D83C
:10087000044B03EB401393F8542412B1012283F884
:100880003A24704704000020072808D8054B03EBE2
:100890004013B3F83804B0FA80F0400970470020E4
:1008A000704700BF04000020054B93F8F8258242F2
:1008B00004D903EB4013D3F8440470470020704779
:1008C000040000200346012200205A77704700BF31
:1008D000826908B50346006BD96A02449A6101B186
:1008E0008847002008BD00BF436A02461B681B6A98
:1008F0005B685B7813F0010008BF5077704700BF5A
:10090000C2628161704700BF704700BF043070470A
:100910000C4B93F80823D3F8041302440144D2B2D9
:10092000C3F8041383F8082393F80823120605D5A7
:1009300093F8082382F0800283F80823024B0122F7
:100940005A707047401E0024000000242DE9F84F23
:10095000164FD7F80C53ED0A23D00026DFF850A02D
:1009600007F54479B0467419D7F810134FF0100307
:10097000524648BF0134D1F828B04846C7F83C83F6
:100980006410E102D8470F280BDD094B03F1100179
:1009900053F8042B013207D18B42F9D12546B542D9
:1009A000E1DCE802BDE8F88F661CF8E7401E002491
:1009B000E0250124194B596ED3F844238A1A322AB0
:1009C00005DCD3F858238A1A002A11DC7047D3F8C3
:1009D000481349B193F85423888802F0010209684A
:1009E000120100FA02F28A610022C3F8582370470C
:1009F000D3F848236AB110683231928810B4446940
:100A0000C3F8581322425DF8044B18BF12048261E8
:100A100070473231C3F85813704700BF401E00249E
:100A2000074AD2F848334BB192F854239988186892
:100A300002F001031B0101FA03F3836100207047F8
:100A4000401E0024044B4FF4007C0020D3F8683390
:100A5000A2F800C00B607047401E002400207047C1
:100A600001207047012070470020704710B41C69B6
:100A700094420CD394460A4661448C42996938BF2B
:100A8000A4EB0C0261445DF8044B70F061BF5DF8AB
:100A9000044B704710B504466FF05CFE01462046DB
:100AA00089B2BDE81040FFF73FBB00BF38B50B4D22
:100AB00000EB400005F5A763C40003EBC003254429
:100AC00093ED027AD3ED037AE7EE007AB0EE670A8F
:100AD0006FF040FED5F83835186038BD04000020AE
:100AE00002692DE9F843C36812EA030828D00546D5
:100AF0000E464FF00047B8FA88F327FA03F21B3B83
:100B0000D24308EA02082A61042B16D8DFE803F072
:100B10003B30251A0300B36A002B3FD003F1FF39A5
:100B200000231FFA89F9B362746A34B1236820463E
:100B3000494698476468002CF8D1B8F1000FDAD123
:100B4000BDE8F88370680028F7D0696B036889B244
:100B50009847B8F1000FCED1F2E7B0680028ECD08A
:100B6000A96B036889B29847B8F1000FC3D1E7E7D2
:100B7000F0680028E1D0E96B036889B29847B8F1C2
:100B8000000FB8D1DCE730690028D6D0296C0368A3
:100B900089B29847B8F1000FADD1D1E7EB6A1FFADF
:100BA00083F9C1E78069B4305CF08CBD10B590F872
:100BB0003DE0BEF1020F76D0144690F83D20844609
:100BC000012A02D1022280F83D200C2921D8DFE839
:100BD00001F007202020222020203A20202052004F
:100BE000DCF824003449DCF80020C1633349C164D7
:100BF00090F8341001290CD0012180F8341090F8BD
:100C00003510012952D000224FF4006380F83420BF
:100C10004365002010BDDCF828002749DCF80020DF
:100C2000C1632649C16490F834100129F1D0012133
:100C300080F8341090F835100129E4D1383221467B
:100C40005DF02CFAE5E7DCF82C001B49DCF800200D
:100C5000C1631A49C16490F834100129D9D0012127
:100C600080F8341090F835100129CCD13C3221465F
:100C70005DF014FACDE7DCF830000F49DCF8002015
:100C8000C1630E49C16490F834100129C1D001211B
:100C900080F8341090F835100129B4D14032214643
:100CA0005DF0FCF9B5E75FFA8EF010BD34322146F5
:100CB0005DF0F4F9ADE700BFB5A809085DA8090823
:100CC000F8B5A0F507642379DB0725D5657994F895
:100CD000543805F001073D46FBB1D4F848341A6892
:100CE000D36A5B08536294F8583823B1B4F8623879
:100CF0000133A4F8623885F00101606C64F0E6FA13
:100D0000012384F85738002384F8553884F856387E
:100D1000A4F85E3884F85438F8BD94F85768012E6A
:100D200003D194F8553884F856382046FFF792FAE4
:100D30004EB9012385EA030184F85738606CBDE899
:100D4000F84064F0C3BA0023394684F85738F5E711
:100D500038B5A0F507640022344D606C03685A6210
:100D6000A1F12903302B31D895F8373495F8381490
:100D70000133DBB2012B85F8373409D9B4F85E387A
:100D800085F837245B08A4F85E384B1C85F83834A6
:100D900095F838240023082AA4F8603815D185F87E
:100DA0003834B5F83A3401339BB2032BA5F83A3402
:100DB00008D92379DB0705D5E36A94F85E0843B3C5
:100DC000216B98470023A4F85E3838BD5B396C2945
:100DD0000CD8B4F85E3885F837245B0843F08003FC
:100DE000A4F85E3895F838340133CFE794F85938D1
:100DF000002BCDD1012185F83734A5F83A34802372
:100E000084F85918A4F85E3885F8381464F05EFA4E
:100E1000BEE7E3696269D054E369E2680133B3FB7A
:100E2000F2F102FB1133E361CCE700BF401E002466
:100E300038B55EF0D3F80D490D4CD1F8FC20A4FB79
:100E400000400C4D42F080720B4B800CC1F8FC202E
:100E50004FF060420949E866C2F8B01F00225A60AC
:100E60001A6842F001021A6038BD00BF00ED00E0D0
:100E700083DE1B43401E0024001000E055CEACC5AD
:100E800070B505460A26084C013E00D170BD94F9A4
:100E900000001BF071FB031E04DB6178EA1851723D
:100EA000A278EA540434EFE7E3200B0838B590F851
:100EB00028300446012B06D0407F08B9012038BDF8
:100EC0000023637738BD406A03681A7B9AB9637F51
:100ED000002BF3D00A4D022305F1200205F1400159
:100EE00057F006FC95F82130D84303F0010300F0D9
:100EF00001006377E6E71B6A002BE8D0002038BDCD
:100F0000E025012438B5044694F82830012B07D099
:100F1000637F0BB100236377012038BD1B6A23B1C7
:100F2000606A03681A7B002AF8D1637F002BF3D034
:100F3000074D022305F1200205F1400157F0D8FBCF
:100F400095F8213003F00102DB076277E4D5DBE797
:100F5000E0250124F0B5002395B0224E0446069307
:100F600002200B9306F180021093139311930092C9
:100F700006F1A002277F1C4D0192626A04950D467E
:100F80000290CDE90E3301238DF80C3007938DF8D4
:100F900020308DF834308DF8483006F1C0030593C9
:100FA000124B099306F160030A933B1D10680C93E2
:100FB0006BF07CFA9FB12A0E06F1620386F861207D
:100FC0002A0A9D70280C69465A701870606A57F09A
:100FD000D5FB636A18686BF069FA15B0F0BD06F1CD
:100FE0006103EDE7E0250124E9080408C5080408C9
:100FF00010B594B0044650220649684670F0A8FC2B
:101000006946606A57F0BAFB636A18686BF04EFA7B
:1010100014B010BD08210B082DE9F8431F46436AA0
:1010200004468846186891466BF040FA237FA06911
:10103000002B3BD0254E020E052386F8E120E23638
:10104000234D012FB0706B634FEA10434FEA10201D
:10105000337070704FF00000D8F800302B64D9F86E
:101060000030AB642363A86523D0022F1CD1D9F8CC
:10107000042028651344D8F8041085F84C00EA656C
:10108000012269652363134B85F860206B66124B60
:10109000627FA3F11401606A002A08BF194657F065
:1010A0006DFBE36A63B1206BBDE8F88304230B4E4C
:1010B000C6E7084B85F84C706865E8652B65E6E780
:1010C000636A18686BF0F2F9EDE700BFE0250124D0
:1010D00000000024D108040818000024C1260124BF
:1010E00000B583B08161019201A9049A00930123A4
:1010F000C2626A46FFF790FF03B05DF804FB00BFD1
:101100002DE9F843DDF820800F4616460021202205
:1011100004461D4670F012FDB8F1000F0CD0D8F84F
:101120000030B8F80A20E3811B0C2382D8F8043081
:101130006282E3821B0C238338466DF0F5FAF306D6
:1011400019D4431EB8B107EB000C01E0013B12D3E8
:101150001CF801EDBEF12E0FF8D1C01A03F1010900
:10116000421EB944032AA8BF0322082BA8BF0823A4
:1011700090461A4606E008280246B9464FF0000895
:10118000A8BF08224FF02033394620462360636011
:1011900070F0DEFB164B04F10800424649462381FD
:1011A000837070F0D5FB611EE21D11F801CFACF128
:1011B0006103ACF1200C192B98BF81F800C091425B
:1011C000F3D104F10A0011F8013FA3F16102203BC1
:1011D000192A98BF0B708142F5D1182365832D0C15
:1011E000E6722373099BA582E361BDE8F88300BF23
:1011F000202020002DE9F04FDFF8509485B0D9F879
:101200006400C9F84403002B5ED00C46154601F576
:10121000FE7603EB020B1DE0002D62D0D9F874338B
:10122000AB4200F0C580D9F87033AB4200F0F780D4
:10123000D9E9DE31AB424BD88D42C0F07281691AD8
:10124000204662F0CDFF013504F5007406F5007606
:101250005D4539D0D9F88023AA42DDD8AA1AD9F839
:101260009073D308396B02F0070802338B4202D324
:10127000BA6B93420BD939461846039362F080FF4C
:10128000039B0746002800F06C81C9F890033A7967
:10129000002A40F01D81D7F828A0BAF1000F00F015
:1012A00059813A6B013520464FF400719B1AFA6858
:1012B00004F5007406F5007608EBC3083B4602EB24
:1012C0004822D0475D45C5D1002005B0BDE8F08F6C
:1012D0008D42B4D24FF400720021204670F02EFCF3
:1012E000B1E74FF400722946204670F027FC8023B6
:1012F000CA4A84F8BE310C2384F8C231D9F870137D
:10130000D9F868339142C4F8C611C4F8CA3100F361
:101310000D81C34A013BC34F82FB0102C81787FB03
:1013200001C70A44C0EB6212C0EB2730BE4F87FBF7
:1013300002C7C2EB821C84F8C1018010A1EB0C0132
:10134000174420F03F0001310843D117C1EBE711EA
:1013500084F8C0010A4484F8BF21B04A934200F3E4
:10136000F180AF4AAF4882FB0312D91780FB0370AC
:101370001A44C1EB6212C1EB2031AB4880FB027012
:10138000C2EB821784F8C5118910DB1B104421F0D1
:101390003F0101331943D317C3EBE01384F8C411A1
:1013A0001A4484F8C3214AF65523A4F8FE314AE7CB
:1013B0004FF0FF3300274FF4F072201D84F8EC311A
:1013C000394684F8ED3184F8EE3184F8EF31522358
:1013D000237063706123A37084F8E7314123E370C5
:1013E00084F8E631722384F8E43184F8E531D9F8E1
:1013F0008833C4F8E83170F0A1FB5523C4F8F071CC
:1014000084F8FE316FF05503C4F8F471C4F8F87134
:1014100084F8FC7184F8FD7184F8FF3113E74FF410
:1014200000720021204670F089FB804B022203CB22
:1014300045F6EB032274227323809023A273A370DA
:10144000F82384F82C200822C4F803006273C4F83F
:1014500007106375D9F87013D9F868335B1A2362E3
:10146000D9E9DE135B1A4AF6552163620023E37261
:10147000E3736377A377E37784F82D3084F82E3015
:1014800084F82F3084F83130694BA3613E232377F1
:10149000012384F83030802384F84030654BC4F851
:1014A0004230654B84F84620A4F8FE11634A03CB12
:1014B000C4F84B101988C4F847009B78A4F84F1063
:1014C00084F8513003CAC4F85200C4F85610BAE682
:1014D0004FF400720021204670F030FB3B6CB8F1F5
:1014E000000F45D104F1200A002B00F081803B6BF6
:1014F000112253492046CDE90088FFF701FE3B6CDD
:101500001A6C002A00F081801B6B504611224D4955
:10151000CDE90088FFF7F4FD04F1400A4FF4E078CC
:1015200071E0E91A204662F05BFE8CE6FF22013B87
:1015300084F8C1214FF6FF72A4F8BF21374A9342C5
:101540007FF70FAFFF2384F8C5314FF6FF73A4F880
:10155000C33128E751464FF40072204670F0EEFA8E
:1015600071E6231F384A43F8042F9E42FBD16AE6F6
:10157000002B7F6C14BF02230123C3EB0813002F41
:101580003FF461AE013BBF6C002B01DD002FF9D1B0
:10159000A2464FF40078002F3FF455AE0AEB080343
:1015A00003959A460BE00025A8F12008CDE900E557
:1015B000FFF7A6FDBF6CCFB1B8F11F0F16D93D796B
:1015C00007F11C0E112239683B6BAAEB0800002DB5
:1015D000E9D17A79A8F120083D6942F02102CDE9EC
:1015E00000E5FFF78DFDBF6C002FE5D1039D2AE6D6
:1015F000CDE9008843464FF4F0780822D9F86C13FF
:101600002046FFF77DFD7F6CC5E75046434611221B
:101610000C49CDE90088FFF773FD7DE7FF03FB0070
:10162000832008829755454181808080FCF20B0819
:101630003F00FF0029940E0D08F30B0814F30B086C
:10164000F4F20B08F8F20B08DEADBEEF401E0024EA
:1016500030B40D4CBFF34F8F0C4BC3F85C42BFF35B
:101660004F8FBFF36F8F0A4B0A4D03F13000DA79C9
:101670002AB1597934F8112092B225F811200C338F
:101680008342F4D130BC70478040012400ED00E07B
:101690007C220024C029012400207047704700BF2D
:1016A00001485DF057B900BFE8220024084810B493
:1016B000D0F8A834D0F8DC4499691A682CB12346D4
:1016C00000F595605DF8044B18475DF8044B7047D2
:1016D000401E002401485DF03DB900BF4C230024AA
:1016E000084810B4D0F80C35D0F8404599691A680C
:1016F0002CB1234600F20C505DF8044B18475DF8FE
:10170000044B7047401E002401485DF023B900BF20
:10171000B0230024084810B4D0F87035D0F8A445A0
:1017200099691A682CB1234600F5AE605DF8044B48
:1017300018475DF8044B7047401E002401485DF0D7
:1017400009B900BF14240024084810B4D0F8D435D7
:10175000D0F8084699691A682CB1234600F2D45093
:101760005DF8044B18475DF8044B7047401E002499
:101770002DE9F04784B08DF80F30431C00F09F80B6
:101780000328044600F39B80824E642303FB00631E
:10179000D3F8A804002800F0928093F8E954202D93
:1017A00040F0878093F8E854012D00F082800125F5
:1017B000D6F8207683F8E85404E0D6F82036DB1B10
:1017C000192B66D8856915F40045F6D14FF0640AE7
:1017D000714B00974FEA41080AFB04FA41460AEBB5
:1017E0000309B24421234846CAF8DC548AF8E93494
:1017F00040238AF8EA340DF10F03CAF8EC54CAF812
:10180000CC340123AAF8D2340A2365F0F3FC002873
:1018100073D1BAF8D2349BB2FF2B40F29180DAF840
:10182000A814FF235D48AAF8D0344B685C4A0340F3
:1018300043EA08031A434A60642505FB046505E092
:10184000B5F8D2349BB2002B00F08C803A460A21C6
:1018500048465DF0BDF860BBD5F8CC34D5F8A81487
:1018600013F8010BB5F8D0248862C5F8CC34013ADE
:10187000B5F8D23492B2013BA5F8D0249BB2A5F8BA
:10188000D234B5F8D2349BB2002BD9D0002AD7D1AC
:101890001EE064232020002103FB0463D3F8EC2422
:1018A00083F8E8140243C3F8EC2483F8E90483F8CE
:1018B000EA14B6F8243601339BB2A6F82436002089
:1018C00004B0BDE8F087D6F82036DB1B0A2B27D8FA
:1018D0008A6912F08002F6D0B5F8D2349BB2FF2BA1
:1018E0000ED94B682D4A13402D4A43EA08031A4388
:1018F000FF23A5F8D0344A60A2E78AF8E854D8E775
:10190000B5F8D23425489BB24A68A5F8D034DBB28A
:10191000024048EA0343134343F000734B608FE7F0
:101920006423202103FB0464D4F8EC3484F8E82415
:101930000B43C4F8EC3484F8E91484F8EA24B8E7DB
:10194000BAF8D234DAF8A8149BB214484A68AAF854
:10195000D034DBB2024048EA0343134343F0007340
:101960004B6069E73946484665F0F0FB03460028BE
:101970009FD1D5F8A82420240A48D4615168014099
:101980000120516085F8E94485F8E83485F8EA34A7
:1019900096E700BF401E0024E8220024009C00FCC3
:1019A0000000FF0100E800FE2DE9F0410468D4E9E1
:1019B0000435A8611A7D1F681F2A49D9203A2021C1
:1019C0002E6801FA02F242F01802FA602A7D1F2AFC
:1019D00048D9203A202101FA02F242F01802F260BE
:1019E0006A6800215868016038461160116841F04A
:1019F0001001116093F80880A269414667F0B2FFB8
:101A00002D7AE2693046294667F0ACFF226A6368A6
:101A10009468184A12F80800515D5A686FF30F0273
:101A200022435A603A5842F001023A50725842F04A
:101A3000010272509A6842F440429A601A6842F079
:101A400001021A601A6842F400721A60BDE8F0815F
:101A500020212E6801FA02F242F01802BA602A7DB3
:101A60001F2AB6D8202101FA02F242F01802B26011
:101A7000B6E700BF18F40B08D3B20F2B21D8124BD6
:101A800000B503F17E0E02E00333734516D093F8E0
:101A900000C08445F8D193F801C08C45F4D102EB25
:101AA00042020A48997800EB82037C30C3F8841024
:101AB00000EB820083F87C105DF804FB00205DF8E9
:101AC00004FB0020704700BF58210B0800000024D1
:101AD00010B40C4C002304F5C56C01E0152B0CD0A0
:101AE00003EB430201331CF802108142F6D1144487
:101AF00094F92A065DF8044B70474FF0FF305DF80B
:101B0000044B7047401E002430B5124D002305F5EC
:101B1000A47C02E001331A2B1AD05CF833408442D3
:101B2000F8D10CEBC30EDC009EF804E08E45F1D139
:101B300002EB4202084B254403EB82017C3395F80B
:101B40004D4103EB8200C1F8844081F87C4030BDF8
:101B5000002030BD90200B0800000024F0B10023CD
:101B600010B504460E4894F804E000F5C56C01E099
:101B7000152B11D003EB430201331CF80210714501
:101B8000F6D183186179206893F92A26D3B20F2BF6
:101B900002D8BDE81040B7E7002010BD0020704714
:101BA000401E002401380E4B0E4A00EBC000D2F854
:101BB000D81003EB800310B4D3F83C3183B00A4C47
:101BC000A34214BF022301231943C2F8D810D2F84C
:101BD000D82013400193019B03B05DF8044B70477C
:101BE0000000002400440258000002400138F8B50B
:101BF00000EBC000124C1D46124B04EB800417464C
:101C00000E46D4F83C01984214BFA120A02065F0F4
:101C100055FBB4F95201B909C4F84C61C4F85451E8
:101C200065F020FBB4F95231002B07DB03F01F00F5
:101C300001225B090449824041F82320F8BD00BF1E
:101C4000000000240000024000E100E0234B5B683C
:101C5000C3F3080310B4DBB9EFF31183C3B9204B0E
:101C60004FF0E02C5A6EDCF81800596E8A42F9D118
:101C7000996E8842F6D8DC6E4FF47A7101FB04F35A
:101C8000181AB0FBF4F05DF8044B01FB020070473A
:101C9000EFF31181102383F312884FF0E02294694F
:101CA000136913F4803F0E4B03D00120C3F868067C
:101CB0009469586EC9B2D3F8682681F31188D96E39
:101CC0004FF47A73024403FB01F0001B5DF8044BF0
:101CD000B0FBF1F003FB0200704700BF00ED00E035
:101CE000401E0024BE4803780BB9012070474368AA
:101CF0002DE9F04F002BDFF8109387B0D9F864601E
:101D000018DD00F108050024B649D5F8F430BFF31A
:101D10004F8F03F59072C1F85C3220339342FAD1B1
:101D2000BFF34F8FBFF36F8F0134436805F586759E
:101D30009C42EADB90F8F815AB4A0491A2FB06122C
:101D4000AA4BAB4E5209DFF8C4A2A3FB0213DB0877
:101D500003EB8303A2EB4303DAB206EB830B06F536
:101D600038730592009300239846049B984500F031
:101D70001481DAF81830DAF80470D3E93D45FFF73A
:101D800065FF9C4999F86DE6012269180190BEF142
:101D9000540F99F86C0602FA07F204EB410104EBC8
:101DA000400301D1A9F87606994240F26A811F8862
:101DB000174200F05F815F88174200F070819F88B2
:101DC000174200F06E81DF8808331742ECD11C1BEC
:101DD00099424FEA640440F25481281B452828BFE9
:101DE000452003EB4000834280F04F8100251F46D1
:101DF000AC462946CDE9028EB3F800E00EEA020EA9
:101E00008E451CD1B3F802E00EEA020E714540F097
:101E10001A81B3F804E00EEA020E714540F0158114
:101E2000B3F80680083308EA0208414508D1984211
:101E300009D9B3F800E00EEA020E8E45E2D0023373
:101E4000984200F2E580BCF1110FDDE9028E40F20C
:101E50001C81DCF1150200F118816749D9F8800670
:101E6000D1F87C339C4238BFC1F87C43019C231AD3
:101E7000002B14DB614B03449C4201D923460533FC
:101E8000C9F88036D1F87C33052B40F20C81053B34
:101E9000DBB289F86C364FF0FF33C1F87C333AB1CE
:101EA00005FA02F2CCF1140C012505FA0CF51543E4
:101EB000534BC5F3C43203EB8202D2F8180205F08B
:101EC0001F0203EB8202D2F81812C5F34412C5F3C5
:101ED000842503EB820241EA0031D2F8182203EB99
:101EE000850341EA0211D3F8183241EA0321454B38
:101EF00081EA1122D3F81C3A82EA1212013302F06D
:101F00000F020F2A40F0A380B1F5803F80F09F8040
:101F1000BEF1540F4FEA111147D03A4AB1F5606F44
:101F2000C2F81C3A4DD0009B998196F8583005981C
:101F3000834210D0DBF8082033689B1A3360736843
:101F4000DBF830209B1A73600023CBF80830CBF805
:101F5000303086F85800336801333360DBF80830DE
:101F60000133CBF808304FF6FF73994207D17368FD
:101F700001337360DBF830300133CBF83030009B35
:101F800008F101085C360BF15C0B1433B8F1080F53
:101F90000AF1200A00937FF4E8AE0123194A0120D8
:101FA00082F8183B07B0BDE8F08FB9F87026B1F59C
:101FB000606F02F10102A9F87026124AC2F81C3AB9
:101FC000B1D199F8013003EB430309EBC303434458
:101FD0005B7C0D2BA7D18023009A9377A5E700BFE8
:101FE0000400002000ED00E01F85EB51CDCCCCCCEF
:101FF00030180020C7FFFF7F0000002420A1070049
:1020000090200B08FC100020401E00243C040020FF
:10201000A3EB070E254F33F8021C4FEA6E0E11405A
:102020000EF1010E87FB0E87A7EBEE774FF0010E46
:10203000012FB8BF0127BD40BC44013F0EFA07F78E
:102040003D431F46D8E60433FAE60633F8E6BEF110
:10205000540F04D1B9F870260132A9F87026144A39
:102060004FF6FF71C2F81C3AD2F8183A0133C2F8A1
:10207000183A5AE702331C1B99424FEA64043FF6B0
:10208000ACAE10B1013889F86C06BEF1540F7FF484
:1020900076AFB9F872360133A9F872366FE70433B8
:1020A00095E6063393E60023F3E600BF56555555F3
:1020B000FC100020264B70B51A785B789A4242D10A
:1020C000244E7368002B22DD06F108000025224C07
:1020D000D0F8AC30BFF34F8F03F1E002C4F86832A0
:1020E00020339342FAD1BFF34F8FBFF36F8F337812
:1020F00013B1037F012B20D042690135716800F5CF
:1021000086701368A94243F001031360E0DCFFF717
:102110009DFD124BD3F81C4B002C0DDD03F53263F3
:1021200003EBC4041968083333F8042CC8689C42D4
:1021300042EA0002CA60F5D170BD002380F8FC308D
:10214000FDF784FFD8E76BF02DF90028B8D170BDFA
:10215000401E00240400002000ED00E0FC100020E0
:10216000800AA0F58010522806D8044B1B5C0D2B6A
:1021700002D8034AD05670470020704790200B08C1
:1021800008F40B0860B182884FF0B0414FF0004373
:10219000B2FA82F2D1F88000D3400343C1F8803014
:1021A000704700BF4FF0B042D2F88030D2F88810AC
:1021B0000B4003F00103C2F8883023B1024BD3F87F
:1021C0008406036818477047401E00244FF0B04251
:1021D000D2F88030D2F888100B4003F00203C2F826
:1021E000883023B1024BD3F888060368184770473C
:1021F000401E00244FF0B042D2F88030D2F8881050
:102200000B4003F00403C2F8883023B1024BD3F82B
:102210008C06036818477047401E00244FF0B042F8
:10222000D2F88030D2F888100B4003F00803C2F8CF
:10223000883023B1024BD3F89006036818477047E3
:10224000401E00244FF0B042D2F88030D2F88810FF
:102250000B4003F01003C2F8883023B1024BD3F8CF
:102260009406036818477047401E0024F8B54FF0E5
:10227000B043D3F88050D3F88820154005F4787522
:10228000C3F888507DB1084F0126B5FA85F4C4F132
:102290001F0407EB840306FA04F4D3F884060368EA
:1022A0009847A543F1D1F8BD401E0024F8B54FF082
:1022B000B043D3F88050D3F88820154005F47C450E
:1022C000C3F888507DB1084F0126B5FA85F4C4F1F2
:1022D0001F0407EB840306FA04F4D3F884060368AA
:1022E0009847A543F1D1F8BD401E002430B10368E2
:1022F00082881B691A4214BF01200020704700BF6A
:1023000010B1036882889A61704700BF18B1838852
:1023100002681B049361704770B50D4682B0044695
:10232000164640B101680C4B0C4A0B449B0A02EB69
:102330004303B3F8980264F0C1FFC5F38101C5F30C
:10234000411305F01302CDE90016A188206868F05A
:1023500047FB02B070BD00BF0000FEA790200B0835
:1023600000B1D9E770472DE9F84FC44F6423044604
:1023700003FB0073D3F89064002E00F06981D3F85A
:102380009884B8F1000F04D098F90630002B40F083
:102390005F81642303FB0473D3F89C5425B195F942
:1023A0000630002B40F05481631CDBB2B8F1000F03
:1023B00004D0152288F8073088F8062015B11622B7
:1023C000EB71AA714FF0640A308D64F077FF2946F3
:1023D0000AFB04FA40466AF065FF404607EB0A092B
:1023E000DFF8BC8299F8A23499F8A024002B0CBF26
:1023F0004FF01E0B4FF03E0B5946FFF7B1FF28463A
:102400009F4D594699F8A1245544FFF7A9FF4C2246
:10241000002128466FF092FBD9F89034994A5B6806
:102420009342C9F8A834DFF87C9240F013815CF045
:10243000F7FDD9F82030C3F30213434493F8AC32CC
:1024400003F01F039FED907A9FED905AB0EE084A7B
:10245000D8406423F7EE003A4FF0000C07EE900AE4
:1024600003FB047340F21458F8EE677AB3F8A4A49F
:10247000C7EE275A07EE90AA9FED857AF8EEE77A25
:10248000C7EE274ADFED837AB0EE007AE5EE877A71
:10249000A5EE875A25EE844A37EE856A74EEE72A60
:1024A000BAF5C87F0CF1010ED5BF4FF496727822B1
:1024B0006423322307EE90EAD8BF4FF41679134411
:1024C000A2F13202F8EEE76AC8BF4FF4827907EE54
:1024D000903AD4BF41464FF4FA7166EEA56AB8EE61
:1024E000E77AC7EE267A07EE102A01EB0902B8EE6A
:1024F000C77A37EE447A77EEE37AFCEEE77A17EEA6
:10250000903AC7EE267AFCEEE77A17EE900A07EECD
:10251000909AB8EEE73A07EE902AF8EEE77A23EEC3
:10252000243A83EE277A37EE453A32EEC77AC3EE85
:10253000267A77EEE37AFCEEE77A17EE901AC7EE8A
:10254000267A77EEE37AFCEEE77A17EE902A02F12C
:10255000020909EB010BB0EE467A07EE90BAF8EEED
:10256000677AA6EEA77AF4EEC74AF1EE10FA7DDCA0
:1025700043EA00095FFA89F9B9F10F0F78D841EA07
:1025800002091FFA89F9B9F1FF0F71D81B05000480
:1025900003F07F6392B200F47F0003433E4843EAB6
:1025A0000C7300EA01210B4313436422284602FB0B
:1025B00004740027C4F8AC340123C4F8B074C4F820
:1025C000B434C4F8B874C4F8BC74C4F8C474C4F89F
:1025D000C87468F0B7F994F8E934202BD9B21AD14D
:1025E00094F8E834012B16D0242384F8E934D4F885
:1025F000A8341A6822F001021A601A6822F4805284
:102600001A601A681A601A6842F001021A6084F8A7
:10261000E91484F8E874002196F82B0064F022FE97
:1026200096F82B3001241D4D5A0903F01F03002199
:1026300004FA03F345F8223096F82A0064F012FEFB
:1026400096F82A305A0903F01F039C4045F82240AF
:10265000BDE8F88F5CF0E4FCD9F81C30C3F302133A
:10266000984498F8AC32EBE6F44619E7013170E78C
:10267000BEF10F0FF8D1002397E700BF401E0024E2
:10268000E8220024001C0058286B6E4E0000164300
:10269000002474490000704200FFFF0000E100E0E8
:1026A00090200B080044025808B1002234E670471D
:1026B00070B50E4C94F8F865AEB104F5876400254A
:1026C00003E001352034B5420DD0237F002BF8D034
:1026D000E06800220028F4D00135217DFFF71CFEC0
:1026E0002034B542F1D1012070BD00BF04000020AC
:1026F00070B590F8EE311C09013C082C0FD81A4E29
:10270000054603F00F0306EB4402B2F8BC0240FAA0
:1027100003F2D20703D595F8F121012A01D0012057
:1027200070BD9A402644013A10406FF0E7FA96F8DF
:10273000D0320E4A034402EBC30452F83320A3887C
:1027400010691840ECD0002395F8EF2102212046B3
:1027500085F8F131FFF7E0FDD5F85021136843F01B
:1027600008031360DBE700BF90200B08042500245A
:1027700070B5154BBFF34F8F144903F58652C1F85E
:10278000683220339342FAD1BFF34F8FBFF36F8F7C
:102790000F4C40F22A430C4AB4F8E45304F5667037
:1027A0002946FEF703FA034618B1002384F8E633FE
:1027B00070BDD4F89863294604F5667001227362EF
:1027C000BDE870406BF0F2BEC095012400ED00E062
:1027D000401E0024014B53F8200070475040005821
:1027E000014B43F8201070475040005819481A4BCD
:1027F00001681A4A41F4807130B482B00160D3F8A4
:10280000F410FF24CA2041F48031C3F8F410D3F847
:10281000F41001F4803101915321019D5462506202
:102820005162D3F8D030DB010CD40C4B00220C49A0
:102830005A659A65DA651A665A669A66196502B02B
:1028400030BC7047126D064B9A42EED102B030BCDC
:10285000704700BF0048025800440258004000582A
:10286000316665422DE9F84FD0F85C710446534B50
:1028700000F59676FDB227F0FF09826800F1E00AC4
:10288000103D4846D2F80080A3FB05352D092946A6
:1028900067F0C4F8D4F81C210023B2F5807F84F8D7
:1028A00020317FD00DD8102A00F084805DD8012A15
:1028B00046D0042A16BF6FF400616FF008013C2374
:1028C0000EE0B2F5805F71D0B2F5803F3BD0B2F53B
:1028D000806F15BF6FF400616FF008013C23042383
:1028E000324608F11806404656F803C001EA0C01CA
:1028F000F150D4F81CB1594666F03EFDBBF5807F1F
:102900002ED024D8BBF1100F3FD037D8BBF1010F28
:1029100002D0BBF1040F34D14FF0080C336852469B
:102920002946484643EA0C0333604023C4F8E830A4
:1029300067F018F83B6843F010033B60BDE8F88F80
:102940006FF00801CCE76FF008013C23C8E7BBF546
:10295000805F22D0BBF5803F1AD0BBF5806F10D1CD
:1029600008F11C064FF0080CD8E7402A15BF6FF499
:1029700000616FF008013C230023B1E7BBF1400F79
:10298000CAD03C364FF4006CC8E74FF4006CC5E782
:1029900008F154064FF0080CC0E708F11C064FF48C
:1029A000006CBBE76FF00801042399E76FF4006146
:1029B000042395E76FF4006192E700BFABAAAAAACF
:1029C0002DE9F04F474D85B02B781BB9012005B09C
:1029D000BDE8F08F444B5C6EFFF738F995F8F83599
:1029E0000193002B00F0C781404B05F5C065404EB8
:1029F0000027A3FB042300955B09A6FB03263D4AA1
:102A0000F60802F2347806EB8606A3EB4606D2F807
:102A1000483BC11A1346F2B203F6142A08EB8606A5
:102A200089460392B9F1000F05DB009BD3F82431EE
:102A30004B4500F387814FF4B4732A4A03FB072305
:102A400093F82037002B00F0BF80009D2A48D5F86E
:102A50005C11AB681A68CBB221F0FF01103BA0FB00
:102A6000030326481B09C35C0B44A9895C68D3682F
:102A7000A4B223EA0103C4F11604D360072C40F288
:102A8000A3801C4A0121D5F86451D2F81C3A8B4628
:102A9000AE4602970133C2F81C3A002228689446D9
:102AA00014E0BCF1140F2BDC13F1080748BF03F14D
:102AB00017073B110CEB271C5F1E013102FA03F3D1
:102AC0000BFA07F78C4247EA030219D303468C42FC
:102AD0005EF8040FA0EB0303E3D8CCF115034FF02D
:102AE000150CE9E704000020401E00241F85EB516F
:102AF000CDCCCCCCFC100020ABAAAAAA18F40B08B1
:102B0000BCF1150F029F40F013819F48C2F384234C
:102B1000C2F3441100EB830300EB8101D3F8DC32F4
:102B2000D1F8DC121B0243EA011302F01F01C2F3C9
:102B3000C43200EB810100EB8202D1F8DC12D2F842
:102B4000DC220B4343EA023383EA132282EA1212A5
:102B500002F00F020F2A40F0EB80C3F30F134FF681
:102B6000FF72934200F0E480B3F5606F00F0EE80F6
:102B7000AAF80C3098F858200398824210D0B16817
:102B8000D8F80020521AC8F80020D8F80420316B79
:102B9000521AC8F804200022B260326388F8580044
:102BA000D8F800200132C8F80020B2680132B260C3
:102BB0004FF6FF72934207D1D8F804300133C8F8BA
:102BC0000430336B01333363009C013708F15C0838
:102BD0005C3620460AF1140AFFF744FE04F5B4738C
:102BE0000093019BBB427FF41DAF68490122002383
:102BF00081F8182BC1F8483B6549D1F8083691F89F
:102C0000D8261B6812F0020FD1F81C171A6A0CBFE5
:102C10000A4342EA81021A62019B012B3FF4D6AEBD
:102C20005B49D1F8703791F840281B6812F0020F09
:102C3000D1F884181A6A0CBF0A4342EA81021A6268
:102C4000019B022B3FF4C2AE5149D1F8D83891F81C
:102C5000A8291B6812F0020FD1F8EC191A6A0CBFF0
:102C60000A4342EA81021A62019B032B3FF4AEAE93
:102C70004749D1F8403A91F8102B1B6812F0020F27
:102C8000D1F8541B1A6A0CBF0A4342EA81021A6245
:102C9000019B042B3FF49AAE3D49D1F8A83B91F833
:102CA000782C1B6812F0020FD1F8BC1C1A6A0CBFFA
:102CB0000A4342EA81021A62019B052B3FF486AE69
:102CC0003349D1F8103D91F8E02D1B6812F0020F46
:102CD000D1F8241E1A6A0CBF0A4342EA81021A6222
:102CE000019B062B3FF472AE2949D1F8783E91F84A
:102CF000482F1B6812F0020FD1F88C1F1A6A0CBF04
:102D00000A4342EA81021A62019B082B7FF45EAEFD
:102D1000204A52F8203C92F8B0001B68D2F8F41018
:102D200080071A6A4CBF42EA81020A431A624DE6E2
:102D3000164AD2F8183A0133C2F8183AAFB14FF632
:102D4000FF7317E7002005B0BDE8F08F12494A78FD
:102D500002EB420201EBC2023A44527C0D2A7FF49C
:102D600007AF80228AF81E2004E7294658220B4824
:102D70006EF0EEFDE3E719460122044BC3F8481B51
:102D800083F8182B22E600BF90200B08FC100020CF
:102D90000400002004100020401E0024BC1B002062
:102DA000464A92F8481B013949B24B1C00F0848016
:102DB000434B480103EB411100B5C2F84C1B811D88
:102DC00013F801E003EB010C92F8501B8E455BD029
:102DD0009CF802E08E4555D000F10A0113F801E09D
:102DE00003EB010C92F8511B8E4546D09CF802E093
:102DF0008E4540D000F10E0113F801E003EB010C09
:102E000092F8521B8E4531D09CF802E08E452BD0B3
:102E100092F8461B31B300F1120113F801E003EB05
:102E2000010C92F8531B8E4535D09CF802E08E457C
:102E30002FD000F1160113F801E003EB010C92F81A
:102E4000541B8E4533D09CF802E08E452DD01A30AD
:102E500092F8551B13F800C003448C4521D0987894
:102E600088421DD05DF804FB0CF1020CBCF8001088
:102E7000A2F8581BCCE70CF1020CBCF80010A2F829
:102E8000621BB7E70CF1020CBCF80010A2F8601B43
:102E9000A2E70CF1020CBCF80010A2F85A1BC8E71C
:102EA00002331B88A2F85E3BDCE70CF1020CBCF895
:102EB0000010A2F85C1BCAE7704700BF401E002448
:102EC000EC230B080120704738B5134D41F20D1368
:102ED000124941F28832D5F8A80BD5F8644B0004AA
:102EE000A060E068014020460B430D21E3605CF0E8
:102EF00081FE38B1D5F8982B034600201343C5F85E
:102F0000983B38BD606900F4F050A0F50060B0FA5D
:102F100080F0400938BD00BF401E0024C0E0FEFF25
:102F2000C74BD3F8E01BD3F8E42B70B58C0F93F8A4
:102F3000685C100EC2F3072C83F8104CC1F3836455
:102F40000001012D83F8114CC1F3016483F8124C88
:102F5000C1F3074483F8134CC1F30724C9B283F8C3
:102F6000144CC2F3035483F8151CA3F8160CC2F3D7
:102F7000C030B3F8161C89B241EA0401C2F303441D
:102F8000A3F8161CC2F3403183F8184CC2F3803406
:102F900083F8190C4FF0000083F81A4C83F81B1CBF
:102FA000C2F3003183F81C1CD3F8E81B83F81D0C16
:102FB00040F2EF80022D00F0C3802A204FEA4C0C33
:102FC00083F8294CC1F3C01201F07F010CF07E0C94
:102FD00083F82ACC4FF0010C93F82A4C1443D3F811
:102FE000EC2B83F82A4CD40F83F82B1C910D83F81B
:102FF0002C4CC2F3417401F00C01C2F3815583F8EB
:103000002D4CC2F3826483F82E4C83F82F1C93F866
:103010002F1CD3F8F04B294383F82F1CC2F34051E7
:1030200083F8301C002183F8311CC2F3004183F87F
:10303000321CC2F3C03183F8331CC2F3803183F8F1
:10304000341CC2F3403183F8351CC2F3003183F8DD
:10305000361CC2F3812183F8371CC2F30121C2F36D
:10306000460283F8381CC4F3074183F8392C220E3A
:10307000090283F83ACC83F83C2CC4F30722A3F866
:103080003E1C2406B3F83E1C89B21143A3F83E1C33
:10309000D3F8F41BC3F8404C0C0ED3F8402C42EA92
:1030A0000442C3F8402C0A0AD3F8404C02F47F4291
:1030B0002243C1F30724C9B2C3F8402CD3F8405CC3
:1030C000D3F8F82B2C43C3F8404C83F8441C110E62
:1030D00083F8451C110C0906C3F8481C1102D3F8EB
:1030E000484C0A4601F47F01214392B2D3F8FC4BCD
:1030F000C3F8481CD3F8481C0A43C3F8482CC4F34F
:103100000352D3F8481C41EA1461C3F8481C93F8F1
:103110004C1C1143C4F3072283F84C1C210A01F410
:103120007061A3F84E1CB3F84E1C89B21143C4F36E
:103130004602A3F84E1C83F8502C83F851CC70BD86
:103140001204C1F3072C0D0E02F47C12C3F8202CDC
:10315000C1F30742D3F8204C44EA0524C3F8204CBD
:10316000D3F8204C22434FF40074C3F8202CD3F83A
:10317000202CC3F8604C013240F10004A40244EA60
:1031800092549202C3F85C4CC1F38034C3F8582CBB
:1031900014E74FEA8C2CC1F3C26594000CF4406232
:1031A000C1F3072C04F47F74C3F8202CD3F8202C2F
:1031B0001443CA0BC3F8204C02F00602D3F8204C8B
:1031C00044EA9174C3F8204CC1F3026483F8245C90
:1031D000012583F8254CC1F3425483F8264CC1F3F2
:1031E000824483F8274CC1F3C03483F8282C93F829
:1031F000282C224383F8282CD3F8204C93F8282C31
:1032000093F8186C023205FA02F2B540D617A2FB09
:10321000052EC3F8605C05FB06EE04FB0EEE0134E0
:10322000A2FB0424A644520AC1F3803442EACE52DF
:10323000C3F8582C4FEA5E22C3F85C2CBEE600BFF0
:10324000401E002462F070BE62F06EBED0F8E8311D
:103250002DE9F04F93F8323085B0DFF878B30446AB
:103260004FEA531A03F01F0306795BF82A200BEB91
:103270008A0916F0020622FA03F202F00102029213
:1032800004D090F8EE61003E18BF012601279F4050
:10329000C9F88070BFF34F8FBFF36F8FD4F8DC3164
:1032A0001A6822F4F8721A609A6822F001029A6091
:1032B000C9F88071BFF34F8FBFF36F8F2423D4F809
:1032C0005051A168C4F8D03100232A6822F00102CD
:1032D0002A6004F5A8722B606B60AB60C4F8D8312B
:1032E00084F8CC31C4F8D031C4F87031C4F8D4318A
:1032F0000192C4F85411B349C4E9593363798D423A
:103300004FEA832202F48052C4F858214FEA033274
:1033100002F40052C4F85C214FEA032202F48062F6
:10332000C4F8602100F0BC81227903F00101D007CC
:1033300000F1588116B10820C4F86401002940F05A
:10334000628194F8F0214AB1D4F8782142F0080261
:10335000C4F878214FF40042C4F8882113F0080F14
:10336000D4F8D0314FF024030198C4F8D0312B6841
:1033700023F001032B6000F083815CF0E5F9012864
:1033800017D0D4F87831002B40F08E816B6823F48D
:1033900090436B60AB6823F02203AB60AB6843F0F3
:1033A0000803AB602B68019843F001032B6066F0C3
:1033B000F7FB2379DB0775D5D4F82C81B8F1000F22
:1033C00000F04B8100234FF4807CC4F83C802366DE
:1033D000E366C4E91133C4E91433C4E91933D4F8FA
:1033E0003431C4F8B8304FF48063E3644FF4803371
:1033F000C4E916C304F13C031846039367F01EFFAB
:1034000003985AF0ABFC039BC4F8C831019B636777
:10341000D4F8D431202B41D1E368626998B2EAB381
:10342000B0FA80F14909C8B394F8CCC1BCF1010FDE
:1034300034D04FF0220CC4F8D811A4F8AC0101200C
:10344000C4F8D4C1DFF890C1C4F8A821C4F878C08A
:10345000DFF888C1C4F88C10C4F87CC0DFF880C1E4
:1034600084F8CC01C4F888C094F870C084450CD0AE
:1034700084F8700094F87100012800F01D814FF469
:10348000006384F87010C4F890301023C4F8D83169
:10349000002384F8CC312023C4F8D031D8F804308C
:1034A000C4F84431002E00F08780D4F83061002E3B
:1034B00000F0BF80002304F1B405C4F8B460C4F880
:1034C000C0302846C4F8D030C4E93233C4E93633BA
:1034D000C4E93833D4F83831C4F8B8304023C4F8DC
:1034E000BC304FF48063C4F8C4304FF48033C4F868
:1034F000D43067F0A3FE28465AF030FC002840F094
:103500009080019B304AC4F8EC30304BC4F8C45171
:10351000964218BF9E4202F118020CBF01230023FD
:10352000964208BF43F001031832964208BF43F0A9
:1035300001031832964208BF43F001031832964245
:1035400008BF43F001031832964208BF43F001035D
:103550001832964208BF43F0010302F556729642B4
:1035600008BF43F001031832964208BF43F001033D
:103570001832964208BF43F001031832964208BF42
:1035800043F001031832964208BF43F0010318329A
:10359000964208BF43F001031832964208BF43F039
:1035A00001033BB90A4BF31AB3FA83F35B09002B0F
:1035B00000F09A8000237360029B002B46D105B077
:1035C000BDE8F08F000C00582800024010000240B7
:1035D000B804024000E100E03DA9090871A909080A
:1035E00075A909080420C4F86401DEB900293FF474
:1035F000A8AED4F8781141F00201C4F878114FF464
:103600008031C4F8801192077FF59BAED4F8782101
:1036100042F00102C4F878214FF40032C4F87C2152
:103620008FE6FEE70C20C4F8640100293FF489AE60
:10363000DFE7D4F8DC311A6842F080021A601A68B9
:1036400042F040021A60029B002BB8D0C9F880718A
:103650004BF82A7005B0BDE8F08FD4F8DC311A6859
:1036600042F480721A609A6842F001029A601A6805
:1036700042F020021A601A6842F010021A6011E744
:103680005CF062F801283FF494AED4F878317BB94D
:103690006B6823F490436B60AB6823F02A0380E6E9
:1036A0000422C4F874213FE601985CF04BFA6DE601
:1036B00001985CF047FAEBE79BB2039805F124010F
:1036C0005AF0ECFC00287FF4E0AE84F8CC012B68C3
:1036D00043F480732B60AB6843F00103AB60AB68CD
:1036E00043F04003AB60D9E6736065E738B5040981
:1036F000013C082C1AD80F4D00F00F0305EB4402D3
:10370000B2F8BC0240FA03F212F0010210D001221A
:10371000254402FA03F3013B18406EF0EFFA95F8E6
:10372000D032054A034402EBC30038BD002038BD47
:10373000104638BD90200B08042500242DE9F047E1
:10374000984D05EB0013D3F86C4C002C00F08F80E3
:10375000B3F8767C06464FEA0019384663F0AEFDB2
:1037600001227B0907F01F07023BBA40082B0FD844
:10377000DFE813F0BF00C700CF00D700DF0009006B
:10378000E700EF00B7008849CB6F23EA0203CB675D
:1037900005EB0903013693F8700CF6B2FFF7A6FFAC
:1037A000074610B11223C671837105EB090393F824
:1037B000710CFFF79BFF824610B11323C671837112
:1037C00005EB090393F8720CFFF790FF804610B1E8
:1037D0001423C67183714D4450462E2195F8742CE4
:1037E000FEF7BEFD95F8752C40460E21FEF7B8FD9C
:1037F00095F8732C2E213846FEF7B2FD23686B4AEC
:1038000023F001039442236033D0694B9C423ED1A4
:10381000654BD3F8902042F48042C3F89020D3F84F
:10382000902022F48042C3F89020E36843F00043E4
:10383000E360A36823F4F073A3602368DA0716D467
:10384000A1685C4A5C4B0A401343A360E368DB0059
:1038500042D5E268594B134043F0E863E3602368C4
:1038600023F400632360236D23F001032365BDE887
:10387000F0874D4BD3F8982042F48052C3F898203B
:10388000D3F8982022F48052C3F89820CDE74C4B0F
:103890009C4213D04B4B9C4263D04B4B9C426ED10D
:1038A000414BD3F8982042F48012C3F89820D3F803
:1038B000982022F48012C3F89820B6E73A4BD3F848
:1038C000902042F40042C3F89020D3F8902022F4D4
:1038D0000042C3F89020A8E7236843F48053236094
:1038E000B7E73149D1F89C3023EA0203C1F89C3094
:1038F0004EE72D49D1F8983023EA0203C1F89830F9
:1039000046E72949D1F8903023EA0203C1F8903004
:103910003EE72549D1F8943023EA0203C1F89430F8
:1039200036E72149D1F8803023EA0203C1F880301C
:103930002EE71D49D1F8843023EA0203C1F8843010
:1039400026E71949D1F88C3023EA0203C1F88C30FC
:103950001EE71549D1F8883023EA0203C1F8883000
:1039600016E7114BD3F8982042F40052C3F8982080
:10397000D3F8982022F40052C3F8982055E7134B4F
:103980009C427FF452AF03F50C33D3F89C2042F0F5
:103990002002C3F89C20D3F89C2022F02002C3F818
:1039A0009C2042E7401E00240044025800300140A1
:1039B00000380040E0FFBF8F07000020FFFF39D82C
:1039C000003C004000340140005001400014005809
:1039D00008B51D20FFF78AFE10B190F9063053B1EB
:1039E0001E20FFF783FE10B190F9063003B108BD29
:1039F0005523C38008BD5523C380F1E72DE9F04F5F
:103A0000DFF8D0A29BB09AF8CC1C31B1A74B93F849
:103A1000804320461BB0BDE8F08F01247C220AF6CB
:103A200064308AF8CC4C6EF089F8DAF84C5B4FF4CD
:103A300080529AF8466B2C68CAF86C2BCAF8644B13
:103A40001EB14FF48042CAF8702B994A4FF40037E8
:103A50000121C2E905719AF8942B002A00F09781A0
:103A60000322944F8AF8942BFA6CD60340F13481E8
:103A70000AA85BF00FFB0C988F4A010AA2FB0121F8
:103A800009094D006668A8428C4A02EA060242EA29
:103A900001026260226842F00302226080F0F88036
:103AA000DAF82016DAF82026521A022AFAD9002269
:103AB00083497E4E0492A260E2681140D6F88423C6
:103AC00041F48051E1607F49A1FB021B41F2883241
:103AD0004FEA5B2B02FB0BFB5A46002A00F0BE802C
:103AE000616B013A0806F8D5774A7549A2634FF42D
:103AF000D572A260E268114041F208120A43E26006
:103B0000BBF1000F09D05A46616B11F0450F02D08E
:103B1000890440F18881013AF6D10022CAF8A02B2D
:103B2000A260674AE1680A4042F48052E2605A4665
:103B3000002A00F09380616B013A0D06F8D5624AC5
:103B40000025A26304994FF6FE72914200F2B481FF
:103B5000DFF86C915D4FDFF8708100222046A26093
:103B600041F23712E16801EA09010A433721E260B4
:103B700041F288325CF03EF8002871D1A76041F232
:103B80002912E16801EA09010A43E260BBF1000F72
:103B900008D05A46616B11F0450F01D0880404D556
:103BA000013AF7D14FF080505AE0626B510700F1B3
:103BB0000F83C4F838806169049A002902F1010278
:103BC0000492049A03DB4FF6FE708242C5D9049832
:103BD0004FF6FE72904200F291834A0040F17081EC
:103BE000226801279307CAF89C7B00F0F982002223
:103BF000DFF8CC802046A26041F20232E16801EA9F
:103C000008010A43E2605CF097F848BB626904F17E
:103C1000180304F11C09CAF8D02BA2690193CAF851
:103C2000D42BE269CAF8D82B226ACAF8DC2B41F2FD
:103C30000312A060E16801EA080104F120080A43C8
:103C4000E260BBF1000F09D0626B12F0450F02D0A9
:103C5000910440F15683BBF1010BF5D14FF00040C8
:103C600001228AF8942BDAF8982B0243CAF8982B91
:103C70002A24204686F880431BB0BDE8F08F616897
:103C800005460E4A0A406260226842F00302226042
:103C90000F49B0FBF5F5B1FBF5F1DAF8200602317A
:103CA000DAF82026121A9142FAD800E70000002420
:103CB000A029002400440258598B4F01002CC0FF5A
:103CC000C0E0FEFFD34D6210C5002000000010C10F
:103CD00010210100401E0024BD6AB96AFE6A11F479
:103CE0007C7F7A6BC1F30510C9D0C2F3CC0206F019
:103CF000010605F0030507EE900A06FB02F2012D0E
:103D0000F8EEE76A07EE102ABAEEE97A00F0898247
:103D1000022D00F0AD80002D40F083823A689506B8
:103D200040F1F7843968B7EE006A3A6BC1F3C1011C
:103D3000C2F30803584A07EE903ACA40F8EEE77A11
:103D400077EE867A37EE877A07EE902AB8EEE76A42
:103D5000C6EE267A67EE877A5049F7EE006A504D34
:103D60000A6B0A6B096BC2F3064307EE103AB8EE12
:103D7000C77A37EE267AC7EE876AFCEEE67A17EE48
:103D8000900A010AA5FB015109094D007AE6454A4E
:103D9000944200F06982444A944200F081829AF889
:103DA000600BFFF7A3FC83469AF8620BFFF79EFCBB
:103DB00007469AF8580BFFF799FC9AF85A3B0446C5
:103DC0009AF85C9B9AF85E8B0193BBF1000F05D0CB
:103DD00058469AF8612B0E21FEF79EFA2FB138460D
:103DE0009AF8632B0E21FEF797FA2CB120469AF829
:103DF000592B0E21FEF790FA002E40F0F48100219D
:103E0000B5F9040063F02EFAB5F90420002A07DBA7
:103E100002F01F04012152092448A14040F8221059
:103E2000DAF8644B1CE6626B520700F1AA82626BFF
:103E3000D3071AD4626B570601D54022A263002231
:103E400001251B492046CAF8A05BA260E268114028
:103E500041F237120A433721E26041F288325BF0C7
:103E6000C9FE00283FF46EAE9CE60122A26354E630
:103E7000DFED107A87EEA66A3A6BC2F3080307EE0D
:103E8000903AF7EE005AF8EEE77A77EEA57A77EEF9
:103E9000877A67EE867A5FE70090D0030044025885
:103EA000598B4F01007000520024024800E100E0ED
:103EB000C0E0FEFF0024744B0499914200F21E8280
:103EC0002268900700F08C81DAF89C7B032F7FF446
:103ED0008EAEDAF8C01BDAF8C42BA069000DCAF860
:103EE000A40B880F8DF82800C1F383608DF829009A
:103EF000C1F301608DF82A00C1F307408DF82B0053
:103F0000C1F30720C9B28DF82C008DF82D10110DCA
:103F1000ADF82E10C2F303418DF83010C2F3C0315A
:103F20008DF83110C2F380318DF83210C2F3403178
:103F30008DF83310C2F300318DF8341000218DF864
:103F40003510002F40F07A8140F6FC7101EA8202C0
:103F5000DAF8C81B42EA91720E92C1F3C2628DF880
:103F60003C20C1F302628DF83D20C1F342528DF82E
:103F70003E20C1F382428DF83F20C1F3C2328DF85A
:103F8000402001220E989DF840C010440CF0070C10
:103F90000CF1020C00FA0CF09DF830C00CF00F0C84
:103FA000CAF8AC0B02FA0CF2CAF8B02B520A00FBAA
:103FB00002F2CAF8B42BDAF8A80B4FF4007BDAF857
:103FC000CC2B4FF001094FEA0048C1F38030CAF80A
:103FD000B8BB8DF84100C1F3C61001F07F018DF828
:103FE000420020468DF84310D10F8DF84410C2F3E3
:103FF00041718DF84510C2F382618DF84610C2F30D
:1040000083518DF84710C2F340518DF848100021BC
:104010008DF84910C2F300418DF84A10C2F3C03147
:104020008DF84B10C2F380318DF84C10C2F3403143
:104030008DF84D10C2F300318DF84E10C2F381217E
:104040008DF84F10C2F30121C2F346028DF85010D3
:104050008DF8512041F207128DF85290C4F8088073
:10406000E16821F48F3121F49F7121F001010A43AD
:104070000721E26041F288325BF0BCFD00287FF44A
:10408000EFADC4F808B041F2101BE26810212046E1
:1040900022F48F3222F49F7222F0010242EA0B02D4
:1040A000E26041F288325BF0A5FD002840F0BC8060
:1040B000DAF820966269910100F18F804023102187
:1040C0002046A360E26822F48F3222F49F7222F02D
:1040D000010242EA0B02E26041F288325BF08AFDA3
:1040E00000284CD1C4F8088041F23712E16820461C
:1040F00021F48F3121F49F7121F001010A4337210E
:10410000E26041F288325BF075FD002837D14FF054
:10411000FF3240236262A36201301F28FCD9E26AA9
:104120002046A14922F0FF0242F06302E26200222F
:10413000A260E268114041F20D120A430D21E260D3
:1041400041F288325BF056FDC8B90AA806E0DAF8F9
:104150002026A2EB0902013200F01781626B12F4F3
:10416000957F626B40F014811204F0D500F12001BC
:10417000D4F8802040F8042B8142F9D1E7E7DAF83F
:10418000982BCAF8982B894A0121A263DAF8982B58
:1041900002432046CAF8982B8AF8941B4FF400710A
:1041A000814AA160E1680A4041F21011114341F2D5
:1041B0008832E16010215BF01DFD00283FF458AD0E
:1041C0007A4AA2630122CAF8980B8AF8942B4FE529
:1041D00004224FF08050A26342E54FF40060D2E722
:1041E0004FF080603CE50198FFF780FA20B19AF823
:1041F0005B2B0E21FEF790F84846FFF777FA20B1C7
:104200009AF85D2B0E21FEF787F84046FFF76EFA0D
:104210009AF85F2B00283FF4F2AD0E21FEF77CF8F0
:10422000EDE5DFED637A25E6604AA263DAF8982BC4
:104230000243CAF8982B8AF8949B19E5012F4FD1B5
:104240001204DAF8C81B02F47C1242EA11420E9200
:104250004FF40072CAF8B02B0E9A01329202CAF8DB
:10426000AC2BCAF8B42BA6E6524AD2F8D41021F4EB
:104270008031C2F8D410D16F41F48031D167D16F51
:1042800021F48031D167D2F8D41041F48031C2F8E2
:10429000D410D2F8D42002F480320392039A7EE53F
:1042A000444AD2F8DC1021F40071C2F8DC10D2F8D4
:1042B000841041F40071C2F88410D2F8841021F403
:1042C0000071C2F88410D2F8DC1041F40071C2F819
:1042D000DC10D2F8DC2002F400720292029A5EE551
:1042E000324A01214FF08050A263DAF8982B42F055
:1042F0008052CAF8982B8AF8941BB1E44FF0807072
:10430000AEE4626B520700F10D82626BD30700F1DD
:1043100004822269D2B2032A40F00182264AA263B3
:10432000626912F4604F0AD0540400F1098212F459
:10433000004F14BF4FF480504FF4803090E4120CC3
:1043400019492046CAF8A82B1204A260E26811405D
:1043500041F209320A43E2605BF0EEFC00287FF490
:104360007FAC6169019BCAF8C01B1A68CAF8C42BEC
:10437000D9F80000CAF8C80BD8F80000CAF8CC0B6E
:10438000ABE50422A263FFF7C8BB4FF00040FAE69A
:10439000130700F1D381626B910700F1CD81626B4D
:1043A000920615D5C6E100BFC0E0FEFFFF0FE01F7B
:1043B0000024744A00440258C5002000D4F880103C
:1043C000DAF8202640F8041BA2EB09020132DCD007
:1043D000626BD304F2D4DDE90C120A984FF4007B2F
:1043E0004FEA11490B9B5FFA82FE4FEA102C29F02D
:1043F000FF091BBA49EA0E092CF0FF0CDFF85CE359
:104400004CEA106CC4F838E0C0F3811EC0F34010D1
:104410001FFA8CFC8DF814E08DF81500C8B2ADF8C9
:1044200016C006938DF81C00C1F30720C1F3035199
:104430008DF81D0020468DF81E10C2F38521ADF8C1
:1044400020908DF82210C2F301218DF82310C2F3C1
:10445000031102F00F028DF824108DF825209DF82D
:104460003B20B9498DF82620C4F808B0E268114015
:1044700041F210120A431021E26041F288325BF0EF
:10448000B9FB00287FF49CAE9DF82420012F9DF8F5
:104490002510D2B2DAF8709BC9B200F0B3800322C3
:1044A000CAF8BC0B8AF8942BB9F5004F00F0C38012
:1044B000B9F5804F00F00381B9F1000F00F0C28020
:1044C000DAF8982B42F00062CAF8982BDAF8982BA9
:1044D00002B39E494FF400722046A163A2609A4A3B
:1044E000E1680A4041F21011114341F28832E16063
:1044F00010215BF07FFB002800F0DC80934AA26370
:104500000122DAF8981B0843CAF8980B8AF8942B12
:10451000FFF7AEBBDAF8780BDAF8682B0328DAF885
:104520006C3BDAF8741B09D8DAF8BCEBBEF5007FF7
:1045300004D0BEF5807F14BF042002201A436368B4
:104540000A43834919400A4342EA0902DFF8F89115
:104550000243204662604FF40072A26041F21012E2
:10456000E16801EA09010A431021E26041F2883260
:104570005BF040FB0028C1D1012241F20D1B8AF8FB
:10458000942BDAF8203601930AE0DAF8982B0243EC
:10459000CAF8982BDAF82026019BD21A013241D0B2
:1045A000C4F808800D21E268204602EA090242EAC6
:1045B0000B02E26041F288325BF01CFB0028E4D180
:1045C000626902F4F052B2F5006FE3D1002F614F3F
:1045D0004FF00101CAF8980BA7F1200218BF02257D
:1045E000CAF8900B04468AF8941B8AF8685C07F1B5
:1045F00010050FCA87E80F0017E90F0085E80F00C4
:10460000FFF737BB0A4305D00322CAF8BCBB8AF8C0
:10461000942B49E74FF48072CAF8BC2B03228AF826
:10462000942B41E74FF000410122CAF8981B8AF809
:10463000942BFFF71DBBDAF8982B42F08052CAF892
:10464000982B43E76269002000219201CDE90A011D
:104650005CD40AA861F058FF024628BB0B9AD3032A
:1046600065D5C4F8088041F23712E1682046DFF8CA
:10467000D8B001EA0B010A433721E26041F28832E7
:104680005BF0B8FA024678B9C4F80890E16841F2E4
:104690000612204601EA0B010A430621E26041F2BC
:1046A00088325BF0A7FA0246DAF8981B0A43CAF888
:1046B000982B0BE701228AF8942BFFF7D9BA002038
:1046C00062690021CDE90A0190011FD40AA861F0B6
:1046D0001BFF02460028E7D10B9A510327D5C4F8E7
:1046E000088041F23712E1682046DFF85CB001EA49
:1046F0000B010A433721E26041F288325BF07AFA1B
:1047000002460028D0D10222A260BFE74FF4006227
:10471000CAE7DFED117AFFF7ADBB0122A2630120EA
:10472000FFF79EBA04221046A263FFF799BA4FF032
:104730008062B9E7202026E5022024E5082022E552
:104740004FF40050FFF78CBAC0E0FEFFFF0FE01FF0
:10475000002CC0FF202A00240024744C3A0F0018BB
:104760002DE9F047344C94F8600BFEF7BFFF064686
:1047700094F8620BFEF7BAFF054694F8580BFEF763
:10478000B5FF94F8468B074694F85CAB94F85A0B47
:1047900094F85E4B0EB11823F3800DB11923EB8012
:1047A0000FB11A23FB80B8F1000F15D13846012153
:1047B000FDF7A6FDFDF778FF30460121FDF7A0FDCE
:1047C0002846FDF79DFD3046FDF76EFF2846012186
:1047D000BDE8F047FDF768BFFEF788FF814608B1E6
:1047E0001B23C3805046FEF781FF804608B11C237F
:1047F000C3802046FEF77AFF044638460CB11D23DD
:10480000E3800121FDF77CFDFDF74EFF4846FDF7F3
:1048100077FD4046FDF774FD2046FDF771FD01214F
:104820004846FDF741FF40460121FDF73DFF0121CC
:104830002046FDF739FFBFE7401E0024F8B50E4CB7
:1048400094F8F875A7B104F5C064C7F10907092504
:10485000013D0FD0A6683079FEF748FF94F8DC10D0
:10486000F27908B1FDF758FDAF4204F5B474EFD109
:104870000120F8BDAB68FFDE04000020F8B5044657
:10488000EFF31185502383F3128803799B0702D538
:1048900090F8EE3133B9012384F8E031EDB285F3BD
:1048A0001188F8BDD0F830311B6803F00103002BEC
:1048B000F4D1D0F8D021D0F8D4110A4302F021026B
:1048C000212AEBD0D0E909129142E4D090B24BD822
:1048D000194623691B1A9BB2A162002184F8E011DA
:1048E000D4F8D0112029D9D1A1698918D6D0B3FA2A
:1048F00083F25209002BD1D094F8CC010128CDD0FD
:104900002120A4F8A6314FF0010CC4F8D821C4F836
:10491000D001D4F8C401D4F85061C4F8A011A4F8AF
:10492000A43184F8CCC140B3194F90F834E0C76388
:10493000184FE64502650764174FC7640AD090F820
:10494000357080F834C0674511D04FF4006380F8AB
:1049500034204365102100222023C4F8D81184F8A4
:10496000CC21C4F8D03199E7081A83B2B4E706F134
:10497000280259F093FB0028ECD100234022326238
:1049800084F8CC31B36843F08003B36086E700BF9E
:1049900015A9090839A9090875A90908BFF34F8F96
:1049A0000549064BCA6802F4E0621343CB60BFF3CB
:1049B0004F8F00BFFDE700BF00ED00E00400FA05E7
:1049C0001C481D4AC1681D4B10B44FF6FF0485B04A
:1049D00021401B4C0A43C260D3F8D010D3F8DC202E
:1049E000C4F8D01C42F00052C3F8DC20D3F8DC201D
:1049F00002F000520192019AD3F8DC2042F080428A
:104A0000C3F8DC20D3F8DC2002F080420292029A44
:104A1000D3F8DC2042F00042C3F8DC20D3F8DC30CD
:104A200003F000430393039B05B05DF8044BFCF7D0
:104A3000FFB900BF00ED00E00005FA050044025890
:104A4000401E002408B51D480023C0F88430BFF381
:104A50004F8F436923F480334361BFF34F8FD0F806
:104A6000803043F6E074C3F34E3CC3F3C90E4FEA03
:104A70004C1C0CEA0401734641EA8372013BC0F806
:104A800074225A1CF8D1ACF1200C1CF1200FF0D18B
:104A9000BFF34F8FBFF36F8FBFF34F8FBFF36F8F96
:104AA0004369002223F400334361C0F85022BFF36E
:104AB0004F8FBFF36F8F72B6FFF770FF00ED00E00E
:104AC00003689B0AA3F58013522B54D870B5364C5B
:104AD00014F803C0BCF10D0F4CD843794FF04C0EC5
:104AE000324802249E080EFB0C0E0CEB8C03B440E3
:104AF000DEF8D45C0CEB4303B6463344EE68002981
:104B00003FD0344300EB83067167C6F88420EC6025
:104B1000EFF31185502383F312882C2202FB0C0142
:104B20000B6F4BB31A1DC1F89430214B0CEB8C0169
:104B3000204C0CEB410189000C4410310B4453F81C
:104B4000041F09B111600A1DA342F8D10023EDB280
:104B5000136085F311882C2303FB0C03D3F89430E6
:104B6000C3B14C2303FB0C03D3F8D42CD36843F01C
:104B70000103D36070BD70470D4B02FB0C32243231
:104B8000D4E726EA0404EC6000EB83046167C4F810
:104B90008420BDE74C2303FB0C00D0F8D42CD36851
:104BA00023F00103D36070BD90200B08401E002449
:104BB000B01E0024D01E002403689B0AA3F58013B6
:104BC000522B00D970470E4AD35C0D2BFAD84FF008
:104BD0004C0C10B40B4C42790CFB03400223D0F870
:104BE000D40CDA409340C26829B922EA03035DF885
:104BF000044BC360704713435DF8044BC3607047B8
:104C000090200B08401E002403689B0AA3F5801324
:104C1000522B10D8084AD25C0D2A0CD840790223B6
:104C200006494FF04C0CD8400CFB02128340D2F8DE
:104C3000D42CDB431361704790200B08401E0024E6
:104C400001490248FBF74CBFB01E002400000140A0
:104C500001490248FBF744BFB01E00240000014098
:104C600002494FF08040FBF73BBF00BFDC1E002431
:104C700001490248FBF734BF081F0024000400402C
:104C800001490248FBF72CBF341F002400080040F4
:104C900001490248FBF724BF601F0024000C0040BC
:104CA000F8B5164D164E2A69EB681A404FF00040D1
:104CB000B2FA82F3EAB120FA03F3012A6FEA03039E
:104CC00002EA03012B610A46F2D1D6F874718FB162
:104CD000013F0023BFB2C6F87431D6F8704134B139
:104CE00023682046394698476468002CF8D1002292
:104CF000DCE7F8BDEF6ABFB2EFE700BF001000408D
:104D0000401E002401490248FBF7EABEE41F0024CC
:104D10000004014010B5064C064804F5D271FBF7BB
:104D2000DFFE04F5FE710448BDE81040FBF7D8BE75
:104D3000401E002400040140001C004001490248BC
:104D4000FBF7CEBE102000240018004001490248A5
:104D5000FBF7C6BE6820002400200040014902483D
:104D6000FBF7BEBE942000240040014001490248E8
:104D7000FBF7B6BEC02000240044014001490248B0
:104D8000FBF7AEBEEC200024004801402DE9F041C5
:104D90004FF425728EB0002173486CF0CFFE734B38
:104DA000734D4FF00008D3F8F02040F27D27A5F5B1
:104DB0006F7605F6F41442F00102C3F8F020D3F840
:104DC000F02002F001020092009AD3F8E82042F0AD
:104DD0000102C3F8E820D3F8E82002F001020192B2
:104DE000019AD3F8E82042F00202C3F8E820D3F891
:104DF000E82002F002020292029AD3F8E82042F080
:104E00000402C3F8E820D3F8E82002F00402039279
:104E1000039AD3F8E82042F00802C3F8E820D3F858
:104E2000E82002F008020492049AD3F8E82042F045
:104E30001002C3F8E820D3F8E82002F0100205922F
:104E4000059AD3F8E82042F02002C3F8E820D3F80E
:104E5000E82002F020020692069AD3F8F02042F0F1
:104E60000202C3F8F020D3F8F02002F00202079209
:104E7000079AD3F8E82042F04002C3F8E820D3F8BC
:104E8000E82002F040020892089AD3F8E82042F0A5
:104E90008002C3F8E820D3F8E82002F080020992EB
:104EA000099AD3F8E82042F48072C3F8E820D3F8D6
:104EB000E82002F480720A920A9AD3F8F02042F4B1
:104EC0008032C3F8F020D3F8F02002F480320B9245
:104ED0000B9AD3F8F02042F40032C3F8F020D3F854
:104EE000F02002F400320C920C9AD3F8F02042F435
:104EF0008022C3F8F020D3F8F03003F480230D9320
:104F00000D9B55F82810002354F83320914226D0E9
:104F100001330E2BF8D1002008F1070862F0CEF91A
:104F2000B845EED14FF0000840F27D2755F8281023
:104F3000002354F8332091420CD001330E2BF8D1CA
:104F4000002008F1070862F0B9F9B845EED10EB0BB
:104F5000BDE8F08106EBC303B3F8B40DF1E706EB4F
:104F6000C303B3F8B40DD7E7B01E002400440258C1
:104F70004C240B08800AA0F5801052280DD8074B4E
:104F80001A5C0D2A09D8064B4C2101FB0233D3F8D9
:104F9000D42C136843F001031360704790200B0872
:104FA000401E00241F4B984210B50ED003F58063BD
:104FB00098420AD01C4A03F58043984218BF904299
:104FC00003D003F5806398421BD15AF029F8174BA0
:104FD0001749DC69DA69C4F3022CC2F3022201EB3F
:104FE0000C0393F8AC3203F01F03D8400F4B114968
:104FF0001B69C3F3C03342EAC303CB5C03FB00F07D
:1050000010BD5AF00DF8094B0949DC69DA69C4F39F
:105010000214C2F302120B1993F8AC3203F01F030F
:10502000D840E3E70000014000400140004402583E
:1050300090200B08F4F30B082DE9F04F002391B0FA
:10504000AD4C0093AD4BAE4FA3F56266AB4D4FF048
:105050000009AC4BD5F800A093F862204FEA9A23E0
:10506000A3F58013522B00F2CE80F35C0D2B00F2DF
:10507000CA80012A17F903B000F01081022A02D178
:10508000BBF1080F3BD14FF000084146584616F0DF
:105090008FFC16F015FD90F900C0BCF1000F18BF91
:1050A000BCF1540F14BF4FF0010C4FF0000C40F056
:1050B000E98008F104081FFA88F8B8F1100FE4D16C
:1050C000009B002B00F0AA808B4A0AE0F35C0D2BBA
:1050D0000ED8FB565B450ED002F58672944200F066
:1050E000998091680B689B0AA3F58013522BEDD928
:1050F00000235B45F0D14B7969799942ECD109F1F4
:1051000001091C35B9F1080FA3D1009B04F5867481
:105110000133042B009399D17B4A4FF0010B92F895
:10512000F83502F5876901330393039B5B4567D02C
:10513000744B99F81020D9F80C6093F876300092EF
:10514000002E5DD0704AD6F800A055686F48B2882E
:10515000002D504401924FEA902040F3AE80664A01
:10516000002405E0013402F58672AC4200F0A28012
:1051700011688142F6D1604B4FF48672019D02FBAB
:105180000434009B0322C9F80C6089F81030019B9D
:10519000C9F81840B3FA83F7C7F11F035800C9F8DC
:1051A0000430B27186F807B002FA00F6A16C012251
:1051B000D4F854C0314302FA00F002FA03F3A164B8
:1051C000216D0143D4F8AC0021654F490E7899B2A6
:1051D000002E00F04E8143EA0C036365CAF81850B4
:1051E000FAF760FF0BF1010B2046FAF72FFF09F1E8
:1051F000200940F20113BBF1090F29F8043C94D1B6
:1052000011B0BDE8F08F013A012A7FF678AF4FF078
:10521000000B38E7BCF1000F7FF471AFA8680022E3
:105220003B4904E001320C31102A00F088834B68BE
:105230009842F7D152B269795046FCF765FC354A7D
:105240004068002351680133884208D0102B02F1D6
:1052500024023FF454AF516801338842F6D1DBB2E7
:105260002D4A013B03EBC30302EB830393F958314F
:10527000002B7FF444AFC9EBC909204B03EB890332
:10528000A36042E7009B002B7FF41EAF09F10109E8
:105290001C35B9F1080F7FF4DCAE36E7BBF1010F26
:1052A0003FF4F1AE09F101091C35B9F1080F7FF4A3
:1052B000D0AE2AE7042C00F049824FF48671124ADE
:1052C00001FB052211690491002900F0048390601C
:1052D00001304FF054019C46C4B20D4882F81011C1
:1052E00082F811416A1C08494A60049A116897685B
:1052F00002915179002216E00C000020B02E0B081C
:1053000008F40B08382F0024040000200000FEA73A
:105310007C0000243C0100240000002401320C30F9
:10532000102A00F00C8343689F42F7D152B20298D2
:10533000CDF814C0FCF7E8FB944B4FF48672DFF80D
:105340007C8202FB05310022059B0132D0E901700D
:10535000C1E9077041464868874208D0102A01F128
:1053600024013FF44DAF486801328742F6D1D2B2F2
:105370008749013A02EBC20201EB820292F958110D
:1053800000297FF43DAF4FF4867182F859410693AE
:10539000542401FB05F37F4882F858419A107E4956
:1053A000059300FB02F201F560747848C2EBC20C71
:1053B00002EBC202184401EB4C1104EB4212C0F89C
:1053C0000CA0C0F8B410C0F8FC203322C0F8B820FC
:1053D0008C22C0F80021714A0298D418FFF7E2FD30
:1053E000069B062B00F0B981072B6D496D4B6E4A69
:1053F00018BF1A466D4B18BF0B464FF48671DDF887
:1054000008A0B0FBF3F3B0FBF2F2013B5F48013AB6
:1054100001FB05019BB2A1F8BC20A1F87430236602
:10542000059B03F1580100F108035046194400237D
:10543000A4F858306366E36564F01CF9DAF80030CC
:1054400043F08003CAF80030049B5B791A46069348
:105450000C2A1CD8DFE812F003021B001B001B0003
:10546000DD011B001B001B00BB011B001B001B0000
:105470009601C7F12F072D0402FA07F3324643EADB
:105480000C036365CAF81850FAF70CFEAAE63F4A07
:105490004FF4867302984FF0000A03FB05230222A3
:1054A000CDF828A059690368079123F00103CDF8CE
:1054B00034A0CDF83CA00360602308934FF48073C0
:1054C0000E93012309930A23CDE90B3208AA63F056
:1054D00053FF0799B1F5807F00F0288240F24081A8
:1054E000B1F5805F00F00E82B1F5803F00F00482DC
:1054F000B1F5806F15BF4FF4006308234FF03C0AED
:105500004FF0040A029A183252F80A100B4342F87C
:105510000A30049B1879002840F0CB81029A136866
:1055200043F0010313600023D8F8042001339742AD
:1055300000F0BC81102B08F12408F5D14FF0FF33A7
:105540000027134A03EBC30302EB8303D3F83C01A8
:10555000174B984214BFA120A02061F0AFFE069A1D
:105560000C2A00F2A081134B03EB4203B3F800CFE7
:105570004FF48673054A104803FB0523DDF808E065
:1055800000F53261A3F818C0002320E004000020D9
:10559000000000246B4CA407C08D01240C000020E7
:1055A000D0DD0600449508001055220040771B000E
:1055B0000000024090200B08FC1000203C01002459
:1055C000964500F09D810133042B00F0BB8151F81A
:1055D0003320002AF4D1D0F81C2B0132C0F81C2B48
:1055E00000EBC300029ADB00C0F8202B19443846B8
:1055F000234690228F884CEA070C0027A1F804C0AC
:10560000C349FCF7F3FA4FF48673C24A40214FF4C2
:10561000403CC14803FB052A4FF48052DAF81C5085
:105620002B6843F010032B602B6843F014032B60AE
:10563000C4E91F77C4E92777C4E92977DAF820306D
:10564000A167E9B2C4F89430069310394FF480632F
:10565000C4F898C0A0FB01014FF4804CC4F884301A
:10566000DAF8B8000909059BC4F8900025F0FF009E
:10567000DAF80C80C4F8882008F11802049102902E
:1056800008F11008226703F17002A44B1A44DAF8FB
:10569000B430C4F88CC0636764F064F9D5F800C016
:1056A000059BC4F820C0D5F814C003F1B8029B4B89
:1056B000C4F824C0D5F804C01A44069BC4F828C016
:1056C000D5F808C00499C4F82CC0D5F80CC0C4F8AB
:1056D000DC304FF48063C4F8C870C4F8CC304FF4A9
:1056E0000033C4F830C0C4F8E0300298C4E9307721
:1056F000C4E93977C4E93B774FF40067DAF8003141
:10570000C4F8B880C4F8D0704FF48047C4F8D830DB
:10571000DAF8FC30C4F8D470C4F8BC3064F022F974
:105720002B68D6F800A063636B69A3636B68E363BF
:10573000AB682364EB6863642B6843F010032B6051
:105740002B6843F014032B60B5881AE50323744AD1
:1057500082F8773011B0BDE8F08F724A724B4CE698
:10576000102900F0E98000F2BD80012900F0E280FC
:10577000042915BF4FF4006308234FF03C0A4FF093
:10578000000ABFE602984FF4867262494FF0020A9F
:10579000036802FB05124FF4805123F001035161AD
:1057A00008AA036000230A930D930F9360230893C4
:1057B0004FF480730E93012309930A23CDE90B3A2A
:1057C00063F0DAFD4FF0040A4FF400639AE60298A2
:1057D0004FF486724F494FF0020C03684FF0040AF1
:1057E00002FB05124FF4807123F001035161602226
:1057F000036000230E910A930D930F930123CDE9CB
:1058000008230A2308AACDE90B3C63F0B5FD082361
:1058100078E602984FF486723E494FF0000A03681A
:105820004FF0020E02FB0512102123F00103CDF808
:1058300028A0516108AA03606023CDF834A0089322
:105840004FF48073CDF83CA00E93012309930A23F3
:10585000CDE90B3E63F090FD4FF4006352E60298F1
:105860004FF486722B494FF0000A03684FF0020E86
:1058700002FB0512012123F00103CDF828A051619C
:1058800008AA03606023099108934FF48073CDF850
:1058900034A00E930A23CDF83CA0CDE90B3E63F073
:1058A0006BFD08232EE64FF0000C61E6DFB27B1E95
:1058B00047E6FDF71BFF824638B1049B0221DA79E7
:1058C000FCF72AFD5423AAF80630029A536C43F4DD
:1058D0000043536422E60223114A82F8773011B064
:1058E000BDE8F08F402915BF4FF4006308234FF047
:1058F0003C0A4FF0000A05E608234FF03C0A01E697
:10590000DB0073E64FF400634FF0040AFAE500BFD2
:105910000100000004000020ABAAAAAA0C0000208D
:10592000382F0024882A1100A0BB0D0008234FF057
:10593000040AE7E50823E5E54FF40063E2E5002308
:105940005B68FFDE00239B88FFDE00BF2DE9F04F80
:10595000B04D8FB095F87880B8F1000F03D10020DA
:105960000FB0BDE8F08F00222F21404616F0FEF860
:1059700006460028F3D090F80590A74FD0F800A075
:10598000A7F8E493FCF7EAF80028E8D0D0E901434F
:105990000193002CE3D0DFF8B8B20022594601E0B1
:1059A000102ADCD04B68013224319C42F8D1D2B2AB
:1059B0009A4B013A02EBC20203EB820292F9583190
:1059C000002BCCD12F2150460293A2F85811C7F8D2
:1059D00098A3FFF7E7FA924A029B904280F0FA8080
:1059E0001A460123039350460292FFF7DBFA029A0C
:1059F000039BC7F89C238B49B0FBF3F2120A8A4839
:105A0000A1FB02210022C7F8A823C7F8A0230A0996
:105A10000909A0FB0202C7F8A4135208A5F87C20CC
:105A20005200A5F87A2097F8D52302F0FF01002A4A
:105A300000F0DE80022250467C4987F8D52359F0D9
:105A4000C5FD0122404687F8E02387F8D62387F872
:105A5000D72387F8D82387F8D92387F8DA2387F85C
:105A6000DB2387F8DC2387F8DD2387F8DE2387F83C
:105A7000DF2387F8D523FDF739FEC5F8800028B16C
:105A80002F21C1804E21F279FCF746FC684A0021A3
:105A9000019B4FF4806CC5F89010B9F10C0FC5F85C
:105AA000A010C5F8A810C5E92143C5E92C11D2F80A
:105AB000D80040F00100C2F8D800D2F8D80000F0B9
:105AC000010004900498D2F8D80040F00200C2F817
:105AD000D800D2F8D82002F002020592059A4FF0C1
:105AE0004002C5F88C204FF48052C5E925C24FF41E
:105AF0008042C5F89C204FF40032C5F8A4204FF036
:105B00000302C5F8AC2076D84A4A02EB4902B2F843
:105B10001C8FC246484A08F108084849C5F8BC200D
:105B200007EB8802C2F89813594600224B680132ED
:105B300024319C4262D0102AF8D14FF0FF32374B0B
:105B400002EBC20203EB8202D2F83C013C4A9042D3
:105B500014BFA120A02061F0B1FB0022DBF80430CB
:105B600001320BF1240B9C424BD0102AF6D10020BD
:105B700007EB8807534660223249FCF737F8D7F81D
:105B8000980358F0EBF800287FF4E9AEB4790027C9
:105B900060260C9063004A4606A9274803F00203DA
:105BA0000893E300CDE9066703F008030026002709
:105BB0000993CDE90A6760F037FD00287FF4CFAE86
:105BC000A30749461C481ED559F074FDB0FA80F071
:105BD0004009C5E65046FFF7E5F91B4A1B49024458
:105BE000A1FB0212920D531E9AB2531C0393FAE6C4
:105BF00087F8D4131EE78A4688468BE7D2B2013A6B
:105C00009DE7D0B2B4E759F055FCB0FA80F04009F6
:105C1000A6E600BF382F0024401E00240000002408
:105C2000006CDC02598B4F01ABAAAAAADC2100242C
:105C30000044025890200B08D8210024BC2F0024D7
:105C400000000240D502000000366E01819F5E1602
:105C50003C010024830AA3F58013522B00D970471E
:105C60002DE9F04115460F4AD65C0D2E17D80E4C83
:105C70004FF04C08013908FB064789B2C7F8E01C11
:105C8000FFF790F907F6D841B0FBF5F2013AD7F8E3
:105C9000D40CC7F8D82CBDE8F04159F097BCBDE84A
:105CA000F08100BF90200B08401E0024830AA3F55A
:105CB0008013522B6ED82DE9F0439046714A85B07F
:105CC000D65C0D2E63D84C256F4F044606FB05F5B8
:105CD00007EB0509D9F8D43C834258D00139C9F8FB
:105CE000D40C083589B2C9F8E01CFFF75BF907F658
:105CF000D4410023B0FBF8F00D440138C9F8DC3C76
:105D0000C9F8D80CC5E9023399F8113D03F0FF0238
:105D1000002B40D04C25022305FB061105FB067520
:105D20000431D5F8D48C85F8113D404659F04EFC2D
:105D3000012385F81C3D85F8123D85F8133D85F853
:105D4000143D85F8153D85F8163D85F8173D85F815
:105D5000183D85F8193D85F81A3D85F81B3D85F8F5
:105D6000113D4A4B9C4219D0B4F1804F16D0A3F597
:105D70007C439C4212D003F580639C420ED003F515
:105D800080639C4260D003F578439C425CD005B0B0
:105D9000BDE8F083704789F8102DBBE74C2303FB67
:105DA000067393F8102D012AF1D0022283F8112DE9
:105DB000374AD8F808100A40C8F80820012283F8AA
:105DC000112D002283F8102D00224C232F4903FBB4
:105DD000067303928845CDE901224FF0020283F851
:105DE000112DD8F80420D8F8083028D001F58061AA
:105DF000884524D022F07002C8F80420254A904536
:105E00000DD0B8F1804F0AD0234902F500629045C9
:105E100018BF884503D002F54062904503D123F0B6
:105E20008003C8F808304C230121002203FB0673CD
:105E300083F8111D83F8102D05B0BDE8F0831749D4
:105E40001140C8F80410EAE74C2303FB067393F8EB
:105E5000102D012A9BD0022283F8112D0C4AD8F86C
:105E600008100A40C8F80820012283F8112D0022EA
:105E700083F8102D0A4B9C42A6D003F578439C4230
:105E8000A2D084E790200B08401E002400000140AF
:105E90008800CEFF00040040000800408FFF0FFF85
:105EA000000C00402DE9F0410468A30AA3F580131B
:105EB000522B03D82C4DEE5C0D2E01D9BDE8F0819C
:105EC0002046FFF7F3FE4C22284B02FB063393F8E3
:105ED000112D012A10D00023254951F83320944276
:105EE0001CD001330E2BF8D10121002061F0BAF94A
:105EF000204B01221A60E1E70221D3F8D42C83F869
:105F0000111D1D4B91680B40062BE4D0B3F5803F6B
:105F1000E1D0136843F001031360DCE705EBC30530
:105F20000126144F95F8B64D314604F01F05204662
:105F300061F098F91B2C4FEA541806FA05F547F85A
:105F4000285009D02E2CB9D131462C2061F08AF985
:105F50004FF480537B60B1E73146192061F082F93C
:105F60004FF000733B60A9E790200B08401E00240F
:105F7000402E0B0800E100E007000100F8B5134CCB
:105F800094F8363403F0FF05002BF9D1104B0126AD
:105F900093F8FC3084F8366403B9F8BD0D4AB4F8C0
:105FA0003474138E34320C483946FAF7FFFD034639
:105FB00010B184F83654F8BDD4F8E8433246394677
:105FC00005486362BDE8F84068F0F0BA401E00245E
:105FD000382F0024804001242822002437B590F86F
:105FE00067380446032B2FD10023204D8DF807304E
:105FF0009DF8073094F868289A4201D803B030BD64
:106000009DF8073005EBC30393F804318BB181F0A1
:10601000010383B19DF8073005EBC303D3F80001FA
:10602000FCF76EF99DF807300133DBB28DF80730CD
:10603000DEE70B46EDE79DF8073005EBC303D3F829
:106040000001FCF763F9EDE7D0E910039B7903F059
:106050000103994204D003B0BDE83040FCF750B9C9
:1060600003B0BDE83040FCF751B900BF382F002421
:1060700038B5044600790D4650B1FDF737FB08B13D
:106080000323C380E2792946BDE83840FCF768B9AC
:1060900038BD10B504462221FFF7EAFF2046FEF77F
:1060A000B3FD20460121BDE81040FEF785BD10B5C7
:1060B00004460121FFF7DCFF00212046BDE8104027
:1060C000FEF77ABD38B510F8133CA0F66C041BBB84
:1060D00094F858388BBBD4E909239A421CD05A1C37
:1060E000A169A262CB5C21695B008A4228BF0022C1
:1060F00043F40073A262A4F85C380A2384F85A3887
:10610000012384F8583894F86738012B01D0042B08
:1061100002D1606CFFF7CBFF94F85438002B6DD19F
:1061200094F855380133DBB2092B84F8553825D162
:106130002046BDE83840FAF78DB894F95A586DB149
:10614000B4F85C18013D20464B0801F00101A4F8A9
:106150005C38FFF743FF84F85A58DDE7D4E9092398
:1061600084F858589A42D7D194F86738012B01D057
:10617000042BD1D1606CFFF78CFFCDE70A2B3DD10A
:1061800094F857382BB9B4F85E3843F00103A4F8FB
:106190005E382379D9070AD5B4F85E08820501D4A0
:1061A000C30718D4B4F864380133A4F86438012262
:1061B000002384F8542894F8572884F85538012A85
:1061C0001CD16179606C84F8573801F00101BDE899
:1061D00038405FF07BB8E36AC0F3470013B1216B2E
:1061E0009847E4E7E3696269D054E369E268013300
:1061F000B3FBF2F102FB1133E361D8E738BD2DE9BF
:10620000F84310F8133CA0F66C047BB1B4F8603886
:1062100001339BB2082BA4F860381BD90021606CB5
:1062200084F85918A4F860185FF050F8374F97F8C1
:106230004081B8F1000F03D101212046FFF7CEFEC7
:1062400094F858384BBBD4E909239A4204D100236F
:1062500087F84031BDE8F883B8F1020F12D808F191
:10626000010814BFFF237F2387F84081A4F85C381E
:106270000823606C84F85A38012384F85838BDE844
:10628000F84314E75A1CA169A262CB5C2169DBB216
:106290008A42EBD30022A262E8E794F95A685EB31F
:1062A000B4F85C9897F8415119F001010BD0012D19
:1062B00001D8012103E0AB1E012B09D800212046A3
:1062C000FFF78CFE04E015F0FD03F2D0012BF6D0B1
:1062D0000135EDB2032D87F84151BBD9013E4FEA9C
:1062E0005909002376B2A4F85C9887F8413184F804
:1062F0005A68002EA7D0ADE7D4E909239A42A9D164
:10630000606C84F85868BDE8F843C2E6382F002472
:106310002DE9F043BFB0BFF35F8FA24A0020516A5E
:106320000346044621F4803151620146C2F89400CC
:10633000C2F898300133C2F89C10112BC2F8A0109B
:10634000F6D10523C2F89430536A43F48033536284
:10635000BFF34F8FBFF36F8F9348944A9449121A3B
:106360006BF0F6FA9348944A9449121A6BF0F0FADB
:10637000934BDA6D042A00F0FB8005D8012A00F067
:106380009283022A00F0A583864A00238D4C0120C7
:10639000D2F888108C4E41F470018C4DC2F88810F0
:1063A00020602361216841F0800121602168014360
:1063B0002160216841F480312160216841F48051DD
:1063C0002160A361E3612362A362E36223636363E9
:1063D000A363E36323646364216821F48021216063
:1063E0007B492366C1F808014FF000614FF6FF00BA
:1063F000784B9160D16801400B43D36058F0EEFDBB
:10640000A36902460F20C3F30323A169334493F821
:10641000AC3203F01F0322FA03F3C5F8843357F0BC
:106420001BF96D4AD36813F0040FD36840F0A280C3
:106430006A4B0021684A0591D96A21F00101D962AD
:10644000DB6A03F001030593936943F440439361CE
:10645000936903F440430593059B93699B04FCD522
:106460004C2200210EA85E4C6BF068FB5D4A42F2A4
:1064700003031268B3EB124F4FF000030893A4F12B
:10648000140308BF1C46E268002A4DD0534B524902
:10649000D86A20F00100D862DB6A03F00103089398
:1064A0008B6923F4404313438B618B6903F44043AE
:1064B0000893089B484A93699F04FCD5414B4FF4CD
:1064C000403749480321D3F8E02042F08002C3F866
:1064D000E0200122D3F8E03003F080030793079B0C
:1064E00087610D9B00910193002364F079FA0223E8
:1064F00022690EA8CDE91733A3781E9201221993C1
:10650000A3881A93A3791B93E3791C93237A1D9391
:1065100000231F934FF48033CDE90E2358F0A6FAE1
:1065200003283BD098B1FEE72B4A2C4B916941F4EC
:1065300040419161926902F440420892DA6A42F065
:106540000102DA62DB6A03F001030893B1E7274B2B
:106550001A6812F00E0F4DD11A6822F00F0242F0A5
:1065600002021A601B6803F00F03022B42D0FEE701
:10657000DC6509E723F007031D4C43F00203D360F9
:10658000D4F8201606E0D4F820365B1AB3F57A7FEB
:106590003FF64EAF53689804F5D549E772B6FEF75B
:1065A000FDF900BF00ED00E00000000058510000C0
:1065B00080720C0800000020040000204DEF0C0841
:1065C000004000580044025890200B0800000024AE
:1065D000008000510003FA050048025800040058EA
:1065E0009C0300240010005C001C02580020005294
:1065F000401E00246E4A936903F070033F2B05D8B8
:10660000936923F0700343F040039361684AD369B0
:1066100003F070033F2B05D8D36923F0700343F0D8
:106620004003D361624AD36903F4E063B3F5806F3A
:1066300005D2D36923F4E06343F48063D3615C4AF9
:10664000136A03F070033F2B05D8136A23F070031D
:1066500043F040031362564B9A69140705D49A69B4
:1066600022F00F0242F008029A61514A936923F422
:1066700070639361136898017FF579AF136941F2F4
:1066800088304C4C23F0070343F003031361D4F824
:10669000201605E0D4F820365B1A834200F2BB8155
:1066A000136903F03803182BF4D1936903F00F0337
:1066B000082B05D9936923F00F0343F00803936176
:1066C0003D4A136803F00F03022B0BD9136823F024
:1066D0000F0343F002031360136803F00F03022B50
:1066E0007FF445AF324A936903F07003402B05D91C
:1066F000936923F0700343F0400393612C4AD369FC
:1067000003F07003402B05D9D36923F0700343F0E5
:106710004003D361264AD36903F4E063B3F5806F85
:1067200005D9D36923F4E06343F48063D361204A3D
:10673000136A03F07003402B00F265811C4F58F080
:106740004DFC0346D5F8B003BA69B969C2F3032218
:10675000164496F8AC2202F01F02D340C5F88433E9
:1067600056F07AFF002840F09D8110231590179075
:106770000EA80E9358F07AF9002840F043813B6848
:106780000E4A43F080033B60D7F8F43043F0020335
:10679000C7F8F430D7F8F43003F002030493049BF5
:1067A000136A43F001031362054BD4F820160CE082
:1067B00000440258401E00240020005200040058EB
:1067C00000E20400013B3FF4E9AED4F820269142F8
:1067D000F8D0D4F82026D4F820369B1A0A2BFAD900
:1067E000BF4C4FF480224FF440130EA80E924FF08E
:1067F00000082F9363F0AAFAD4F8EC3041F20302B8
:10680000B849032643F002030EA80227C4F8EC306F
:10681000D4F8EC3003F002030393039BD4F89430D4
:1068200043F00203C4F89430D4F8943023F0020308
:10683000C4F894300B68AC49B2EB134FAB4BAC4A85
:1068400028BF0A465A601A6822F47C5242F4005269
:106850001A601A6842F060021A600E96CDE92B8821
:1068600063F074FA4FF4E0430EA8CDF8E4800E9381
:10687000CDE9258863F06AFA18230EA8CDF8B88010
:106880000E93CDF8CC8063F061FAD4F8D4300522B1
:106890000EA843F48033C4F8D430D4F8D430CDF803
:1068A000588003F48033129611970293029B4FF4A1
:1068B00080330E932193FA23CDE90F230423CDE9EE
:1068C0001488139363F042FA4FF400230EA80E933A
:1068D0004FF40033369363F039FAD4F8E0303A4697
:1068E0004FF48071834843F00103C4F8E030D4F8DA
:1068F000E03003F001030993099B4346CDE90068AA
:1069000064F06EF823693A467B4823F0FE7343F047
:1069100088732361D4F8E03043F00403C4F8E03016
:10692000D4F8E03003F004030693434606994FF48D
:106930000071CDE9006864F053F8236923F07E43C9
:1069400043F0FC43236158F049FB6C4B6C4A4146D1
:10695000C5F884031846D21A6BF0F0F869486A4A01
:106960006A49121A6AF0F4FFBFF35F8F684D46461A
:10697000684C01276B6A23F480336B62C5F89480FE
:1069800023E0002946D0D4F80090637A103414F83C
:10699000060C1B0643EA007343EA410314F8051C86
:1069A00043EA814314F8041C43EA414314F8031CEE
:1069B000C5F89860013643EA0143C5F89C90032E60
:1069C00043F00103C5F8A03026D06368217A002B7C
:1069D000D7D0D4F800900029D7D129F01F01A3EB1C
:1069E0000108B8F1200F38BF4FF0200840466AF088
:1069F00073FF431E014607FA03F0804508BF19469E
:106A0000C9B2C2E7FEE7136A23F0700343F0400304
:106A1000136293E6FEE7AAE50523C5F894306B6A96
:106A200043F480336B62BFF34F8FBFF36F8FBFF3BD
:106A30004F8FBFF36F8F0022C5F85022BFF34F8FE7
:106A4000BFF36F8F6B6943F400336B61BFF34F8FFC
:106A5000BFF36F8FC5F88420BFF34F8FD5F88050F8
:106A600043F6E0762A49C5F34E34C5F3C9056401FF
:106A700004EA06002B4640EA8372013BC1F860221B
:106A8000F9D2203C14F1200FF2D1BFF34F8F4B69A4
:106A900043F480334B61BFF34F8FBFF36F8F3FB031
:106AA000BDE8F08363E50E4A02201B49D865D2F8A1
:106AB000F4300343C2F8F430D2F8F43003400E93BC
:106AC0000E9AD1F8003883F30888D1F80438984733
:106AD000FEE704210320FBF783FE72B6FDF75EFF9D
:106AE000004402580010005C7FBB2200008400407C
:106AF0007FBB22300000025800080258C029012440
:106B000080400124E0250124C029012451EF0C0814
:106B100000ED00E0B40300240090F01F10B4EFF388
:106B20001182102383F312880B4B4FF0E0200024D6
:106B3000D2B2596E0131596681699966C3F86846C7
:106B4000016982F31188D3F820265DF8044B0132E5
:106B5000C3F82026704700BF401E002410B4EFF396
:106B60001181102383F312884FF0E0229469136996
:106B700013F4803F0C4B03D00120C3F868069469DE
:106B8000586EC9B2D3F8682681F311880244D96ED1
:106B90004FF47A7000FB01F31B1B5DF8044BB3FB51
:106BA000F1F300FB02307047401E00242DE9F0474E
:106BB000DFF89080FBF74AF84FF48679002106460B
:106BC000D8F804501D4F002D2DDD00231C4609FB75
:106BD0000382013392F80521AB4244EA0204F6D164
:106BE00021435FFA81FA7B68C3F30803C3B9EFF36B
:106BF0001183ABB9F9F788FB801BB0F5FA6FCCBFF6
:106C0000002104F001010029DDD1BAF1000F04D008
:106C10000B4B93F86D26542A08D05046BDE8F087F8
:106C2000FFF79CFFE8E78A460024DCE7B3F8742608
:106C300050460132A3F87426BDE8F08700ED00E06D
:106C4000401E002404000020454B5B68C3F308038A
:106C50002DE9F0430546002B5ED1EFF31183002BA5
:106C60005AD1404B4FF0E0245A6EA069596E8A42C7
:106C7000FAD1996E8842F7D8DE6E4FF47A7101FB33
:106C800006F4241AB4FBF6F401FB0244344E102738
:106C90004FF0E02C4FF47A7E4FF001087268C2F397
:106CA0000802CAB9EFF31182B2B95A6EDCF81800C3
:106CB000596E8A42F9D1996E8842F6D8D3F86C9011
:106CC0000EFB09F1091AB1FBF9F10EFB0212121BBE
:106CD000AA42E3D3BDE8F083EFF3118287F3128871
:106CE000DCF81800DCF81010C90303D5C3F8688677
:106CF000DCF81800D3F86490D2B2D3F8681682F3A7
:106D000011884944D3F86C900EFB09F2121AB2FBB9
:106D1000F9F20EFB0122DAE7EFF31181102383F37E
:106D200012884FF0E0229669136913F4803F0D4BEF
:106D300003D00120C3F868069669586EC9B2D3F82B
:106D4000682681F311884FF47A710244D86E01FBF2
:106D500000F4A41BB4FBF0F401FB024496E700BF6F
:106D600000ED00E0401E00242DE9F0473A4B471E9D
:106D70003A4D10264FF0E0204FF47A7C4FF0010896
:106D80006A68C2F30802002A52D1EFF31182002A86
:106D90004ED15A6E8469596E8A42FAD1996E8C42EC
:106DA000F7D8D96E0CFB01FEAEEB040EBEFBF1FE74
:106DB0000CFB02EE6A68C2F30802E2B9EFF311823B
:106DC000CAB95A6E8469596E8A42FAD1996E8C4258
:106DD000F7D8D3F86C900CFB09F1091BB1FBF9F162
:106DE0000CFB0212A2EB0E02B2F57A7FE2D3013F56
:106DF000C6D2BDE8F087EFF3118286F3128884696A
:106E00000169C90302D5C3F868868469D3F864A010
:106E1000D2B2D3F8681682F31188D3F86C9051443B
:106E20000CFB09F2121BB2FBF9F20CFB0122D9E7B1
:106E3000EFF3118186F3128884690269D20302D5C7
:106E4000C3F868868469D3F864E0C9B2D3F86826C9
:106E500081F311887244A4E7401E002400ED00E095
:106E600001302DE9F84F7E4C01F1FF387D4D1026A1
:106E70005FFA80FB01275DF033FD4FF4FA794FF0A4
:106E8000E0214FF47A7C6B68C3F30803002B40F0D9
:106E9000C080EFF31183002B40F0BB80636E8869E4
:106EA000626E9342FAD1A26E9042F7D8E26E0CFB6A
:106EB00002FEAEEB000EBEFBF2FE0CFB03EE6B68B7
:106EC000C3F30803002B40F08680EFF31183002BFF
:106ED00040F08180636E8869626E9342FAD1A26E3F
:106EE0009042F7D8D4F86CA00CFB0AF2121AB2FB4D
:106EF000FAF20CFB0323A3EB0E03B3F57A7FDED388
:106F0000B9F10109BFD14FF47A7958465DF0BAFE64
:106F10004FF0E021CC466B68C3F30803002B40F030
:106F20008B80EFF31183002B40F08680636E8869BD
:106F3000626E9342FAD1A26E9042F7D8E26E0CFBD9
:106F400002FEAEEB000EBEFBF2FE0CFB03EE6B6826
:106F5000C3F308030BBBEFF31183F3B9636E8869C6
:106F6000626E9342FAD1A26E9042F7D8D4F86CA028
:106F70000CFB0AF2121AB2FBFAF20CFB0323A3EB8E
:106F80000E03B3F57A7FE2D3B9F10109C3D1B8F1A9
:106F90000108BFF470AFBDE8F88FEFF3118386F3FB
:106FA0001288D1F818A00A69D20303D5C4F868760C
:106FB000D1F818A0606EDBB2D4F8682683F311888C
:106FC0000244E06E0CFB00F3A3EB0A03B3FBF0F307
:106FD0000CFB0233D3E7EFF3118386F31288D1F869
:106FE00018A00A69D20303D5C4F86876D1F818A0AE
:106FF000606EDBB2D4F8682683F311880244E06E39
:107000000CFB00F3A3EB0A03B3FBF0F30CFB02331E
:1070100071E7EFF3118286F3128888690B69DB034D
:1070200002D5C4F868768869636ED2B2D4F868E68F
:1070300082F31188734439E7EFF3118286F31288E3
:1070400088690B69DB0302D5C4F868768869636ECA
:10705000D2B2D4F868E682F3118873446EE700BFB9
:10706000401E002400ED00E02DE9F043144C83B0F5
:10707000DFF85090DFF8508004F5906602E00834A5
:10708000B44219D094F90650002DF8D1276808347D
:1070900007EB08039B0A09EB4303B3F8980260F07F
:1070A0000DF934F8041C01232A463846CDE9005571
:1070B00063F096FCB442E5D103B0BDE8F08300BFB5
:1070C0000425002490200B080000FEA7704700BF95
:1070D0000246074B02209A4208D801335B08400061
:1070E0009A4280B202D2FF28F8D97047704700BF99
:1070F0007FF0FA0211F001010ED170B590F828501E
:1071000082B00446012D08D0C368B3F1807F01D955
:107110000123037702B070BD70470B4B466AD3F86A
:107120004401FFF7D5FFE368B080B3F1807FF1D968
:107130004FF0B70C0A4630462B4601A925778DF84B
:1071400004C051F0D5FAE5E7382F00242DE9F041CD
:107150001F46436A94B01446064618680D4665F00B
:10716000A5F90B940022274C069204F590738DF834
:1071700020201392009304F5A0730C97019302232F
:10718000CDE9092202930123CDE90E22CDE9102297
:107190001D4A8DF80C308DF834308DF8483004924B
:1071A00004F58072337F05921A1D07922BB32B0EC4
:1071B00004F5817404F8013C2B0CA570DFF84C80B9
:1071C0002D0A23706570D8F84401FFF781FF746AB7
:1071D000737FA080A3B16946204651F0CFFA746A4C
:1071E000206865F063F9D8F84801FFF771FF03469E
:1071F0003846A38014B0BDE8F08104F20114DBE747
:1072000005A9E9E7E0250124E9080408382F00244E
:107210002DE9F04F002385B0DFF800A34FF00109FE
:107220000193B94B0AF1F00BB84FA3F17C080BE0C6
:10723000019B09F101090AF1280A0BF1050B013341
:10724000062B019300F0F1809AF80030022BEFD169
:107250009BF90320511C00F0EB80D2B2944602EB64
:107260004204A94B9DF8041003EB84040F2A5ED856
:10727000A74802E00330B84259D00378002BF9D177
:1072800045788D42F6D18578D8F840616068A56070
:10729000B042257000F04481D8F86461B04200F03B
:1072A0005E81D8F88861B04200F06281D8F8AC61A4
:1072B000B04200F06281D8F8D061B04200F06C8139
:1072C000D8F8F461B04200F08081D8F81862B0427A
:1072D00000F07681D8F83C62B04200F08081D8F8A6
:1072E0006062B04200F07681D8F88432984200F0B3
:1072F0008C81D8F8A832984200F08181D8F8CC323D
:10730000984200F0A581D8F8F032984200F09A81B6
:10731000D8F81433984200F0A781D8F8383398424F
:1073200000F0A881D8F85C33984200F097810132D0
:107330000C34D2B2624599D9002303939BF90420FF
:10734000531C79D0D2B2964602EB42046E4B9DF8A4
:10735000041003EB84040F2A5DD86D4802E003306B
:10736000B84258D00378012BF9D145788D42F6D137
:107370008578D8F840616068A560B04225705FD01C
:10738000D8F86461B04200F0EF80D8F88861B0426C
:1073900000F0F880D8F8AC61B04200F0F880D8F87E
:1073A000D061B04200F0FD80D8F8F461B04200F046
:1073B0000281D8F81862B04200F0F880D8F83C6238
:1073C000B04200F01781D8F86062B04200F00C8142
:1073D000D8F88462B04200F02481D8F8A8329842EC
:1073E00000F01981D8F8CC32984200F02581D8F805
:1073F000F032984200F01A81D8F81433984200F025
:107400004B81D8F83833984200F04081D8F85C338B
:10741000984200F0358101320C34D2B296459AD2AE
:1074200000220023CAE9042302E705B0BDE8F08F7B
:107430004FF00F0C002212E74FF00F0E002283E7EF
:1074400000231E46029306EBC600013608EB8000BF
:1074500090F958C1BCF1000FDDD1624680F844318B
:10746000AC462C4B1546029AC0F848C1134480F82C
:107470005991CAF81430132380F858313046FAF77E
:1074800091FB039B002BCBD0DAF814402046F8F791
:10749000B7FDDAF81000F8F7B3FDDAF81830C16874
:1074A000DAF80420596240215D60996002F1200100
:1074B0009D631960C3E90355C3E90555C3E9075541
:1074C000C3E90A55C3E90C55A4B1DAF81C303032CF
:1074D000E1681D625962C3E900254FF48032C3E9B7
:1074E0000255C3E90455C3E90655C3E90B55C3E981
:1074F0000D559A620023304607491A46FAF776FB83
:1075000001238AF80C3093E67C000024D6210B0876
:1075100058210B083C010024390A0000883000245F
:107520001846029300EBC00E013008EB8E0E9EF958
:107530005861002E7FF4FBAE029A8EF84431594B0D
:10754000CEF8485113448EF85991CAF810301423DC
:107550008EF85831FAF726FB01230393EEE6242038
:10756000012302901846DDE724201E4602906AE7B8
:107570004820022302901846D4E76C20032302908F
:107580001846CFE7022348201E4602905BE70323FC
:107590006C201E46029056E7902004230290184665
:1075A000C0E7042390201E4602904CE70623D82013
:1075B0001E46029047E70523B4201E46029042E78C
:1075C000D820062302901846ACE7B4200523029089
:1075D0001846A7E74FF4907002900820A2E7FC201D
:1075E0000723029018469DE74FF4907308260293F4
:1075F000002328E70723FC201E46029023E74FF4D0
:10760000B470022302900A208CE74FF4A273092081
:107610000293012386E74FF4B47002230A260290F6
:1076200011E74FF4A270092602900CE74FF4D873CB
:107630000C260293042306E74FF4C6730B2602932D
:10764000032300E74FF4D8730C200293042369E767
:107650004FF4C6730B200293032363E74FF40773C1
:107660000F20029307235DE74FF4EA730D20029386
:10767000052357E74FF4FC730E200293062351E7CE
:107680004FF407730F2602930723DCE64FF4FC73D5
:107690000E2602930623D6E64FF4EA730D260293D4
:1076A0000523D0E63C0100242DE9F04F4C484FF073
:1076B000010A4C494FF002094B4B4FF004080827D0
:1076C0001026202540244FF0800EDFF820C130F82E
:1076D000022F12F0010F03D01960083323F804AC15
:1076E00012F0020F03D01960083323F8049C12F043
:1076F000040F03D01960083323F8048C12F0080F2C
:1077000003D01960083323F8047C12F0100F03D063
:107710001960083323F8046C12F0200F03D01960AD
:10772000083323F8045C12F0400F03D019600833CB
:1077300023F8044C12F0800F03D01960083323F8AB
:1077400004EC12F4807F05D04FF4807B196008337D
:1077500023F804BC12F4007F05D04FF4007B1960BD
:10776000083323F804BC12F4806F05D04FF4806B0B
:107770001960083323F804BC12F4006F05D04FF4ED
:10778000006B1960083323F804BC12F4805F05D045
:107790004FF4805B1960083323F804BC12F4005FD7
:1077A00005D04FF4005B1960083323F804BC12F4D1
:1077B000804F05D04FF4804B1960083323F804BC88
:1077C000D20B05D04FF400421960083323F8042C83
:1077D00001F5806161457FF47AAFBDE8F08F00BFAD
:1077E0004A230B08000002580425002400240258F4
:1077F0002DE9F0470546086888B00C464FEA902C02
:10780000BDF84080ACF5801C9DF844A0BCF1520F3F
:1078100058D819462E4B13F80C600D2E52D806EB93
:10782000C6032C4F06EB430307EB8307FEF73EFA34
:1078300094F80590A379BAF1000F01D083F0010309
:107840005A004FF48071DB00384602F00202CDF896
:10785000088003F0080303924A46049360230193CF
:107860004FF40073CDE90613002301A905935EF0E0
:10787000DBFEA379384649469F0726D457F01AFE07
:107880004C22154B02FB063393F8112D012A10D11F
:107890000221D3F8D42C83F8111D104B91680B40B2
:1078A000062B06D0B3F5803F03D0136843F00103E5
:1078B00013602168637901F1340269600021D018F6
:1078C0002860D15008B0BDE8F08757F0F3FED7E745
:1078D00090200B08142B0024401E002407000100F8
:1078E00010B4284C94F8303763B3226D904234D0F2
:1078F000012B27D0D4F82C21824236D0022B21D064
:10790000D4F80822904232D0032B1BD0D4F8E422C2
:1079100090422ED0042B15D0D4F8C02390422AD008
:10792000052B0FD0D4F89C24904226D0062B09D0EA
:10793000D4F87825904222D0072B03D0D4F85426CF
:10794000824210D0DC22591C02FB034284F830171B
:10795000106518465DF8044B70470023DBB25DF8F4
:10796000044B184670470723F8E70123F6E7022384
:10797000F4E70323F2E70423F0E70523EEE7062309
:10798000ECE700BFFC1000200548D0F8103323B10D
:10799000DB6A13B100F5447018470248704700BF16
:1079A000401E0024C82F0B0838B51D4CD4F8603297
:1079B0001B8843B91B4D002384F86F3285F80833C8
:1079C000C5F8043338BDD4F86422002AF2DDD4F8B7
:1079D0006812012A488806D00123124DA4F86C02CF
:1079E00084F86E32E7E78A880132121A9A42F3D19C
:1079F0000C4D0022D5F8103305F54470C5F83C2332
:107A00001B699847D5F810339B68002BD3D005F538
:107A1000447098470028CED15DF05CFFCBE700BFF3
:107A2000382F0024401E00240748D0F80C331BB127
:107A3000064B93F86E320BB100207047D0F810332C
:107A400000F544705B681847401E0024382F00245E
:107A5000184A10B4184C92F8083344602344174C69
:107A6000036092F8080394F86F32834218D892F8B2
:107A70000803834207D300235DF8044B1A461846D7
:107A8000C1E90032704792F808031A1E5DF8044BF2
:107A9000C0F180030CBF01200220C1E90032704711
:107AA00092F80843002201201B1B5DF8044BC1E93A
:107AB00000327047401E0024E0290124382F0024A2
:107AC000104B114A93F8081392F86F0293F80823A9
:107AD000904293F808230FD8904204D3D3F804338C
:107AE00000201844704793F80823D3F80433C2F1F8
:107AF0008002104418447047801AD3F804331844A5
:107B0000704700BF401E0024382F002438B5194D9F
:107B1000194CD5F86022937B012B08D0D4F804339C
:107B200003F2FF736FF30A03C4F8043338BDD4F8CB
:107B300010335B6A63B104F544709847D4F810338E
:107B40009B681BB104F54470984778B1D5F8602262
:107B5000D4F804335288013B514213440B4003F2E2
:107B6000FF736FF30A03C4F8043338BD5DF0B2FE4F
:107B7000ECE700BF382F0024401E0024F0B51C4C59
:107B800085B01C4B94F808231B4D0393134495F8C0
:107B90006F1294F808230293914294F8083316D890
:107BA00099420CD294F808630F46C6F18006D9B901
:107BB000334601223F2BCDE900670DD860B994F818
:107BC0000803401AB0FA80F0400905B0F0BDCB1AA6
:107BD000002701221E46EDE76946002302A866F051
:107BE00049FC95F86F12EAE773180222E2E700BF3A
:107BF000401E0024E0290124382F00242DE9F047FD
:107C0000174684B000293ED0441E294DDFF8AC90C1
:107C10004FF0000A04EB0108264E0DE096F80833F9
:107C20000846994296F808331DD2C3F180031844E0
:107C30003F281BD8A04526D095F86F0214F8013FC5
:107C4000411C4844C9B280F820300B0685F86F12F9
:107C5000E4D5002096F8083385F86FA201469942D2
:107C600096F80833E1D3C01A3F28E3D996F80833D1
:107C70009942DFD0104B5B78002BDBD00020FFF760
:107C80007DFFA045D8D1694602A8FFF7E1FEDDE9F6
:107C9000003213443F2B00D910B904B0BDE8F0877F
:107CA00002463B4602A866F0E5FB04B0BDE8F0875B
:107CB000382F0024401E002400000024C029012485
:107CC00030B585B0694602A8FFF7C2FE58B9094C25
:107CD00004F54475D4F8103328465B6898470028AB
:107CE000F8D005B030BD0246012302A866F0C2FB01
:107CF000EDE700BF401E002438B50023124C134DA1
:107D0000C5F80C335CF0E2FAC4F86802FFF73CFEF9
:107D1000D4F86832C4F86002A3B19A885B88D21A9A
:107D2000436802FB0333C5F80C33F8F70FFE94F8F1
:107D30006F22044695F808339A4201D0FFF7C0FF3E
:107D4000C5F8044338BD00BF382F0024401E00246E
:107D50002DE9F041104E154682180446D6F80C3332
:107D60000F469A420D4A88BF1D1A92F86F2296F864
:107D700008339A4201D0FFF7A3FF002021462B468B
:107D80003A46C6F83C03D6F81003846A0448A44671
:107D9000BDE8F041604700BF401E0024382F00249A
:107DA000502100248C461346014662461846CFE710
:107DB0002DE9F043484F93B0484DFFF7F5FD97F894
:107DC000083395F86F229A4201D0FFF779FF00241B
:107DD000D7F80C63C7F80443002E6DD0DFF800819C
:107DE0000AE097F8083395F86F229A4201D0FFF71E
:107DF00067FF2034A6421BD922464146684603F05D
:107E000013FE684666F090FC012201466846FFF7C3
:107E1000F5FEA3B2002BE4D1D7F84833002BE0D015
:107E20009A881B6859690A4218BF12049A61D8E7F8
:107E3000FFF76CFE97F8083395F86F229A4201D04D
:107E4000FFF73EFF0023DFF8989098461C46C7F8DE
:107E500004332246494609A803F0E6FD2122002109
:107E6000684669F06BFE202269462046FFF770FFE6
:107E70002022054609A9684669F095FEA3B2203480
:107E800050B9202D08D15BB1A642E2D8B8FA88F0EB
:107E9000400913B0BDE8F08308F10108002BF3D1CD
:107EA000D7F84833002BEFD01A689B8851690B42F2
:107EB00018BF1B049361E7E7FFF728FE97F8083324
:107EC00095F86F229A4201D0FFF7FAFE00230120B5
:107ED000C7F80433DDE700BF401E0024382F00241C
:107EE00020F30B0808B559F0B9F91B20FBF7FEFB8E
:107EF00008B12923C3801C20FBF7F8FB08B1292314
:107F0000C38062F0B9FE11485FF048FB104B93F854
:107F10007522012A09D0022A05D193F87C22012A70
:107F200012D0022A0ED0012008BD0A4AD3F85C05FF
:107F3000C3F8582562F0AEFC0023074A184682F8C1
:107F4000233008BD054AF1E7054AEFE74404002461
:107F5000382F00242404002400ED00E0E403002472
:107F6000040400240A4B93F87C241AB9094A92F8B5
:107F7000600570470849CA6D032AF7D10020054AF9
:107F80004FF0010C83F87C0482F860C5C865EEE709
:107F900000000024382F00240040005808B50322B8
:107FA0000E4BDA6572B60E4B53E9021251EA020328
:107FB00006D100231A4609490A664B66FCF742FDC2
:107FC000084B4EF6602C5B6E0CFB00F05B1842F128
:107FD0000002C31842EBE072EDE700BF004000581A
:107FE000A8340024401E00240021032008B5FAF71D
:107FF000F7FB72B6FCF7D2FC154C08B5D4F8703517
:1080000094F87605ABB91420FEF7AEFE00BFD4F8A5
:1080100070355BB1196894F876259B8809690B4027
:1080200012B91BB1FFF7E0FF002BFBD0F8F7C2FC41
:10803000ECE719689A880B69134020B1002BE2D154
:108040000B691340FAE7002BDDD00B691340FAE708
:10805000382F00242DE9F04F00218BB041F62C720F
:10806000B74869F06BFD0420FAF7B4FB0146052020
:10807000FAF7B0FB51EA000340F05581B14B03938E
:10808000039BE422B049AE48D3F8B04469F060FCE9
:10809000AB4B1E465C621C67C3F8B440C3F8B840E3
:1080A000C3F8BC40C3E90744C3E91A445FF086F94A
:1080B000FFF722FE002108460BF0A8F8F8F746FC6F
:1080C000B0F1000840F399810024A04DDFF8A0C270
:1080D00006F1E4092746A24605F5AF6B9C4E0194D4
:1080E000CDF808C004E00AF5006AD04540F3AD8041
:1080F000029A536EC2F84433F8F75CFC20225946CA
:108100005046FFF725FE12229249584669F04BFD72
:108110000028E8D1BA4525D001998F4B01EB4102E7
:1081200003EB82034A1C8D4918460193AAEB07030F
:108130000592049303F078FC019B4946059A41F8A7
:108140004C3B049BC9F80C700192C9E90433D9F87F
:108150001C30C9E908330123C9F80830804BC9F83D
:1081600028308946039B57461222D3F8B034C9F809
:108170001C30A918335D013291F8781599420BD063
:108180000024202AF5D120375946B845384653DB1C
:10819000FFF7DEFD0022ECE70134152CF1D1D019F8
:1081A00070492022FFF7D4FD00230A2209A96D4857
:1081B000CDF824B003F0E6FC0746099800230A2214
:1081C000013009A9099003F0DDFC0790002309980C
:1081D0000A2209A90130099003F0D4FC069000237B
:1081E00009980A2209A90130099003F0CBFC0590F7
:1081F00009A9099800230A220130099003F0C2FC62
:108200000023049009980A221946013003F0BAFCB1
:1082100097B10599DDE9063243EA4212049B5B01FE
:1082200043EAC123A7F2BC7143EA600342EA412258
:1082300043EA0243C9F81C30019B642B43D05746E4
:108240000AF5006AD0453FF753AF019B642B1ED05F
:10825000BA451CD00C22404C4049AAEB070502FB52
:108260000344013320461A46019303F0DDFBD9F89D
:108270001C20C9F80040C9F81450C9E9082201229D
:10828000C9F80820364AC9E90375C9F82820019BB6
:10829000002B03F1030117DC4FEA4803B3F1805FC1
:1082A000C0F2AC80264B986830B91A461B791BB1D6
:1082B0001368002B40F0D880002108460BB0BDE8C1
:1082C000F04F0AF0A3BF67214C261D4BDFF8A490A6
:1082D0004FF0010A06FB01F432460021224F1D191E
:1082E000284669F02BFC32460021284669F026FC1E
:1082F0001B4E134A04F11003019942F804901834FC
:10830000C5F808A004312F62AE6242F8038013441E
:108310000432C3F80480039BD3F8B03413511444DF
:1083200063606B62B8E74FF47A72002366F05AFE1E
:108330000E4B40F2B27240F26D14B0FBF3F31DE04D
:10834000783A002400000024DC2F0B08382F00248A
:1083500064F30B0840F30B08D034002454F30B08EB
:10836000A57D0408B03400240068214C8051010030
:10837000401E00247CF30B085B1A013212F0030547
:1083800014BF21464FF4B7718B42F5DA8549002DB1
:1083900064D003910399D1F880148B42C0F29C8081
:1083A000814D01245B1A55F8041F01349942F9DD0F
:1083B0000133A2F2BC72039D43EA44133C2443EA16
:1083C00042237A4AB0FBF2F102FB11024FF46160E2
:1083D000B2FBF0F100FB11221C20C5F88404B2FBB3
:1083E000F4F004FB1022521042EA401242EAC12289
:1083F00042EA0343C5F8B03442E603214C266C4BF5
:10840000DFF8B891012706FB01F4324600214FF056
:10841000020A1D19284669F091FB324600212846C0
:1084200069F08CFB624B039A04F1100143F804904D
:10843000C8F10063D2F8B00404F11802BB405C4CF0
:108440005C4E85F805A0AF602E62635021444B60FE
:10845000231D98501A445060686223E70C4603912C
:108460001D21C4F8841495E7514C002200230146D5
:108470000546A064E063C4E910232246D46C02F1EF
:108480004C035CB39C684E1E9D64B442C2E9235504
:10849000DD630DD04E1CB44210D113F8481C0029E6
:1084A0003FF40AAF1A6421461A4643F8083CE5E750
:1084B00000293FF401AF53F80C2C2146A1427FF470
:1084C000FBAE00293FF4F8AE146CE66B0136E663B0
:1084D0001C6493641A46D1E7012469E7344A0226F2
:1084E000254613E0D36B16635B01C2E9045520D027
:1084F00003F6FF7301EB133319465363CB1A9163F1
:1085000052F84C7F4E1C1C440130C7B11379711EC8
:10851000002BE7D1136916637BB103F6FF7301EB00
:1085200013335769536337B107F6FF7701EB173100
:10853000E4E73346E0E73146E0E73346F1E7DFF8CA
:1085400080C001393F25CCF894038A0F1A488B006C
:10855000CCF888433E24CCF86C034020CCF884133C
:10856000CCF87803CCE9DC45D1B140F2FF101B1800
:1085700042F100025B0A43EAC25303F140020C4895
:108580001344CCF87C2303EBC101CCF880334A02BE
:10859000CCF86813CB0DCCE9E300CCE9D8238BE60B
:1085A0000123EAE700000024800400248051010038
:1085B000783A00240068214C98F30B088CF30B08E0
:1085C000401E00240000000038B5074B14460D463D
:1085D0001B681B6A984702464FF40073002012681C
:1085E0002A60238038BD00BFA859002408B5054B78
:1085F0001B6823B15B699847013840B208BD4FF052
:10860000FF3008BDA8590024002070472DE9F04133
:10861000CBB116460F4603EB02080E4C256800232B
:1086200039463046AD681A46A8470028F6D0236878
:10863000002BFCD05B6998470028F8D0013607F57D
:108640000077B045EAD1044A0020044B12681A6052
:10865000BDE8F081A8590024A41E00248421002430
:108660002DE9F041F3B116460F4603EB0208114C19
:1086700003E0216811B14B699847216800230D6917
:10868000304639461A46A8470028F2D12368002B05
:10869000FCD05B6998470028F8D0013607F50077D1
:1086A000B045EAD1044A0020044B12681A60BDE8C4
:1086B000F08100BFA8590024A41E002484210024B6
:1086C000002070470020704708B5FAF7FDFB98B10D
:1086D0000B4B986D58B1026893F855308088126939
:1086E00010402BB9003818BF0120013840B208BD36
:1086F000B0FA80F04009F8E74FF0FF3008BD00BF46
:10870000A859002400207047034B93F82800003834
:1087100018BF0120704700BFA8590024816D03468F
:108720000A6A52681278FF2A09D090F8F020013ABC
:1087300052B2002A80F8F02006DD0120704708229E
:10874000002083F8F02070470B6A002202205B684B
:108750001A707047836D1B6A5B681B78FF2B0AD108
:1087600090F9F030002B03F1FF3280F8F020D4BFF5
:108770000220012070470020704700BF836D1B6AF4
:108780005B681B78FE2B0CD0FF2B08D190F9F030E2
:108790005A1E002B80F8F02001DD012070470220D6
:1087A00070470020704700BF034B93F82800032850
:1087B00094BF002001207047A8590024004870474A
:1087C000D4590024034B93F82800003818BF012027
:1087D000704700BFA859002470B5124C05460E46DC
:1087E00094F82830042B0ED0082B19D1236A834229
:1087F0000ED0002394F8F62063620AB1C4F8F83072
:10880000FAF762FB30B10823C4E9085684F828302F
:10881000022070BD044B09221B6884F82820A36144
:10882000012070BDA8590024A41E0024034B93F816
:108830002800032894BF002001207047A859002475
:1088400000487047D4590024164B002030B493F8E8
:108850002A4014B1DD698D4205D0013010330B2858
:10886000F5D130BC7047104BBAB1D3F8141101EBFD
:1088700040218A4201D1022C08D093F8E42212B997
:10888000012283F8E422012283F8FD2003EB001388
:10889000012283F8262130BC704703EB001383F8D4
:1088A0002621DEE7A45A0024A859002430B400236E
:1088B0001A4C04F1FC0084F8D03103E0013310308D
:1088C0000B2B19D0C5698D42F8D190F82AC0BCF1A4
:1088D000030FF3D192B1D4F8141101EB43218A4272
:1088E00005D094F8E422A2B1012284F8FD2004EB23
:1088F0000314012384F8263130BC7047D4F8CC210E
:1089000004EB03130421013283F82611C4F8CC21AF
:10891000F2E7012284F8E422E6E700BFA859002428
:10892000C0B1836823B10F4B072283F8FE20704744
:108930000C4A042192F8FC0082F81031032882F8D6
:10894000FE10C2E9423314BF4FF480738023C2E9A2
:1089500040337047034B012283F8E42283F8FD2063
:10896000704700BFA8590024704700BF2DE9F047A9
:10897000002BDDF820A0884607460CBF4FF02009E9
:108980004FF030095646002A144616F8011B23DD25
:1089900011B3334601E0002C05DD13F8012B254609
:1089A000013C002AF7D1023D3CB149463846C04758
:1089B000013DFAD29AF8001059B13846C047334603
:1089C00016F8011B0029F8D1A4EB0A041819BDE818
:1089D000F0872046BDE8F087002C04F1FF35E4DC89
:1089E00000240029E9D1F4E703685A1C02601970D9
:1089F000704700BF10B56FF000440246044404E025
:108A0000B3EB0E0015D1A24214D012F8013BA3F132
:108A10004100192811F8010BA0F1410C98BF203337
:108A200000F1200EBCF1190FEAD91B1A04D100285D
:108A3000E9D110BD002010BD184610BD884230B5E8
:108A40004FF001043AD301FB04F4B0FBF4FC8C4575
:108A5000F9D2BCB102BB06E0A14203F8015B11D818
:108A60001446B0FBF2FCBCF1090F0CF157050CF1F8
:108A7000300E04FB1C00B4FBF1F2EDDCA14203F864
:108A800001EBEDD900221A7030BDA14203F8015B61
:108A9000F8D81446B0FBF2FCBCF1090F0CF1370515
:108AA0000CF1300E04FB1C00B4FBF1F2EDDCA14232
:108AB00003F801EBEDD900221A7030BD8446002A7C
:108AC000EAD1D0E7002870B503DA2D23404201F83F
:108AD000013B092886464FF0010307DD03EB8303C2
:108AE0005B00B0FBF3F2092AF8D89BB10F4CA4FB52
:108AF000030CBEFBF3F2092A4FEADC0C02F1570625
:108B000002F1300503FB12EE07DD092B01F8016BC2
:108B10006346ECD800230B7070BD092B01F8015B94
:108B20006346E4D800230B7070BD00BFCDCCCCCC25
:108B30000378202B03D110F8013F202BFBD0092B09
:108B4000F9D02D2B00F0A9802B2B75D0B7EE000AA1
:108B5000A3F13002D1B2092977D8F2EE046ADFED31
:108B60005F7A07EE102A10F8013FB8EEC77AA3F13A
:108B70003002D1B2A7EEA67A0929F0EE477AF0D9F1
:108B80002E2B66D003F0DF03452B40F0838010B41A
:108B900042782D2A00F096802B2A00F08380A2F1E3
:108BA00030030130092B00F284800024002303EB02
:108BB000830302EB430310F8012FA2F13001303B95
:108BC0000929F4D9B3F59A7F1A46B7EE007A28BF7F
:108BD0004FF49A72072B09D91346DFED416A083B1F
:108BE00027EE267A072BFAD802F00702DAB1F2EE66
:108BF000046A012A27EE267A15D0022A27EE267A61
:108C000011D0032A27EE267A0DD0042A27EE267AE1
:108C100009D0052A27EE267A05D027EE267A062ADD
:108C200018BF27EE267A002C45D0C7EE877A5DF86C
:108C3000044B20EE270A70474378B7EE000A013054
:108C4000A3F13002D1B2092987D92E2BDFED237A87
:108C500098D143780130A3F13002D1B2092991D8DB
:108C6000B2EE047AF0EE475A06EE902A10F8013F71
:108C7000B8EEE66AA3F13002D1B2C6EE076A09295E
:108C800027EE257A77EEA67AEED903F0DF03452B9F
:108C90003FF47DAF20EE270A70474378BFEE000A0D
:108CA000013055E782780230A2F13003092B7FF6BC
:108CB0007CAFB7EE007A67EE877A5DF8044B20EE62
:108CC000270A704782780230A2F13003092B01D8BD
:108CD00001246BE7B7EE007AA7E700BF00000000B1
:108CE00020BCBE4C022870B51CD80F4BC943C6002F
:108CF00003EBC00001F0010190F8585390F859239C
:108D000081EA0504A2420DD0D0F854233AB14D1B9C
:108D1000106892886942694109018A40826133443E
:108D200083F8594370BD00BFA85900240E4B1B683F
:108D300010B54BB10D489A881968037803F0010308
:108D40001B0102FA03F38B61094C5BF0DBF923682A
:108D5000002BFCD05B6998470028F8D0054A00201A
:108D6000054B12681A6010BD88210024942100244C
:108D7000A8590024A41E00248421002408B5FAF771
:108D80003DFE48B10F4A137F0133DBB2072B137747
:108D900003D9002382F8283008BD936D43B11868C9
:108DA00092F855109B880069034041B1002BF0D127
:108DB000054B01211B6882F82810936108BD002B28
:108DC000E7D0F5E7A8590024A41E002410B50379C4
:108DD000184C002B14BF0122002284F8542025D007
:108DE000154BA26D5B78003B18BF012384F8F63069
:108DF00082B111689388096994F855200B403AB103
:108E000043B1237F0022013384F82820237710BD4B
:108E1000002BF6D0FAF7F2FD0028F2D1074B012221
:108E200020771B6884F82820A36110BD84F82830BF
:108E300010BD00BFA859002484290024A41E0024CA
:108E400008B51D4B5878FAF751FC38B14FF01F0C9C
:108E500000222021A0F806C0F9F75EFA174B1B6824
:108E60004BB117489A881968037803F001031B0176
:108E700002FA03F38B61134B0021032093F90320C3
:108E8000F8F7FAFD50B1104A936D5BB1196892F88A
:108E900055209B8809690B4012B91BB9012008BDF8
:108EA000002BFBD1FAF7AAFD0028F7D1074A084B9F
:108EB00012681A6008BD00BFB03100248821002468
:108EC0009421002484290024A8590024A41E0024ED
:108ED000842100240E4838B5836D0D4614463BB1FD
:108EE000196890F855209B8809690B4052B15BB90D
:108EF000FAF716F8074A4FF400730020926C2A60C4
:108F0000238038BD002BF3D14FF0FF3038BD00BFB8
:108F1000A8590024502A0024F8B5854C94F85460D0
:108F2000002E00F0BC8094F828506B1E082B1DD832
:108F3000DFE803F09A8E4E1C35059E1C27007D4B02
:108F40005B6A002B40F08D807B4B072225691B68F4
:108F500084F82820A361002D00F08380636901203C
:108F6000D4E90121A84794F828506B1EDBB2022BEC
:108F700071D9042D18BF082D0CBF012600263046DC
:108F8000F8BDF9F7A1FF002840F0BC806A4AA36948
:108F90001268FA339342ECD2FFF7F0FEC3E7654B59
:108FA0001F6A002F40F0A680F9F78EFF0028BAD084
:108FB00004232569277784F82830002DDFD06369E2
:108FC00038466268A168A84794F828506B1ECDE720
:108FD000F9F7A6FF00283ED1584B606293F82C1099
:108FE000DA8D84F832102286196B1A6B090E120C76
:108FF00084F8331084F834201A6B196B120A84F841
:10900000361093F8341084F8352084F8371093F82C
:10901000351093F83520090902F00F0284F83C104E
:1090200084F83D209A6BD88FA263DA8FD98FC2F370
:109030000B1301F00F02042143EA102384F84020AF
:1090400003F00F0384F8281003F5FA63E3876AE757
:10905000F9F73AFF38BB384BA2691B689B1AC82B3B
:109060003DD800263046F8BD022384F828305AE760
:10907000F9F72AFF002889D0626A0023012A2377A2
:1090800044D9216A013A0131C4E9081294F8F62062
:109090000AB1C4F8F830082384F828306FE7304666
:1090A00084F82860F8BDF9F73BFF0028D3D1244BA2
:1090B0001B78002BA3F10203B3FA83F308BF012549
:1090C0005B096577A377F9F72BFF00287FF464AF7E
:1090D0001A4B03229B6C84F82820E36223E7FFF7F6
:1090E0004DFE94F82860042E18BF082E0CBF0126F0
:1090F000002644E7104AA369126864339342FFF4E0
:1091000012AF36E7042384F8283038E7FAD194F810
:10911000F62063620AB1C4F8F830F9F7D5FE0028EA
:10912000F0D1054B09221B6884F82820A36198E739
:10913000A8590024202A0024A41E0024502A002418
:10914000A82A00242DE9F843284C80468946174672
:1091500094F828C01E46BCF1040F12D0BCF1080FD1
:1091600002D00020BDE8F883002394F8F620636263
:109170000AB1C4F8F830F9F7A7FE28B3042384F83D
:10918000283019F01F0F26D10125194B41464846BA
:109190001D624FF400732A46C4F87093C4F87853E4
:1091A000C4F874335DF09EF8A8B9124B0522284626
:1091B000C4F804901B68C4F8088084F82820A361D0
:1091C000C4E90476BDE8F8830A4B09221B6884F8D9
:1091D0002820A361C5E7FFF7D1FD2569002DC0D088
:1091E00000226369A1681046A847BAE7A85900247D
:1091F000202A0024A41E00242DE9F041274D084612
:1092000011461A46AC6D3CB12668A38834692340E8
:1092100095F855407CB383BBC3062ED10123204C67
:10922000C5F8700323624FF40073C5F87823C5F8BE
:1092300074335DF057F800BB236A002BFCD1DFF8D4
:10924000708041F20D16174FD8F84450D8F80040FE
:109250002D04A56041F28832E3680D2120463B4091
:109260003343E36056F0C6FC58B1D8F834300343BA
:10927000C8F83430EDE7002BCED14FF0FF30BDE819
:10928000F081636903F4F053B3F5006FE1D1064A4E
:10929000064B12681A60BDE8F08100BFA85900248F
:1092A000202A0024C0E0FEFFA41E00248421002404
:1092B000A42900242DE9F041224D10460A46AC6D48
:1092C0004CB12668A18895F8555034692140002D8D
:1092D00031D0002931D100215DF080F868BB1A4AF5
:1092E000536A002BFCD1DFF8708041F20D16174F46
:1092F000D8F84450D8F800402D04A56041F28832D7
:10930000E3680D2120463B403343E36056F072FC96
:1093100028B1D8F834300343C8F83430EDE7636936
:1093200003F4F053B3F5006FE7D1094A094B126813
:109330001A60BDE8F0810029CDD14FF0FF30BDE8C3
:10934000F08100BFA8590024202A0024C0E0FEFFBD
:10935000A41E002484210024A42900242DE9F04720
:10936000384C1F4605460E4694F828309046042B8C
:1093700011D0082B3DD1236A83420CD0002394F8EE
:10938000F62063620AB1C4F8F830F9F79DFD50B3D6
:10939000042384F82830D4F8F890C9F34F230F2B16
:1093A000C4E9016528D8D4F824A0BAF1000F23D06D
:1093B00094F8F63003B324484FF400723146484421
:1093C00068F0C6FA09F50073C3F34F22C4F8F83009
:1093D0005B0A102A02D0BAF1010F28D19BB21A4EB3
:1093E0005A1EAD1A09E0194B09221B6884F828207F
:1093F000A3610120BDE8F08701230621284601254D
:10940000324684F828100021C4F810806761257363
:109410005CF0E4FF0028EDD0FFF7B0FC266926B130
:1094200063690022A1682846B0470320E2E7226A68
:109430000AF1FF33042102200132636284F828100C
:109440002262D7E7A8590024EC7E0024A41E002441
:1094500010B5144CA36D6BB1196894F855209B8816
:1094600009690B4022B12BB1002384F8283010BDCC
:10947000002BF9D094F82830032B0CD8237F01332C
:10948000DBB2072B2377EFD8074A0123126884F851
:109490002830A26110BD0548FDF71AFEA4F860004F
:1094A000ECE700BFA8590024A41E0024801A06007F
:1094B00030B5002299B00446952513468DF80C105E
:1094C0008DF80D5044F040050493012065F3070228
:1094D0008DF81C300A938DF830308DF84430159398
:1094E00017931C4D069010908DF8580002A8CDE9F6
:1094F0000D33CDE913330B0E099005F15C0063F3D6
:109500000F220B0C090A63F317420DF107030593B1
:1095100061F31F62104B0292089306230F4A0DEB72
:1095200003010B93082312920F9104A985F8F430DC
:109530004FF024F9EA6D136A002BFCD19DF8073037
:10954000FF2B00D01CB99DF8060019B030BD4FF0BC
:10955000FF30FAE7A85900241D870408558704083E
:1095600030B597B000231E4C0DF107020890084655
:1095700008218DF8143007938DF828300B938DF85F
:109580003C301593174D84F8F4106944099004F1A8
:109590005C0006959FED107BCDE90232CDE91033DA
:1095A0000122CDE91233022304928DF850200E934C
:1095B0008DED0C7B4FF0E2F8E36D186A0028FCD1CA
:1095C0009DF80730FE2B03D0FF2B0CBF012002209B
:1095D00017B030BDAFF300800000000000000000B5
:1095E000A85900247D87040830B52A4C9DB0FD257C
:1095F00000230122002000218DF8065004F15C05B3
:1096000063628DF83C3010938DF8503015931893A9
:109610001A930E928DF86420CDE912320DF10603F3
:10962000CDE90C01CDE916010CA9284611934FF0A4
:10963000A5F8E26D136A002BFCD10DF107010122A0
:1096400028468DF8143009930B9304928DF8282046
:1096500084F8F420CDE902310F49069102A9CDE941
:1096600007334FF08BF8E36D186A0028FCD19DF8A2
:109670000730FF2B07D0094A0923126884F82830E5
:10968000A2611DB030BD0423022084F828301DB033
:1096900030BD00BFA859002455870408A41E00242B
:1096A00010B58078FAF722F890B10A494FF0410CD2
:1096B00004460022D1F87C3380F806C00133C1F89B
:1096C0007C332021C371F8F727FE2368A2889A61B2
:1096D00010BD00BFA8590024F0B503798BB02C4D04
:1096E000002B14BF0122002285F8542003D185F8F5
:1096F00028300BB0F0BD05F15C07044690F900106E
:1097000038464FF05DFCA678002E34D1214B22481C
:10971000C5F8F0306E66FDF7DBFCA5F860004FF48D
:109720007A70FDF721FB6B6E13B11A689B88936109
:109730001A4CEC460FCCACE80F000FCCACE80F0095
:1097400094E803008CE80300694638464FF016F8A9
:10975000EB6D1A6A002AFCD11EB10D213046F8F7D4
:10976000DBFD0F4B012100221B6885F828102A77AA
:10977000AB610BB0F0BD3046F9F7B8FF06460028E4
:10978000C4D01E2300222C21C380F8F7C5FDBDE7FD
:10979000A8590024AC590024801A0600D83A0B08B6
:1097A000A41E00242DE9F041954C92B094F8546029
:1097B000002E00F0BD8194F828305A1E082A00F2CD
:1097C0004C81DFE812F02D006200A8004A0123015D
:1097D00059011A004A0109005AF064FC002840F0BF
:1097E0008582884AA3691268FA33934280F03281F5
:1097F000FFF72EFE94F82830DFE75AF053FC0028DC
:10980000EFD0636A0022012B227740F28782226A1E
:10981000013B08210132636284F828102262EAE0E9
:1098200000210846FFF744FEE26DC5B2136A002B23
:10983000FCD10A20FDF708FA636E13B11A689B8801
:109840009361012D40F00681002740F2AB11082002
:109850006777FFF72DFEC0B2052800F0B881012818
:1098600000F09781E26D136A002BFCD10A20FDF70E
:10987000EBF9636E13B11A689B889361637F002BC9
:1098800000F03182022384F82830657F00213720E0
:10989000A5F10205FFF70CFE2920B5FA85F56D0943
:1098A000AD072946FFF704FEE26DC5B2136A002B2F
:1098B000FCD10A20FDF7C8F9636E13B11A689B88C2
:1098C0009361002D40F0C680637F022B00F0C481BD
:1098D00000210920A577FFF7EBFD002800F07A8131
:1098E0000025E26D136A002BFCD10A20FDF7ACF9CC
:1098F000636E13B11A689B889361002D00F0AA80F3
:1099000000210A20FFF7D4FDC0B2002840F0958165
:10991000032384F82830102103A8FFF721FE002834
:1099200040F09880BDF80D309DF80C205BBA9DF892
:10993000111062F307009DF80F2023869DF819305F
:1099400062F30F209DF810201B019DF8145062F364
:1099500017409DF81A20DBB261F31F60DDF8151087
:1099600043EA121302F00F0209BAC4F8320003F5F9
:10997000FA6384F84020A1632909E387BDF8123017
:10998000E26DE38605F00F0384F83C1084F83D3067
:10999000136A002BFCD10A20FDF756F9636E13B150
:1099A0001A689B889361A37FA3B94FF400711020BC
:1099B000FFF77EFDE26DC5B2136A002BFCD10A20D1
:1099C000FDF742F9636E13B11A689B889361002D0D
:1099D0007FF40EAF0C48FDF77BFB04220021A4F8B6
:1099E0006000134684F828206162042B18BF082BFE
:1099F0000CBF01260026304612B0BDE8F08100BF42
:109A0000A8590024A41E002440787D014FF4007161
:109A10006068FFF7A5FD012800F09080022800F0A3
:109A20009380B8B9E26D136A002BFCD10A20FDF7D0
:109A30000BF9636E13B11A689B88936104230020AD
:109A4000256984F828302077002DD4D06369D4E9C3
:109A50000121A84794F828305A1ED2B2022AC4D84D
:109A6000AA4BA2691B689B1AC82B00F287800026AC
:109A7000304612B0BDE8F081E26D117B136A002917
:109A800042D05269002A3FD094F8E420002A3BD00B
:109A9000B3FA83F35B09002BDCD0002302A9012277
:109AA0009B48ADF808308DF81830079308938DF86F
:109AB0002C3011938DF84020CDE90313022105913C
:109AC0000DF10701CDE9091203A9CDE90C33CDE968
:109AD0000E334EF053FEE36D1D6A002DFCD19DF850
:109AE000073003F01F03052B00F0EA80FFF7B0FCFE
:109AF0002769002F3FF45FAE63692A46A168012001
:109B0000B84794F8283058E663680022217B8048E3
:109B100003EB01214FF480734EF0EAFD227B01320A
:109B2000D2B2A2F102032273B3FA83F35B09B2E764
:109B3000304684F8286012B0BDE8F081734AA3690A
:109B400012686433934285D2E26D136A002BFCD114
:109B50000A20FDF779F8636E13B11A689B88936148
:109B6000FFF776FC2569002D3FF425AE00226369DE
:109B7000A1681046A84794F828301EE6FFF768FC55
:109B800094F82860082E18BF042E0CBF012600266A
:109B900031E702AB03A95E480493042303978DF8D1
:109BA0001870079705930A978DF82C500C97CDE9FC
:109BB00008774EF0E3FDE26D136A002BFCD19DF8AF
:109BC0000B30AB2B7FF44FAE022363774BE6E26D95
:109BD000657748E610214F48FFF7C2FC00287FF464
:109BE0007FAE94F8533013F001033FF479AE94F84C
:109BF0004420921100F0A580012A7FF471AE94F800
:109C00004B201621444F02259200D2B2C5F1080321
:109C10008B4228BF0B46C3F108059840C91A42FA87
:109C200005F24FF0000540EA020017F8012FEDD1D0
:109C3000013083023546E36253E6E26D136A002B7E
:109C4000FCD10A20FDF700F8636E002B3FF4D0AD85
:109C50001A689B889361CBE529463A20FFF728FCD8
:109C600002ABC7B203A90493042329480593012337
:109C700003958DF82C308DF818500C95CDE90755CB
:109C8000CDE909554EF07AFDE36D1A6A002AFCD140
:109C90007FB91A6A002AFCD10A20FCF7D5FF636E4F
:109CA00013B11A689B889361029D2DBAC5F3807524
:109CB0000EE61A6A002AC4D01A6A002AF9D1C0E74F
:109CC000124B072225691B6884F82820A361002D08
:109CD0003FF4CDAE63690120D4E90121A84794F88F
:109CE00028305A1EB9E684F82830C0E6E26D136ABF
:109CF000002BFCD10A20FCF7A7FF636E13B11A6892
:109D00009B889361042384F8283074E6A41E002401
:109D1000045A0024EC590024F359002459D0042398
:109D2000E26D84F82830136A002BFCD10A20FCF77E
:109D30008BFF636E002B3FF48DAE1A689B88936196
:109D400088E694F849001146DFF89CC0032500F02E
:109D50000F0294F84D00062780019340C0B2C7F16E
:109D60000802AA4228BF2A46C2F108079140AD1A4C
:109D700040FA07F04FF0000741EA00011CF8010F1C
:109D8000EDD194F84A000231DFF860E00C27800141
:109D90004FF0060CC0B2CCF108024FF0000CBA42F2
:109DA00028BF3A46C2F108089540BF1A40FA08F0A9
:109DB00045EA00051EF8010FEDD10135D81705FA67
:109DC00001F2A2FB033102FB00125B0A43EAC25319
:109DD00030E7FFF709FC02287FF43CAEE36D1A6A16
:109DE000002AFCD1A2E700BFF5590024F259002453
:109DF0002DE9F0410546884617461E462B4C94F83F
:109E0000280004280AD0082806D1236AAB423BD098
:109E1000FFF7EAFB0228F2D0012031E0A37F8BBBE1
:109E200069021820FFF744FBC0B278BB94F82830D1
:109E3000082B29D0FE23E26D84F88033117B1C4B64
:109E4000C3F8288051B1526942B194F8E420002A45
:109E500014BF4FF400724FF4807201E04FF480722F
:109E6000144813491A634EF089FC0122062300208E
:109E7000C4F80480A56027616661227384F82830E5
:109E8000BDE8F0812946CCE7FC23D4E7E26D136AF4
:109E9000002BFCD10A20FCF7D7FE636E13B11A68C1
:109EA0009B889361FFF7D4FA0320E9E7A8590024BF
:109EB00018050024045A002470B5204E05460C46AF
:109EC00096F82830042B08D0082B1ED1336A834221
:109ED00019D0FFF789FB022817D100213720FFF79F
:109EE000E7FA21461720FFF7E3FAC0B2A8B9B37F1B
:109EF0006BB969021920FFF7DBFA70B90823C6E9CC
:109F0000085486F82830022070BD012070BD294613
:109F10001920FFF7CDFA0028F0D0F26D136A002B5C
:109F2000FCD10A20FCF790FE736E13B11A689B886F
:109F30009361FFF78DFA032070BD00BFA85900247C
:109F40002DE9F0411F4C07468846164694F828C074
:109F50001D46BCF1040F09D0BCF1080F02D000204F
:109F6000BDE8F081FFF740FB0228F8D1A37F9BB149
:109F700039461120FFF79CFAC0B2A0B9124B052256
:109F80000120C4F804801B6884F82820A76026619B
:109F9000C4E90553BDE8F08179021120FFF788FA82
:109FA000C0B20028EAD0E26D136A002BFCD10A206F
:109FB000FCF74AFE636E002BD1D01A6800209B8804
:109FC0009361CDE7A8590024A41E0024092917D0C5
:109FD000B1FA81F35B0999B1013903604A0001F0DC
:109FE000030102F00802C1EB01119300C1EB011162
:109FF000A3EB92038900C3EB031381809B00438092
:10A00000704700BFB5EEC00ADFED357A0023F1EEF0
:10A0100010FA30B5C8BF30EE270A87B0D8BF30EE8F
:10A02000670ADFED307A054603A9029320EE270A7E
:10A03000CDE90033FDEEC07A17EE904A84EAE47071
:10A04000A0EBE47058F0DEF9002C03A8B4BF2D2378
:10A0500020238DF8003064F067FB01282AD0022805
:10A0600034D003281ED003A9684667F06FFD684608
:10A0700064F05AFB044669462846033CE4B2224693
:10A0800067F066FC002328462B5564F04DFB2E221A
:10A09000431C0DEB04012A54E81867F0DDFD284647
:10A0A00007B030BD302303A968468DF8013067F052
:10A0B0004DFDDCE743F23002302303A96846ADF8DA
:10A0C00001208DF8033067F041FDD0E743F2300303
:10A0D00003A96846ADF8013067F038FDC7E700BF57
:10A0E0006F12033A00007A4408F0C6BC38B5054642
:10A0F00058B14C1E14F8011F284619B9BDE8384064
:10A1000008F0CEBC08F0B8FCF4E738BD08B5CB07C2
:10A1100001D4FAF797FC08BD014B1B681B6A18476E
:10A12000A8590024094A936D73B11968988892F868
:10A1300055300A6910401BB1B0FA80F040097047F1
:10A14000003818BF0120704701207047A85900242B
:10A15000024B186808B1836918477047A859002452
:10A160000378022B12D00E4943680269D1F84803E4
:10A17000023A184010B4400AD1F84043D1F83C13D9
:10A1800004FB02005DF8044B08447047044B42682E
:10A19000D3E9CC0100EB410000EB5220704700BF37
:10A1A000A85900242DE9F04F83B002F00207874E32
:10A1B000019308B9002F4ED1D6F83843C4BB4FF0F5
:10A1C000FF3E834C4FF0000CF146F246F046E36947
:10A1D00094F82A50984249D015B3012D06EB0C1B78
:10A1E0000ED19BF82751EB070AD415F07E0F07D14B
:10A1F000ED0940F0A380656AA84584BFA846E14602
:10A200000CF1010C1034BCF10B0FE0D1BEF1000FCA
:10A2100080F2BB80BAF1000FC0F29D80D44628E0E6
:10A22000E6460CF1010C1034BCF10B0FCFD1EDE779
:10A23000D6E9CF3505FB0434A042C0D396F8E4320A
:10A2400013B9012386F8E432012386F8FD3000209B
:10A2500003B0BDE8F08F96F8E432002B77D00123ED
:10A26000022086F8FD3003B0BDE8F08F002D40F0ED
:10A270008E80D6F8C8410CF1020506EB0C180134AB
:10A2800006EB051EC6F8C8410EF1FC0ECEF80440E0
:10A29000C8E946040024CEF8084006EB051494F8FB
:10A2A0000641042CD7D80FF2080E5EF824F000BF48
:10A2B000C5A20408FBA204084FA20408FBA20408DC
:10A2C000FDA2040812F00104D6F814E16DD106EBEA
:10A2D0000510019B4FEAE20E90F80781032B6EF305
:10A2E000C71880F807815ED94FF6FF70834228BFF8
:10A2F000034606EB0510A0F8043197BB500707D5BD
:10A3000006EB051090F8073143F0010380F80731A0
:10A31000D3060AD506EB051595F80731C3F34502B8
:10A32000013262F3460385F80731D6F81431012073
:10A3300003EB4C230B6003B0BDE8F08FE2460CF159
:10A34000010C1034BCF10B0F7FF441AF5EE7012329
:10A3500086F8E43283E7B9F1000FFFF678AFCC4618
:10A3600087E7D6F8CC01D6F8C83101300133C6F8FA
:10A37000CC0106EB0C10C6F8C831C0F81C3106EB56
:10A380000513042083F80601B8E7F44671E7D6F810
:10A39000C8410CF10205013406EB051EC6F8C841A0
:10A3A000CEF8004179E72346A3E733680EEB4C2152
:10A3B000084A9C680023A04700283FF448AF06EBFA
:10A3C0000515022385F8063141E700BFA85900248E
:10A3D000A45A00244988040870B5114D82B00E4675
:10A3E00095F8FC30022B16D1020AC4B2D5F830031E
:10A3F000002301A910440322FFF7D4FE012808D14D
:10A4000095F8FC30019A022B0CBF22F8146042F838
:10A41000246002B070BDC0F3D41200F07F04E5E701
:10A42000A85900242DE9F04F444E0D4683B017463D
:10A4300096F8FC102B6803293ED0022961D14FEA1F
:10A4400013294FF4807A5FFA83F8421E012A23D839
:10A450004FF0010B9F421AD901288CBF0024012420
:10A46000D6F8A8221AB1D6F8C41299424CD0D6F820
:10A4700030030023092201A94844FFF793FE012875
:10A4800023D0022814D020B12B689F42E8D80320A3
:10A490002F6003B0BDE8F08FB8F1000F13D096F82D
:10A4A000E43213B9012386F8E432012386F8FD3043
:10A4B000022003B0BDE8F08F4FF0800AC3F3D41937
:10A4C00003F07F08C1E7D346C4E796F8FC100229E1
:10A4D00013D00329ECD1019B53F8282022F07042BD
:10A4E000B2FA82F22B685209A2421FD0D8445B44D0
:10A4F000D0452B601DD20229EDD1019B33F81820E5
:10A50000EEE74FF4807AD9E7D6F84013013A02EB30
:10A5100041224902B2FBF1F21344B3FBFBF20BFB05
:10A5200012320AB15B449B1A2B60AEE79F42B0D84F
:10A53000ADE709F101094FF00008A6E7A85900248A
:10A540002DE9F04FDFF884918B4685B0174699F8D6
:10A55000FCC00968BCF1020FD9F8305340F082808A
:10A56000CEB24FF4807305EB1125A6EB01089044A1
:10A570009844B94208F1FF38B8FBF3F84AD200F02A
:10A580000103A8446FF0404A0193BCF1030F07EBAD
:10A590000604A8EB0503284614BF4FF480728022FE
:10A5A000641A03A9944228BF1446944228BF002E7F
:10A5B00014BF012200220A32FFF7F4FD01282AD13C
:10A5C00099F8FCC0DBF800E0BCF1020F0EF10103CA
:10A5D00024D0B44255D9039806EB0A02011F00EBC0
:10A5E000820201EB840142F8043F8A4203F1010335
:10A5F000F9D1DBF80030A11B19448F42CBF80010D1
:10A6000002D1019B002B48D18F4205F101054FF08B
:10A610000006BAD8012005B0BDE8F08FB44246D993
:10A6200003986FF00042811E324401EB440100EBBD
:10A63000420222F8023F914203F10103F9D1A11B2A
:10A6400071448F42CBF80010DED1019B002BDBD090
:10A6500086466FF000434FF6FF72012023442EF828
:10A660001320D8E701F07F06C1F3D413BCF1030F28
:10A67000A6EB01081D4414BF4FF48073802390445F
:10A6800076E7AEEB060E0EEB04018F42CBF800101E
:10A69000BAD1019B002BB7D003986FF040434FF025
:10A6A000FF32234440F82320DBF80010ACE7AEEB88
:10A6B000060E0EEB04018F42CBF80010A4D1019BD3
:10A6C000002BA1D0DDF80CE0C3E700BFA85900249F
:10A6D00030B50446C06983B010B9012003B030BD65
:10A6E0000D460023032201A9FFF75CFD0128F5D1E7
:10A6F000B4F92020002A19DB019B012D4FEA4211F9
:10A7000003EB421203D0022D1BD1E5205854A3685D
:10A71000D3612378032B04D10023137753779377E6
:10A72000D377636A190C53839182D6E7064A92F86D
:10A73000E41209B982F8E4020123022082F8FD3014
:10A74000CCE7E368E4E700BFA85900242DE9F04115
:10A75000022382B004460E4694F83C20042A7CD89A
:10A76000DFE802F02E03704F3F00414D4FF6F777C0
:10A77000DFF8008118E0BC4562D859F067FC012879
:10A780004FF00001034638D1206BFFF725FE01286A
:10A79000034632D10199D5F844034A1E216382420F
:10A7A00028BF0246C5F8442395F8FC0001A9226B96
:10A7B00003281FFA82FC1046DDD14245DDD93FE077
:10A7C0007100204601F0FE01FFF782FF01280346D9
:10A7D00043D1626B002A14BF0222012284F83C207C
:10A7E000BAE794F82830042B02D1002384F82830EB
:10A7F000A36B0BB1204698470123184602B0BDE871
:10A80000F0811B4D0021E26AD5F8C43205F52870AD
:10A81000C5F8C4229B1AD5F8402302FB03F3D5F8F0
:10A82000A82202EB4322C5F8A822D5F8AC2202EBFD
:10A830004322C5F8AC22FFF74BFF012803460CD199
:10A840000422CBE7626B04F130010020FFF778FEB1
:10A850000128034601D10322C0E7022BCDD194F891
:10A860002820042AC9D1002284F82820C5E700BF87
:10A87000A8590024F7FFFF0F38B5044694F8343088
:10A88000052B60D8DFE803F031251D130D0394F884
:10A890002830082B3FD02D4B0122022083F8E522DF
:10A8A00038BD94F82830082B30D0012038BD002165
:10A8B0002046FFF70DFF012845D1042084F834001D
:10A8C000DCE7D4E90B01FFF787FD01283BD103202A
:10A8D000F4E74FF0FF31206BFFF77EFD012832D106
:10A8E000E36A002BF3D00220E8E7184D04F13001B1
:10A8F0000120D5F838230232FFF794FD012813D048
:10A900000238C0B201281ED80520D7E70023012055
:10A9100084F82830CAE700230122022084F8283076
:10A920000A4B83F8E522BBE7E368D5F84013226BB6
:10A9300003EB4123C5F84423C4E90332E36A002B47
:10A94000BCD16262BAE7002038BD00BFA85900241C
:10A95000F8B50446022094F83830032B07D8DFE816
:10A9600003F021180B0200212046FFF7B1FE431E21
:10A97000DBB2012B40D9F8BD0120626B04F130013C
:10A98000FFF7DEFD01284FF00303F0D184F83830E3
:10A99000E1E700211D48FFF79BFE01284FF002036D
:10A9A000F4D0E4E71A4BE66893F8FC20D3F84013A0
:10A9B000032AD3F8C45214BF4FF480728022256159
:10A9C00002FB01F1AF1A2A4406EB4126E660D3F8F8
:10A9D000A862C3F8C422A6EB4126C3F8A862D3F844
:10A9E000AC62A6EB4121C3F8AC12E36A2563626353
:10A9F00053B965620123C9E794F82830062BBAD110
:10AA0000002384F82830F8BD2763F3E7485C00246E
:10AA1000A85900244368C3F308020A44B2F5007F32
:10AA20002DE9F041054682B00C4605D223446B6007
:10AA3000012002B0BDE8F08190F91A10481C0AD03C
:10AA4000434A02EB011292F8271121F0010182F82A
:10AA50002711FF22AA7695F91B20511C0FD03C48E4
:10AA6000FF2600EB021090F82721C2F345010139BF
:10AA700021EAE17161F3460280F82721EE762A7817
:10AA8000022AD3D0324FD7F84023B4EB422F4FEAFB
:10AA900042282CDCD7F848631E407242A24226DCD2
:10AAA000A2192869424513D32A7E12072BD5D7F85D
:10AAB000C422411C8A421CD300D100214344A4EB90
:10AAC0000808686108469B1B08EB060429616B6057
:10AAD0000028ADD097F8FC20032A33D080B24FF67F
:10AAE000F7729042A4D81A4614446C60A0E7002084
:10AAF0009FE797F8E4220ABB012387F8E43287F83E
:10AB0000FD306B68DAE701A959F0A0FA0128EED10F
:10AB10006B68A4EB08042869984429786861344478
:10AB2000A8EB0603019802291A466B602861CFD171
:10AB3000D7F85013B3EB412FD6D379E7012287F82A
:10AB4000FD20BBE7034A90423FF672AFCBE700BF60
:10AB5000A8590024F7FFFF0F2DE9F0474FF0010837
:10AB600082B0044694F83830032B00F2A480DFE86A
:10AB700003F055170C020020236C84F8280003B161
:10AB80009847022002B0BDE8F0870022236C84F8C9
:10AB900028200BB120469847012002B0BDE8F0877D
:10ABA00023786768022B03D0444BD3F848331F4007
:10ABB000C7F34F272046FFF7D3FA404E3F1A05460A
:10ABC000BFB207EB050C022201A9002328461FFA99
:10ABD0008CF9FFF7E7FA01284FF400724FF00001FB
:10ABE000D0D1019866F0AAFFE3694FF400712046C6
:10ABF0000BB16368EBB1D6F84033013B994547D2BE
:10AC00000135FFF707FF0028DBD196F8E43213B9CE
:10AC1000012386F8E43286F8FD80D2E72046FFF76C
:10AC20002BFE012802D0022845D1032084F83800E9
:10AC300098E7019B4FF020324FF0100E4FF02E0C92
:10AC400042F62E6AC3F80120C3F80520A3F80920B4
:10AC500083F800C0D4F824C0A3F820A083F80BE048
:10AC6000C3F82220C3F8262083F82A20E26BA3F839
:10AC70001AC02CFA0EFC5A8722FA0EF2A3F814C05E
:10AC800083F82BE09A86D6F84033013B9945B7D339
:10AC9000C3EBC35320465902FFF7BCFE28B996F810
:10ACA000E43223B1012386F8FD300220BEE7012300
:10ACB00086F8E432F6E7002064E700BFA8590024D4
:10ACC000B1F904300F2B2DE9F0410D4682B0044656
:10ACD000164634D02046FFF743FA94F91B80B8F1AA
:10ACE000FF3F3DD05C4F07EB0813D3F81831984273
:10ACF00012D097F8E432002B70D0012387F8FD3092
:10AD00002378022B60D02269002A75D1002301200C
:10AD1000336002B0BDE8F081D7F8141101EB48218F
:10AD2000002967D0AB88204601331BB201EB4311E9
:10AD3000AB803160FFF714FA28600120E9E74FF497
:10AD40000071FFF767FE002844D04FF6FF732046DE
:10AD5000AB80FFF705FA94F91B80B8F1FF3FC1D132
:10AD60002378022B3ED02269002ACFD03A4F97F8A1
:10AD7000FC30032B67D093B24FF6F7718B4294BF30
:10AD800000230123002BBFD130B997F8E432002B08
:10AD90004CD0012387F8FD300023112201A9FFF7D1
:10ADA00001FA012826D10199D7F81431CB1A48BFEE
:10ADB00003F2FF13B3F5B05F4FEA63222CD24FFAD0
:10ADC00082F884F81B80ABE7D7F850236368B3EBB5
:10ADD000422F9BD2002002B0BDE8F081012387F80A
:10ADE000E4328AE71C4F6368D7F85023B3EB422F55
:10ADF000CAD38BE7237884E797F8FC30032B19D06C
:10AE000093B24FF6F772934294BF00230123002BB5
:10AE10007FF47CAF0020DEE797F8E43213B901231A
:10AE200087F8E432012387F8FD30CAE7012387F869
:10AE3000E432AEE7094B9A4294BF00230123002B72
:10AE40007FF464AFE6E7054B9A4294BF00230123E9
:10AE5000002B7FF459AF97E7A8590024F7FFFF0FA5
:10AE600010B50378044690F818C0023B012B02D9B4
:10AE70001CF0060F5DD11CF0200F3CD194F91A2074
:10AE8000511C0AD0314BFF2103EB021393F8272109
:10AE900022F0010283F82721A17694F91B305A1C75
:10AEA0000FD02A4901EB031191F82731C3F3450272
:10AEB000013A22EAE27262F34603FF2281F8273167
:10AEC000E2761CF0080F0DD0204B93F8C822072A19
:10AED00005D093F8E422A2B3012283F8FD200022DA
:10AEE00083F8C8220023E26A237084F82830FAB17C
:10AEF000BDE810401047164B0022E069D9691033B5
:10AF0000884206D001320B2AB8D0D9691033884262
:10AF1000F8D10E4901EB021191F82731C3F3450234
:10AF2000013A22EAE27262F3460381F82731A5E78B
:10AF300010BD0121FFF7CCFB0128F9D194F818C00E
:10AF400099E7012283F8E422C6E700BFA85900244C
:10AF5000A45A002438B51A4C94F810332BB970B1A8
:10AF600090F828201AB1184638BD002038BD014697
:10AF7000442204F53A7066F0EBFC012038BD04F57C
:10AF80003A7501464422284666F0D8FD94F8FC3014
:10AF900003224FF6FF71022B2846A4F8021318BFB4
:10AFA0001346D4F84C1384F80023102284F8E832B6
:10AFB000C4F80C1384F801235CF004FBDDE700BF48
:10AFC000A85900242F4A4FF0FF3CF8B5A2F1FC002D
:10AFD0000023644603E0013310320B2B14D092F8A7
:10AFE0002A100429F7D100EB031191F82711CE079D
:10AFF000F1D4651C116A01D08C45ECD91C46013393
:10B000008C4610320B2BEAD1002C01DA0120F8BD5E
:10B010001D4DA71C260105EB0713B3F80411D1B988
:10B02000AB19D5F81411194AD3F8180101EB4421D2
:10B030002B681C690023A047A8B1022809D1D5F8C4
:10B04000CC3105EB07170122013B87F80621C5F833
:10B05000CC310020F8BD05EB0413D3F818012B68A0
:10B06000DB689847DCE7D5F8CC3105EB07170321FF
:10B070000122013B87F8061185F8D021C5F8CC31B3
:10B08000E7E700BFA45A0024A8590024AD880408AB
:10B0900010B58C18A14215D001F1FF3E013C41F2E0
:10B0A000210C1EF8012F082380EA022002B2400082
:10B0B000002A8CEA420180B2B8BF88B2013BF5D1C8
:10B0C0007445EED110BDF8B5164D6B78BE2B26D168
:10B0D000AC1C154F022229464FF6FF70FFF7D8FF30
:10B0E00022884AB1A618BE4219D2052A17D921468C
:10B0F0003446FFF7CDFFF3E721460222FFF7C8FFF2
:10B100000222A1180634FFF7C3FF084B641BA3F803
:10B11000824341F60F53C31A58425841F8BD0020EC
:10B12000FCE700BF0000020800000408A859002442
:10B130000823484041B240000029C0B2B8BF504087
:10B14000013BF7D1704700BF30B5056804468D421A
:10B1500018D901F1FF3E681E00231EF801CF082117
:10B1600083EA0C034FFA83FC5B00BCF1000FDBB2F7
:10B17000B8BF53400139F5D17045EED16A1C226049
:10B180002B7030BD00236A1C22602B7030BD00BFC5
:10B19000DFED186ADFED187ADFED184AE0EE267A67
:10B1A0009FED177A9FED175ADFED175A9FED176A3B
:10B1B000DFED176A9FED170AC7FEE47AC7FE877AAC
:10B1C000FDEEE77A17EE903AC3F3160203F0FF4361
:10B1D00042F07E5207EE903A07EE102AE7EE055A4B
:10B1E000A5EE876AE6EE076AA6EE870A20EE270A32
:10B1F000704700BF3BAA384B00007E4E0000FF4E58
:10B2000000000000ED185E3C81900FBBAF9D2A3E10
:10B21000B2D19F3EE886023F10EE103AB5EEC00A6A
:10B22000DFED163AC3F31602DB159FED155AF1EE6A
:10B2300010FA00EE103A42F07E53DFED125A07EE9C
:10B24000903A9FED116ADFED116AB8EEC00AA7EEE1
:10B25000A35ADFED0F4A9FED0F4A20EE240A9FED1F
:10B260000E7A37FE047AE5EE275AA5EEA76AE6EED7
:10B27000276AA6EEA70A37EE000A7047DACDFE3C31
:10B28000B9D593BE5CB8903FAA841DC022E061404E
:10B290001872313F000080FF07F1B3C29FED067ABC
:10B2A000F7EE007A60EE870A60EE800A30EEA70AB9
:10B2B00080EE800A704700BFDB0FC94010B52DED4E
:10B2C000028B08EE101ADFED807ADFED800A04466B
:10B2D000B8EE488A28EE008A28EE278AB0EE480A9F
:10B2E00064F0C2FE9FED7A7AF0EE407AB4EEC70ABF
:10B2F000F1EE10FA40F3BD809FED746ADFED756AE0
:10B30000B0EE677A77EEC67AB4EEE67AF1EE10FA2E
:10B31000F6DC9FED717AF4EEC77AF1EE10FA40F3A5
:10B32000C5809FED6B7A77EE677A27EEA76ADFED2F
:10B330006B5ADFED6B6A9FED6B7AE6EE256A9FED47
:10B34000660A67EE865ADFED610A38EE000AA6EE5D
:10B35000267AE5EE877AB0EE678A64F085FEDFED47
:10B360005C7AB4EEE70AF1EE10FA5BDDDFED576AC6
:10B370009FED587AF0EE407A30EE660AF4EEC77A26
:10B38000F1EE10FAF6DCDFED547AB4EEE70AF1EEF6
:10B3900010FA62DDDFED4E7A37EEC00AF7EE007A82
:10B3A0009FED517A20EE004ADFED4C6ADFED4C4A0A
:10B3B0000023B0EE673A9FED4B5AE4EE264AC4ED07
:10B3C000097A60EE043AA361A8EE073A6361F0EEF1
:10B3D000675A2362F8EE006AE361A4EE245AE8EEAD
:10B3E000475A87EE836AA3EE850AB6EE007ABDEC73
:10B3F000028B77EEC07A26EE077A66EE266A27EE93
:10B40000865A67EE277A25EE866A26EE807A84EDE4
:10B41000015AC4ED007A84ED046AC4ED027A84ED29
:10B42000037A10BDDFED317AB4EEE70AF1EE10FADF
:10B43000A9D5DFED266A9FED2E7AF0EE407A30EE48
:10B44000260AF4EEC77AF1EE10FAF6D4DFED227A8E
:10B45000B4EEE70AF1EE10FA9CDCDFED267AB4EEEA
:10B46000E70AF1EE10FA99D5DFED207A37EEC00A3F
:10B4700094E79FED1E7AB4EEC70AF1EE10FA7FF55D
:10B4800048AF9FED126ADFED1A6AB0EE677A77EE89
:10B49000867AB4EEE67AF1EE10FAF6D49FED0E7AE3
:10B4A000F4EEC77AF1EE10FA3FF73BAF9FED117A59
:10B4B000F4EEC77AF1EE10FA7FF537AF9FED0B7A15
:10B4C00077EE677A31E700BF27D4D236DB0FC94069
:10B4D000DB0F4940E4CB1641DB0FC93F92E741B98E
:10B4E0009730083C15A82ABEF304353FDB0F49C04E
:10B4F000E4CB16C1DB0FC9BFDFED2D0A08B564F040
:10B50000B3FDDFED2C7AB4EEE70AF1EE10FA28DD98
:10B51000DFED276A9FED287AF0EE407A30EE660A7A
:10B52000F4EEC77AF1EE10FAF6DCDFED247AB4EE31
:10B53000E70AF1EE10FA2FDDDFED1E7A37EEC00AD2
:10B5400020EE007A9FED1E6ADFED1E6ADFED1E7AA7
:10B55000E7EE066A20EE076AE6EE877AA6EE270A8D
:10B5600008BDDFED1A7AB4EEE70AF1EE10FADCD589
:10B57000DFED0F6A9FED167AF0EE407A30EE260A84
:10B58000F4EEC77AF1EE10FAF6D4DFED0C7AB4EEF1
:10B59000E70AF1EE10FACFDCDFED0E7AB4EEE70A3F
:10B5A000F1EE10FACCD5DFED097A37EEC00AC7E725
:10B5B000DB0FC940DB0F4940E4CB1641DB0FC93F2D
:10B5C00092E741B99730083C15A82ABEDB0F49C065
:10B5D000E4CB16C1DB0FC9BFDFED2F7ADFED2F0AF9
:10B5E00030EE270A08B564F03FFDDFED2D7AB4EEAA
:10B5F000E70AF1EE10FA28DDDFED286A9FED297ADF
:10B60000F0EE407A30EE660AF4EEC77AF1EE10FA08
:10B61000F6DCDFED217AB4EEE70AF1EE10FA2FDD69
:10B62000DFED1F7A37EEC00A60EE006A9FED1E6AFA
:10B630009FED1E7ADFED1E7AA6EE867A20EE266A50
:10B64000E6EE877AA6EE270A08BDDFED1A7AB4EE99
:10B65000E70AF1EE10FADCD5DFED106A9FED167AFD
:10B66000F0EE407A30EE260AF4EEC77AF1EE10FAE8
:10B67000F6D4DFED097AB4EEE70AF1EE10FACFDC8A
:10B68000DFED0E7AB4EEE70AF1EE10FACCD5DFED7D
:10B69000097A37EEC00AC7E7DB0FC93FDB0FC940A5
:10B6A000DB0F4940E4CB164192E741B99730083CA3
:10B6B00015A82ABEDB0F49C0E4CB16C1DB0FC9BFFA
:10B6C000B0EEC07AF0EEE06AF0EE407AC6FE875A3D
:10B6D000F5EE405AF1EE10FA3BD086FEC75A85EEE1
:10B6E000256A9FED1D2A9FED1D3A9FED1D4ADFED56
:10B6F0001D4ADFED1D2AF7EE005ADFED1C3A9FEDE3
:10B700001C5AA6EE423AE6EE223AA6EE034AE6EECE
:10B71000235AE6EE044AA6EE245A85EE250AF4EEF4
:10B72000C76AF1EE10FA03D59FED127A37EE400AA0
:10B73000F5EEC00AF1EE10FA03D59FED0F7A37EE61
:10B74000400AF5EEC07AF1EE10FA48BFB1EE400AB9
:10B7500070479FED070AE2E739094E3DE3B59E3E8B
:10B7600088FA163E45FE7F3F99FB243F69A2163EAC
:10B77000A7DFA834DB0FC93FDB0F49402DE9F04FAD
:10B78000884689B01E461178531C0393002900F0A7
:10B790001681002514460746A94609E038460135BA
:10B7A000C047039C621C21780392002900F08F801F
:10B7B0002529F3D16078A31C3028CDE9033923D0A3
:10B7C000A0F130034FF0000ADBB2092B26D96C2818
:10B7D0002AD078287FD8572878D9A0F15803202B71
:10B7E00079D8DFE803F0BD78787878787878787859
:10B7F0007882AF787878787878787878AA78787856
:10B80000789E788A7878BD00E31CA0784FF0010A12
:10B810000393A0F13003DBB2092BD8D804AA03A903
:10B8200058F02CFD6C28D4D1039B1A785C1C782A24
:10B830000394B7D8572A40F28E80A2F15803202BE8
:10B84000B0D801A151F823F07FB90408A5B70408C6
:10B85000A5B70408A5B70408A5B70408A5B7040848
:10B86000A5B70408A5B70408A5B70408A5B7040838
:10B87000A5B70408EDB804089BB90408A5B70408E7
:10B88000A5B70408A5B70408A5B70408A5B7040818
:10B89000A5B70408A5B70408A5B70408A5B7040808
:10B8A0003DB90408A5B70408A5B70408A5B704085E
:10B8B000A5B7040825B90408A5B70408ABB904085E
:10B8C000A5B70408A5B704087FB9040828B9284615
:10B8D00009B0BDE8F08F039C64E72528FBD1039CE9
:10B8E000252138460135C0475CE7039C56F8041B08
:10B8F00038460135C9B2C04754E70DF1140B002298
:10B900000A2156F8040B5B46039CFDF797F8534653
:10B91000049A41463846CDF800B0FDF727F80544B3
:10B9200040E7039C56F8040B0023049A414600901C
:10B930003846FDF71BF8054434E7039C56F8043BF2
:10B940001D602FE70DF1140B56F8040B039C5946AC
:10B95000FDF7B8F8DBE7002AB9D0252AC0D021E7E7
:10B96000A0F158020DF1140B102156F8040BB2FA95
:10B9700082F25B465209FDF761F8039CC7E7A2F12A
:10B9800058020DF1140B102156F8040BB2FA82F292
:10B990005B465209FDF752F8B9E70DF1140B56F862
:10B9A000040B5946FDF78EF8B1E70DF1140B002298
:10B9B0000A2156F8040B5B46FDF740F8A7E70D4651
:10B9C00085E7F8B5134C07460D461646D4F88403B0
:10B9D000C0B11149FEF78AFB3946D4F88403FEF75B
:10B9E00085FB0E49D4F88403FEF780FB0C493346EF
:10B9F0002A46D4F88403FFF7C1FE0A49D4F8840329
:10BA0000FEF774FB94F8883313B1012384F889336B
:10BA1000F8BD00BFA859002468C70B0830E90B081F
:10BA2000E9A0040875C70B080EB400B584B0084936
:10BA300005AB019001A853F8042B0393FFF79EFE7A
:10BA40000022019B1A7004B05DF804EB03B070474C
:10BA5000E989040803685A1C02601970090A03681E
:10BA60005A1C02601970704702681346511C01602D
:10BA700013F802CB0360D31C5178036093781B0446
:10BA800043EA0123111D43EA0C030160D07843EA25
:10BA900000607047A0F13003092B07D920F0200087
:10BAA000413819288CBF00200120704701207047C1
:10BAB000303809288CBF00200120704741381928F0
:10BAC0008CBF002001207047613819288CBF0020EE
:10BAD0000120704720280BD0092809D00A2807D058
:10BAE0000D2805D00B3801288CBF0020012070479D
:10BAF00001207047A0F14103192B98BF20307047F7
:10BB0000A0F16103192B98BF2038704702B3844617
:10BB100010B5841803E0981A15D1A44514D01CF868
:10BB2000013BA3F14100192811F8010BA0F1410ECE
:10BB300098BF203300F12002BEF1190FEBD91B1A78
:10BB400004D10028E9D110BD002010BD184610BD59
:10BB50001046704770B5044608460D4662F0E4FD95
:10BB6000064602E014F8013F43B13246294620461A
:10BB7000FFF7CCFF0028F5D1204670BD1C462046BB
:10BB800070BD00BF2DE9F043064686469EF800C012
:10BB900074460EF1010EBCF1200FF7D0BCF1090F75
:10BBA000F4D0BCF10A0FACF10B00EFD0ACF10D05F5
:10BBB000B5FA85F56D09002DE8D10128E6D9BCF16B
:10BBC0002B0F3DD0BCF12D0F39D0102A3ED04FF0B5
:10BBD000FF3E9046BEFBF2FE02FB0EF7FF43FFB2B4
:10BBE000002014F801CBBCF1390F4CF02009ACF166
:10BBF000300C0DD85FFA8CFC944510DA704526465F
:10BC000002D819D1674517D21D404FF0FF30E8E741
:10BC1000A9F1570CB9F1600F5FFA8CFCECD801B1B7
:10BC20000E6003F00103D5B9002803DA002B18BF1A
:10BC30006FF00040BDE8F08300FB08C0D1E70125AC
:10BC4000102A94F801C004F10104C0D1BCF1300FF6
:10BC500010D06FF0704E0F274FF01008C0E7B0F112
:10BC6000004F04D91BB14FF00040BDE8F0834042C3
:10BC7000BDE8F08360786FF0704E0F274FF010082A
:10BC8000A0F14106192E04F1010698BF2030782852
:10BC90000CBF02343446A3E701230A22002171E7D6
:10BCA00003880021194A30B503F0030E90F802C052
:10BCB000174CA3F5FA630EEB4E0E0CF1FF3C40F26D
:10BCC000B5550CEB8E0C04EB4C044FEA930C238D12
:10BCD000847905FB0C3390F803C022444FF47A7446
:10BCE0000CF1FF3C634490F804C003EB43030CEBFE
:10BCF000C30C43790089CCEB0C1C03EB8C03C3EB26
:10BD0000031302EB8302C2FB040130BD80436D3894
:10BD1000D83A0B08F8B516461F463F4D044639463B
:10BD200030464FF47A72002363F05CF93B4B0544D4
:10BD30003B4F3C4E83FB0510E9172844C1EB6011D3
:10BD400083FB0103C8170B44C0EB631087FB003C67
:10BD5000C317C3EBAC0386FB03764FEAE37ECEEB5F
:10BD6000E61EC1EB0116A5EB860CC0EB00154FEAF1
:10BD70008E0684F806C0A1EB8501617103EB4301D7
:10BD8000A0EBC10040F2B55101FB1E332071B3F5A9
:10BD9000896F35DA40F2DA218B4237DCB3F5B77FB1
:10BDA0002149B4BF4FF0000E4FF0010E0EEB4E00D4
:10BDB00075464FEA4E0701EBC001C88F1B4907EBE0
:10BDC0000E0C01EBCC0C0B210CF1160C01E03CF835
:10BDD000020D984211DD0139F9D17744124901EB86
:10BDE000C701088D012106F5FA6E0133A170754473
:10BDF0001B1A22812580E370F8BD0131C9B2F2E738
:10BE0000032540F296500627AE46D7E7022540F2BA
:10BE100029400427AE46D1E780BC92C7898888882C
:10BE2000ABAAAA2A73B06D16D83A0B08003B0B08D0
:10BE30000D4B10B5D3E9004354EA03020AD1014681
:10BE4000002340F2011218460B80C1F802208B71CA
:10BE50000B8110BD054A1268121943F10003FFF768
:10BE600059FF012010BD00BFA0340024A41E0024EF
:10BE70002DE9F047044688B094F83030042B11D8EF
:10BE8000DFE803F04A135B035400237E9A0640F177
:10BE9000E2800023112205A9E069FEF783F9012859
:10BEA00000F0D98008B0BDE8F087C64D01AE04F1BE
:10BEB0001C0705F53A79324639464846FEF700FF39
:10BEC000012800F0E1800228ECD195F902335F1CD3
:10BED0000AD005EB0313FF2193F8272185F80213FD
:10BEE00022F0010283F8272195F903335E1C0FD05D
:10BEF00005EB031393F82721C2F34501013921EA29
:10BF0000E17161F34602FF2183F8272185F80313CD
:10BF1000042384F83030AFE7AB485BF053FB4FF6B7
:10BF2000FF720123228484F83030A5E70020E36A01
:10BF3000207008B0BDE8F0471847A24D95F81033BF
:10BF4000002BAFD104F11C0705F53A7801AE32465B
:10BF500039464046FEF7B4FE012840F0E780DDF8A0
:10BF60000490B9F1000F00F0C08099F800300BB1D7
:10BF7000E52BECD1D5F81431B9EB030348BF03F23C
:10BF8000FF13B3F5B05F4FEA632280F00E81120118
:10BF90008E4B13449A7B042A0CD0D5F8C821013269
:10BFA000C5F8C8215A6004229A73D5F8CC31013300
:10BFB000C5F8CC3195F90233581C0AD005EB0313B0
:10BFC00093F8272122F0010283F82721FF2385F827
:10BFD000023395F90333591C0FD005EB0313FF21EE
:10BFE00093F8272185F80313C2F34501013921EAAB
:10BFF000E17161F3460283F827212022002148469F
:10C0000065F09CFDD4F83120D4F8353005A8C9F886
:10C010000020C9F8043094F83B30B4F8392089F88E
:10C020000A30A9F80820637E89F80B30FFF700FF7B
:10C03000BDF81430002B40F0FC8044F281720321E3
:10C04000A9F81020A9F80E30A9F81820A9F8163080
:10C0500084F8301010E720465BF0B4FA2369002B17
:10C060006BD0237E03F0F70213F00403227671D124
:10C07000122A00F086800022E36A204684F82820F5
:10C0800008B0BDE8F0471847DDF80480B8F1000FAC
:10C0900000F09E8098F80030002B00F0998098F80E
:10C0A0000BA01AF0080F7FF406AF0B2204F1310148
:10C0B000404665F078FD00287FF4FDAE637E8AEA95
:10C0C0000303DF0640F1EB8095F902335E1C3FF479
:10C0D0000BAF05EB0313FF2193F8272185F802131B
:10C0E00060F3000283F82721FEE695F8E832092282
:10C0F000022B3FF40DAF95F81033002B7FF408AFFF
:10C1000085F82033404685F81C3385F81023C5E9AF
:10C11000C933D5F8FC32C5F81433D5F84433C5F823
:10C120001833FEF719FD01283FF411AF02287FF400
:10C13000B9AE042384F830309EE6237E1B079AD5DF
:10C14000204B93F8C822002A7FF4ACAE072283F874
:10C15000C82290E70023A5682046E66A294684F8AD
:10C160002830FEF757FC002840F0938094F82830E0
:10C17000002B7FF497AE0223C4E90B6584F82830C6
:10C1800090E6E06A0421626AA063204684F83C30AD
:10C1900084F8281063636362C4E90B22C4E90233A4
:10C1A00008B0BDE8F0475BF00DBA95F8E43213B97A
:10C1B000012385F8E43201236FF00F0285F8FD308A
:10C1C000E6E600BFA8590024905C0024C05A002471
:10C1D00095F90233591C0AD005EB0313FF2193F89C
:10C1E000272185F8021322F0010283F8272195F90F
:10C1F00003335A1C0FD005EB031393F82721C2F326
:10C200004501013921EAE17161F34602FF2183F81A
:10C21000272185F80313237EDB067FF579AE3F489F
:10C220005BF0D0F94FF6FF720223228484F830309D
:10C2300022E605A8B5F98C53FFF732FD4FF47A7268
:10C24000002362F0CFFE3C2392B205FB03014FF4C2
:10C250007A700023C1FB002302A8FFF75BFD9DF865
:10C260000A309DF80B209DF80E1042EA4312BDF8EB
:10C270000830A3F2BC7342EA43229DF80D305B0103
:10C2800092B243EA51039DF80C1043EAC1239BB2DA
:10C29000D5E6002E3FF406AE2046334649E6B8F810
:10C2A0001420B8F81A3043EA0243D5F840236362F9
:10C2B0005202D8F81C30B3FBF2F102FB1131A3603B
:10C2C00009B113445B1AE36084F819A095F90233AD
:10C2D000591C0AD005EB0313FF2193F8272185F899
:10C2E000021322F0010283F8272195F903335A1C27
:10C2F0000FD005EB031393F82721C2F34501013951
:10C3000021EAE17161F34602FF2183F8272185F8D4
:10C310000313032384F83030AEE500BF905C0024A3
:10C320002DE9F04190F8283082B00446013B082BFB
:10C330000BD8DFE803F0393D1F24052A0A2F34000B
:10C340000121FEF703FA012802D002B0BDE8F08116
:10C3500000222378216C84F82820002BF5D00322BA
:10C36000E162D4E9010384F82820834238BF034600
:10C370002046A36002B0BDE8F041FEF771BD002188
:10C3800002B0BDE8F041FEF7E1B902B0BDE8F0410E
:10C39000FEF7DEBA02B0BDE8F041FEF76DBA02B0BA
:10C3A000BDE8F041FEF7D8BB02B0BDE8F0415FE563
:10C3B000DFF84C814268D8F84853036B1540D8F831
:10C3C000401390F800E0E8184E02B0EB412F41D343
:10C3D0004FF6F777BEF1020F14D021690846002905
:10C3E00063D16068A3680021E26A834284F8281060
:10C3F00038BF0346A360002AA7D0204602B0BDE89C
:10C40000F0411047D8F850136068B0EB412F34D298
:10C410002069217E09073AD5D8F8C41200F1010C31
:10C42000614530D298F8E41200294FD1012388F8F1
:10C43000E43288F8FD30626894F800E0236B9B1BBF
:10C4400032442B44521B00259E4262602363C4E9A0
:10C4500004C0BFD9BEF1020F0ED021690029C0D09F
:10C4600098F8FC00032843D089B24FF6F770814258
:10C47000B7D898186060B5E76068D8F85013B0EB8B
:10C48000412FF6D3AEE7DAD14FF0000CD7E701A980
:10C4900057F0DCFD01287FF458AF2069DDF804C0B7
:10C4A00094F800E06268236BC9E798F8FCC0BCF11F
:10C4B000030F11D01FFA81FCBC4594BF4FF0000C54
:10C4C0004FF0010CBCF1000FC8D1A2E7012188F8A0
:10C4D000FD1094F800E0B2E7DFF820C0614594BF9A
:10C4E0004FF0000C4FF0010CBCF1000FB6D190E7FB
:10C4F000024881423FF675AFBBE700BFF7FFFF0F71
:10C50000A85900242DE9F0410446154608469442F6
:10C51000B4FBF2F607D205FB1644134B1B5D00F883
:10C52000013BBDE8F0819642B6FBF2F70CD20E4B10
:10C5300005FB176705FB1644DA5D1B5D00F8012B50
:10C5400000F8013BBDE8F081BA42B7FBF2F807D929
:10C5500005FB1878044B13F8082000F8012BE7E7D7
:10C560004046FFF7CFFFF3E724F40B0830B56F4CDC
:10C5700083B0B4F8BC37B3F57A7F03D94FF47A733C
:10C58000A4F8BC37B4F8BE37B3F57A7F03D94FF4BB
:10C590007A73A4F8BE37B4F8C017B1F57A7F04D91E
:10C5A0004FF47A731946A4F8C037B4F8C207B0F54F
:10C5B0007A7F03D900231846A4F8C237B4F8C437E9
:10C5C000B3F57A7F4CD94FF47A73B4F8C6279A4200
:10C5D000A4F8C43749D900238842A4F8C63780F0AC
:10C5E0008F80B4F8D227B4F8D4379A4202D9002306
:10C5F000A4F8D2374E4B1B88EBB14E4DAA78062AD1
:10C6000052D9297900297ED19FED4B7A94F8DC2705
:10C6100007EE903AAB7906EE902AF8EEE77AB8EE9C
:10C62000E66AC6EE276A0BB137EE077AB4EEE67A11
:10C63000F1EE10FA46DC94F8E527032A25D83F4BA3
:10C6400003EB421394F8E427C4F8F437032A14D810
:10C65000EA213B4B02FB0133C4F8F83703B030BD8D
:10C66000B4F8C627B2F57A7F18D8884212D29A4217
:10C67000B7D30023A4F8C437B3E70022304B84F8C3
:10C68000E427C4F8F83703B030BD00222B4B84F800
:10C69000E527D7E70021A4F8C017E8E70022884281
:10C6A000A4F8C627E3D3F5E7264901EB820191ED13
:10C6B000227A29790029A9D0531F032BBBD9002A3C
:10C6C000B9D025E067EE877ABCEEE77A8DED017A86
:10C6D0009DF8043007EE103AB8EEC77AF4EEC77A48
:10C6E000F1EE10FA01DD0133DBB2EBB1102BA8BF84
:10C6F0001023DBB2934238BF134684F8DC379AE745
:10C70000A4F8C0376DE7053A032A94D99FED0A7A59
:10C71000B7EE000A80EE070A64F01CF82B8883420B
:10C7200028BF03462B8086E70123E2E7A8590024AF
:10C73000481C0020882F00246F120338385D002425
:10C74000B85D0024D83A0B082DE9F04F9D4E83B018
:10C7500096F8FC3700AFA3F11702022A00F2938289
:10C76000994B7B6096F814380024DFF878A23B6080
:10C77000964B03F1780998461FE098F90420142A93
:10C7800000F07C82584665F0B9FA1BF4003F21D0D6
:10C79000012800F07382082800F3708215B11BEAAB
:10C7A0000A0F06D1396858465FF0BCFE002800F039
:10C7B000658208F10C08C14512D0D8F800B01BF012
:10C7C0000105DAD05846013465F098FA1BF4003FB1
:10C7D000E4B2DDD10128DEDC08F10C08C145ECD162
:10C7E000013C022C00F24A820023022086F8BC3869
:10C7F0000FF034FC96F8C438D6F8C058022B00F07D
:10C80000EE82002800F04483714B4FF47A7E96F854
:10C8100021A94FF0000C03F56A794FF0640B33F84F
:10C82000082CB2F57A7FB3F8462088BF23F808ECCD
:10C83000B2F57A7F33F8062C88BFA3F846E0B2F54C
:10C840007A7F33F8042C88BF23F806ECB2F57A7FA0
:10C8500002D9002223F804CC33F8061C9142B3F825
:10C860005A10B3F85C2098BF23F806CC914293F895
:10C870006B2003F1650102F1FF3288BFA3F85AC0B3
:10C88000632A93F86C2002F1010288BF83F86BB031
:10C89000D2B2092A4FF0000288BF83F86CC013F8A7
:10C8A0003200013211F8014F844238BF81F800C0D4
:10C8B000032AF4D1BAF1010F03F1EA0318BF03F818
:10C8C00064CC9945ABD1DFF8209199F80230042B64
:10C8D00000F0B2822BB9B9F80030B3F5F07F00F266
:10C8E000F081FFF743FE3B4896F83419FDF76EFBE5
:10C8F000103096F85319FDF769FB103096F863195C
:10C90000FDF764FBB6F87229B6F870391343B6F830
:10C91000742913431BB213B10123A6F876392E4BA9
:10C920002B40002B00F0C182E80700F172826904FD
:10C9300000F1CC812A0740F13582284AD6F8143913
:10C9400015401340C6F8C058C6F814392C0440F1FD
:10C950000D82002386F81B3886F82B38E80440F156
:10C96000108296F88339012B02D9012386F8833986
:10C97000DFF86CA053460AF1780402E006339C42CB
:10C980000CD01A780A2AF9D19978DA78914202D330
:10C990005A79002AF2D00A2025F01AFD00234FF41C
:10C9A000806086F8BC380FF059FB002800F05D82EB
:10C9B0000B4DAB469BF8051019B39BF80000F0B186
:10C9C000534616E0A8590024D83A0B08E861002421
:10C9D000C25D0024EC62002409600002FE9FFFFD9E
:10C9E00030630024BC020200882F002406339C42DE
:10C9F00007D01A788A42F9D15A79002AF6D025F060
:10CA0000E7FC0BF1060B5C45D4D199F802A0BAF112
:10CA1000080F00F0CC8196F82139D6F81429A3F13B
:10CA20000103C2F3C031B3FA83F386F8031A5B093A
:10CA300086F8003A96F82239A3F10103B3FA83F39A
:10CA40005B0986F8063A96F8B937032B02D900231A
:10CA500086F8B937B749D6F8C0380A400B4096F87F
:10CA6000F217C6F81429C6F8C038002900F0D3819F
:10CA7000B6F81C3A002B40F0C281D6F8203AB3F544
:10CA8000000F02D30023C6F8203AD6F8283AAA4A63
:10CA90001A401AB140F20223C6F8283A96F8243A0E
:10CAA000013B042B02D9012386F8243AAAF1050A96
:10CAB000A24BBAF1030F93F8A08540F23081B8F190
:10CAC000000F1CD000233B60DFF898A206E0ABF11A
:10CAD000060BABEB090BD84540F2FA80D3461AF8A7
:10CAE000010F0028F3D00EF02DFF0028EFD0817940
:10CAF0008B07ECD53B680122002B40F0EE8099F8C3
:10CB0000063013B1002389F80630B6F8323A03F044
:10CB10000F02042A03D8C3F30313022B03D94FF4E3
:10CB20002063A6F8323AB6F8343A03F00F02042A2A
:10CB300003D8C3F30313022B03D940F60123A6F84D
:10CB4000343A96F8A51A96F8B12A96F8A43A914282
:10CB500005D9002286F8A52A53B1A6F8A82A96F886
:10CB6000B02A9A4204D2002386F8A43AA6F8A83A3A
:10CB700096F8A62A96F89A3B9A4202D9002386F89C
:10CB8000A63ADFF8E4C10CF1800B6346796813F82C
:10CB9000032D02EB42020A4492F85CA292F85D92E5
:10CBA00092F85EE213F8010F99795045DA78A8BF40
:10CBB00050464945A8BF494672451870A8BF7246FD
:10CBC00063459971DA70EDD103F1200CDC45DCD1BD
:10CBD000D6F83828002A00F026810020012102E042
:10CBE0000635AC420ED02B782B2BF9D16B78043361
:10CBF00001FA03F31342F3D0063522EA03020120BF
:10CC0000AC42F0D108B1C6F838284D4C6D4604F15D
:10CC10000808234601E098456DD013F8012F072A34
:10CC2000F9D9002304F8013F0133082BFAD1B6F8F3
:10CC30001A29AD46B6F818399A4202D3414BC6F8C4
:10CC40001839414BFF22414C03F1780086F8CC2B78
:10CC500013F9082C142A05D053F80C1C34EA0101EE
:10CC600000F0E7800C339842F2D1394B5A79022A0E
:10CC700000F0AB800C37BD46BDE8F08F3549364833
:10CC800050F054FCB0E5354A11467A60DA0001EB09
:10CC9000C30393F8A41021B1D3F8A830002B00F0FF
:10CCA000E0807B68134493F8A520002A3FF45AAD36
:10CCB00093F88431002B7FF455AD182386F8FC37A8
:10CCC00050E54FF4F073A9F800300AE6244A35E63F
:10CCD0003B680022002B3FF412AF99F81130002B73
:10CCE0007FF413AF99F80530012B3FF408AF002A09
:10CCF0007FF405AF09E788B02022FF21E9464846C6
:10CD000064F01CFF0E4A03E0424549F823308ED000
:10CD100012F8013F59F823100131F5D081E70023C3
:10CD200089F80430B8F1000F00F0BD8001233B60AA
:10CD3000CAE600BFBDD77718FDFDFFFF481C0020E5
:10CD40009A2F0024AE014A01F46100240100020080
:10CD5000A8310024E8610024DCC40C08D83A0B0890
:10CD6000F6DFFFFD8F2F00243D5D002496F81B3871
:10CD7000002B00F087800023E80486F82B383FF56D
:10CD8000F0AD29067FF5EDAD96F8FC27182A04D8FA
:10CD90004A4BD340DA073FF5E4ADDFF834A10AF19E
:10CDA0007804FBE5AB047FF5D1AD454AC6E599F8BB
:10CDB0000630002B3FF42FAE99F81130012B7FF491
:10CDC0002AAE022389F8113025E63E4A1279002A5C
:10CDD0007FF450AF0C375A71BD46BDE8F08F002884
:10CDE0003FF412AD90F904404FF0FF0901E080F8E4
:10CDF000089020460FF022F90028F8D104E596F8B3
:10CE0000180A0EF09FFD00287FF437AEA6F81C0A22
:10CE100033E62D4A92E52D490B430A43C6F8C03844
:10CE2000C6F8142924E62B2025F0D2FAD6F83828A3
:10CE3000D3E686F8CC2B18E7D6F8143925F48055BC
:10CE400023F48053C6F8C058C6F81439B9F8203016
:10CE5000B3F57A7FBFF445AD4FF47A73A9F820306B
:10CE60003FE5172386F8FC371BE7D6F8C03823F0D8
:10CE70000063C6F8C038D6F8143923F00063C6F84A
:10CE8000143995E542F201031D427FF474AF65E564
:10CE9000D6F8143925F0800523F08003C6F8C05871
:10CEA000C6F81439B0E4424617E7D6F8143945F00D
:10CEB000080543F00803C6F814393EE500410001B7
:10CEC000F6BFFFFDB0310024F79FFFFD0004050011
:10CED000306300242DE9F04F844E83B096F8D03BA8
:10CEE000013B012B40F2EC80D6F8002C804BDFF8A0
:10CEF000208202F2DC524345C6F8002C80F0F2801A
:10CF0000DFF8109201229B467A4D09F10207019247
:10CF1000B9F80210002900F0BD80052907EB0102D5
:10CF200040F2B880AA4280F0B580BBF800003C46D1
:10CF3000C0F30B000BE0118814460A44002900F0EE
:10CF4000A980AA4280F0A680052940F2A3806188CA
:10CF50008142F0D161798B07EDD123885846DBF807
:10CF6000081094F804A0009350F0E0FABBF8001009
:10CF7000BAEB113F00F0948000230193BBF804103A
:10CF80000BF11C0B5BF8140CC1F30B015BF8044CA8
:10CF900056F0D4FBC3452060BAD3D6F8C038564CFF
:10CFA000C6F81439FFF7D0FB96F8E437EA22534D60
:10CFB00003FB0242A4F18003C6F8F82796F8E527A0
:10CFC00003EB4213C6F8F43724F000FC4FF0FF33B4
:10CFD000D6F8F8072B652DF001FC25F03FFA04F593
:10CFE000AF6304F5BE6102E00633994262D01A785D
:10CFF000002AF9D19C78D878844202D35879002845
:10D00000F2D096F88039B6F8841985F8542003EBED
:10D010008303642203EB830302FB01F100229B00E4
:10D020006429C6F8002CC6F8042CB8BF6421642B10
:10D03000C6F8082CB8BF6423C6F8FC1BC6F8141C3D
:10D04000C6F8F83B2E492F4BC6F80C2CC1F84C37CC
:10D05000C6F8102CA6F8182C86F81A2C30F09AFE78
:10D0600096F81E1CB6F81C0C27F028FE3FF0AAF814
:10D0700019F01EFA96F8D03B013B012B2AD9224B1E
:10D08000012201981B6886F8192CC6F8003C03B0F1
:10D09000BDE8F08FDBF80810584650F047FA6BE710
:10D0A000009BA11D58469A1F50F076FA00287FF485
:10D0B00065AF61E796F8F327003A18BF0122A0E7B1
:10D0C000F4F7C4FD114B0222034486F8F02BC6F896
:10D0D000EC3B09E7F4F7BAFD0223C6F8EC0B86F83F
:10D0E000F03BCCE70123019357E700BFA859002488
:10D0F000E0C30C0800000408B85D002418050024F3
:10D10000481C002018630024A41E002460E31600BD
:10D1100028CE0C0800000208114B0122032810B58C
:10D12000044683F8542705D9601CBDE81040C0B2FE
:10D1300010F0E0B80B4BEA2203F5826083F8E44775
:10D1400004FB0200C3F8F8072DF048FB2CF0ECF8C4
:10D150002CF0CEF9601CBDE81040C0B210F0CAB887
:10D16000481C0020A8590024054B0121D3F8242C89
:10D1700083F8201C42F40012C3F8242C704700BF2F
:10D18000A859002470B5046886B005460E46C4F35D
:10D19000100343BB01220393CDE901332023CDE9E2
:10D1A000042304F17843B3F5801F1AD3A4F101637B
:10D1B000B3F5801F10D2A4F58013022203F1784347
:10D1C000694601A802925B0C039351F085FA50B1B5
:10D1D0004FF0FF3006B070BD052057F029FF58F022
:10D1E00071FB2346EAE73146204657F01BFB18B98E
:10D1F0002B6820332B60EDE76FF00200EAE72DE9A2
:10D20000F0416B4E90B03378B12B7ED1FDF75BFFD0
:10D2100080F00104E4B2674B04F00104664DB3F8FA
:10D220006B32664FADF80030BD4270D3002C00F079
:10D23000BC802822002106A864F080FC604B049684
:10D240009B1B05935F4BDA68D40770D45D4BD3F812
:10D250000C21D00774D44FF480730222694604A8CD
:10D26000ADF83C3060F022F9022269464FF6FF70BB
:10D27000514DFDF70DFF4FF000080446BD4269D344
:10D280000025022201A904A8ADF8045060F00EF9AF
:10D29000022201A92046FDF7FBFE40BA022202A9A4
:10D2A000C043ADF8080004A860F000F90E9888B1FA
:10D2B00006ABC0F120022946184464F03FFC9DF9FA
:10D2C0003C0018B906A904A8FFF75CFF00238DF8FD
:10D2D0003C000E939DF83D307BB13A4BDA6842F04A
:10D2E0000102DA60DA68D20707D5D3F80C2142F0E0
:10D2F0000102C3F80C21D3F80C319DF93C00B0FABF
:10D3000080F0400910B0BDE8F081012483E7AB69EB
:10D310001C3535F8181CD3F8008055F8140CC1F3EF
:10D320000B0156F00BFA804518BF01247CE7264A12
:10D330005A6002F188325A60DB68D90786D58AE7DD
:10D34000214AC3F8042102F18832C3F80421D3F83A
:10D350000C3180E7AE8802A904A88DF80D80C6F3D1
:10D360000B061C35B31DADF8083035F81C3CC3F373
:10D370000B021B0BADF80A2006228DF80C3060F072
:10D3800095F8062202A92046FDF782FE044655F8CC
:10D39000141C324604A860F089F8204655F8141C85
:10D3A0003246FDF775FE044668E70120AAE700BF94
:10D3B00000000208D83A0B08E0C30C0828CE0C087D
:10D3C00000000408002000522301674570B5284C76
:10D3D000FFF7BAF994F8D03B013B012B35D9D4F8CB
:10D3E000003C01220325234E03F2DC5384F8282C51
:10D3F000C4F8003CFFF703FF58B13378B12B08D1D4
:10D40000FDF761FE013D0BD060B9FFF7F8FE002883
:10D41000F3D1013DEED1052057F00AFE58F052FA43
:10D420000028F8D094F8D03B0022013B84F8282C47
:10D43000012B14D9104B012100221B6884F8191C00
:10D4400084F8292CC4F8003C70BDF4F7FFFB0B4BAB
:10D450000222034484F8F02BC4F8EC3BBFE7F4F756
:10D46000F5FB0223C4F8EC0B84F8F03BE2E700BFC5
:10D47000A859002400000208A41E002460E316003E
:10D4800010B5084A0124084B82F8544783F8F24744
:10D49000FFF79CFFFFF71EFD2046BDE810400FF090
:10D4A00029BF00BF481C0020A859002490F89230E2
:10D4B000B7EE007ADFED6A6A014607EE903A90F81F
:10D4C0009630684AB0EE476A05EE103A90F894300C
:10D4D000F8EEE77A04EE903A90F89530B8EEC55A37
:10D4E00005EE903A90F8983067EEA67A04EE103A7E
:10D4F00025EE265AF8EEE44AF8EEE55AB8EEC44AAC
:10D5000025EE275A64EEA64A65EEA65A24EE264A70
:10D5100064EE854A65EEA75A24EE274AB0EE473AF4
:10D52000F0B590F8917000F16F0602F11805002433
:10D53000137807EE903AF8EEE77A67EE857A67EEB1
:10D54000867AFDEEE77A17EE903AFA2BA8BFFA2317
:10D5500023EAE3730B72537807EE903AF8EEE77A1A
:10D5600067EEA47A67EE867AFDEEE77A17EE903AD8
:10D57000FA2BA8BFFA2323EAE3734B72937803EEE6
:10D58000903AF8EEE33A63EEA57A67EE877AFDEE1D
:10D59000E77A17EE903AFA2BA8BFFA2323EAE3734F
:10D5A0008B72938807EE903AF8EEE77A67EE847A0A
:10D5B00067EE867AFDEEE77A17EE903AD5ED007ABF
:10D5C000B3F57A7FF8EEE77AA8BF4FF47A7323EACF
:10D5D000E3738B812B68002B3FDD90F89730B0EE22
:10D5E000436A02EE903AF8EEE22AA2EEE66A63EEB1
:10D5F000863A83EEA76AA2EEA66A65EEA77A0134A0
:10D6000067EE877A67EE867AFDEEE77A17EE903A54
:10D61000FA2BA8BFFA23BC4223EAE37306F8013FC2
:10D6200000DDF0BD012C13D190F8933007EE103AD5
:10D6300090F89B3006EE103AB8EEC77AB8EEC66A9C
:10D6400027EE267A26EE266A0435083208316FE77F
:10D65000B7EE007AB0EE476AF6E7B7EE006ACCE7BD
:10D660000AD7233C10420B0890F899306BB3B0F8FE
:10D6700064308BB190F89A20642102EB8203C3EBF3
:10D680000313B3FBF1F3A0F86430962312FB03F30A
:10D69000B3FBF1F3A0F8663043884BB190F89A30B1
:10D6A000642203EB8303C3EB0313B3FBF2F3438066
:10D6B000B0F850304BB1962290F89A3013FB02F339
:10D6C0006422B3FBF2F3A0F85030704790F8213099
:10D6D0004BB3438B83B190F82230FA22642113FBC1
:10D6E00002F203EB8303B2FBF1F2B3F57A7F4283DC
:10D6F000A8BF4FF47A738383838843B1FA2290F8EA
:10D70000223013FB02F36422B3FBF2F38380C3885D
:10D710004BB190F8223003EB8303B3F57A7FA8BFB7
:10D720004FF47A73C380704710B5064C4FF4807283
:10D73000002104F50F7064F001FA0023C4F83C33B3
:10D7400010BD00BFA06A0024034BD3F8400308B10A
:10D7500005F0A6B9704700BFA06A002408B50B46C3
:10D7600005490246D1F8400328B10449FEF706F8FE
:10D77000BDE80840E8E708BDA06A0024E9A0040865
:10D78000024B0146D3F84003FCF7B0BCA06A00246A
:10D790000048F5E7FBCA0B080CB4C30607B500D573
:10D7A00061B905A904980191FFF7D8FFFFF7F0FFD1
:10D7B000012003B05DF804EB02B070470020F8E7E9
:10D7C00008B5FFF7DDFFBDE80840E1E710B5044606
:10D7D0000348FFF7D5FF2046BDE81040F0E700BF43
:10D7E0007EC70B08034B0146D3F8400308B105F090
:10D7F00043B97047A06A00240CB407B510F02000AC
:10D800000BD079B92320FFF7EDFF05A9049801910A
:10D81000FFF7A4FFFFF7BCFF012003B05DF804EBA6
:10D8200002B070470020F8E70FB407B504A951F81B
:10D83000040B0191FFF792FF03B05DF804EB04B015
:10D8400070477FB52948FFF79BFF294B1B7923B908
:10D85000284804B0BDE87040B2E7FCF763FC08B9A3
:10D860002548F6E7FCF774FC08B92448F1E7244D95
:10D870002B68DB6998470028F7D0FCF74DFC02685D
:10D880000446037D81795208407CE61D0C340290E9
:10D8900020790190E08800901A48FFF7C5FF16F83C
:10D8A000010BFFF79FFFB442F9D11748FFF768FF5C
:10D8B00095F8FD30022B06D007D9032B0ED1134863
:10D8C000FFF75EFF0AE01248FAE71248FFF758FF39
:10D8D00095F8E432022B05D0032B05D004B0BDE847
:10D8E000704055E70C48EBE70C48E9E783C70B08A5
:10D8F000B03100248DC70B089CC70B08AAC70B08C2
:10D90000A8590024B9C70B08E7C70B08EDC70B08D7
:10D91000F3C70B0800C80B0806C80B081FC80B0884
:10D920000FB407B504A951F8040B0191FFF716FFD6
:10D93000FFF72EFF03B05DF804EB04B070472DE94C
:10D94000F04385B0214EFAF71FF80269838900255C
:10D950000188044602928268DFF88480019242883E
:10D96000DFF880901A4F009242681A48FFF7D8FFFC
:10D9700015B91948FFF724FFD8F800309D4212DA94
:10D980003378052B20D809EB8303D3F85C27B388C1
:10D990002946013538460093063636F8043CFFF731
:10D9A000BFFF062DE4D156F091FC4288838864685D
:10D9B0009B1A03FB0444FAF783F802460748214602
:10D9C00005B0BDE8F043ABE70022E0E7E46D0024DA
:10D9D0009BC80B0831C80B088FC80B08AAC80B08D6
:10D9E0009C310024D83A0B080EB403B503AA52F8B0
:10D9F000041B0192FDF7E5FF074BD3F840332BB929
:10DA0000064B0749D3F88403FCF770FB02B05DF8BE
:10DA100004EB03B0704700BFA06A0024A85900249B
:10DA2000FBCA0B080EB403B503AA52F8041B0192FB
:10DA3000FDF7C7FF054B0649D3F88403FCF756FBF7
:10DA400002B05DF804EB03B0704700BFA859002492
:10DA5000FBCA0B082DE9F04798460B7981460F4623
:10DA600003F0E0051646402D32D10024614DDFF869
:10DA7000A081DFF8A89116E03B7903F00703013B92
:10DA8000042B04D8DFE803F014171A1D2100315DC0
:10DA90005848FFF7C9FE7B79013BA34202DD4846A7
:10DAA000FFF76EFE01347B79A342E5DCBDE8F08729
:10DAB00031572846EDE736F81410FAE736F9141016
:10DAC000F7E756F824104046E3E756F82410F0E74D
:10DAD00003F00703052B56D8DFE803F0031E2628C2
:10DAE0002B3D3478602D54D02BD8002D72D1B7F84F
:10DAF0000550B7F8076021463E48FFF795FEAC4257
:10DB000038DBB44236DCB8F1000FCFD032462946BC
:10DB10003948BDE8F04787E696F90040602D38D0D7
:10DB20000FD8002D56D14FE03488DBE7B6F900401E
:10DB3000F4E7D6F800A0202D54464BD033D9602D01
:10DB400027D0802DB2D132782C4B2D48002A14BF1B
:10DB50003146194634E0202D34683BD0EFD82146B9
:10DB60002448FFF761FED7F80510A14202DB4B42C3
:10DB7000A34220DDFFF70CFE23463A6848462149C0
:10DB8000BDE8F04730E7202D23D01CD9602DD8D137
:10DB900000247B7944FA03F3DB07BDE8F0474CBF70
:10DBA00019481A4840E651461948FFF73DFED7F894
:10DBB00005108A45DED8B8F1000F3FF477AF15485D
:10DBC000BDE8F04730E60024B7F90550B7F9076023
:10DBD00091E700247A79104B03EBC20393F878277E
:10DBE000A242C7DDD3F8743753F82400BDE8F047EC
:10DBF000C6E500BF19F20B081DCD0B0840EA0B0863
:10DC00003DD30B08CFC80B086FC90B084DF10B08AB
:10DC100007C90B08C9C80B08D83A0B08C7C80B08B6
:10DC2000F0B5067906F0E003402B03D145794FF0BB
:10DC3000FF3406E0602B4FF00105F8D1447905FA76
:10DC400004F40023012006F00706AB4200D1F0BD2A
:10DC5000052E0FD8DFE806F00308101D242448B174
:10DC6000C85CD75C78400FE020B1C856D756C71BB8
:10DC7000784278410133E8E70028FBD031F81300FF
:10DC800032F81370784080B220420CBF012000208F
:10DC9000F0E70028EED031F9130032F91370E6E70F
:10DCA0000028E7D051F8230052F82370DAE708B5CE
:10DCB000034610460AB9002008BDDB0601D500293D
:10DCC000FAD0FFF783FDF6E7F8B50D4E054696F856
:10DCD000683393B9F8BD25B12388C3F30B039D4284
:10DCE00004D0A288D4E9020163F032FE1C34BC42A5
:10DCF000F1D3002386F86833ECE7024C024FF6E7D5
:10DD0000A06A0024E0C30C0828CE0C08037903F0B5
:10DD10001803102B1ED003D833B9B0F80B0070478E
:10DD2000182BFAD000207047124BB0F80B0093F973
:10DD30001831591C0CD1104B93F8E43703EB430214
:10DD400003EB820303EBC30300EB430080B2704795
:10DD5000DBB2F3E7074BB0F80B0093F919315A1C0B
:10DD600005D1054B93F8E53700EB4310EEE7DBB246
:10DD7000FAE700BF18050024A859002470B505462D
:10DD8000B0F809004FF0BCFB064B0446284693F858
:10DD90006863FFF7BBFF16B1E368184470BDA36862
:10DDA000FBE700BFA06A00242DE9F04F164685B0BE
:10DDB000334C1A464FF00009A246CDE9010100217B
:10DDC0003046FFF774FF06F0100300900393FFF74F
:10DDD000BBFC2379029A03F01803934203D0002A74
:10DDE00044D1182B42D14FF00D0B0BFB09A3B3F814
:10DDF00009004FF085FB80462046FFF787FF074666
:10DE0000D8E90221024401442046FFF709FF80F0CF
:10DE100001010546009AC9B23046FFF748FF039B4F
:10DE2000009003B115BB0BFB09FBB3065AF80BB00E
:10DE30000ED56DB959461348FFF7F6FCD8F80820FF
:10DE40002B4621463A440198FFF704FEFFF7A0FC59
:10DE500059460D48FFF7E8FCD8F80C20002321466E
:10DE60003A440198FFF7F6FDFFF792FC09F101092A
:10DE70000D34B9F52C7FAAD105B0BDE8F08F00BFF5
:10DE80006C520B08E9C80B08EAC80B0870B51646B7
:10DE900005460C460846FFF771FF33460246214609
:10DEA0002846BDE87040D5E52DE9F041037903F03F
:10DEB000E002402A4AD009D82ABB03F00703052B09
:10DEC0001CD8DFE803F0161B161B090F602A44D08C
:10DED000802A3ED0BDE8F081D0F805102148BDE889
:10DEE000F0411DE5D0F8052051421F48BDE8F04142
:10DEF00016E5B0F80720B0F80510F6E7B0F90720EE
:10DF0000B0F90510F1E746790024184D184805EBE3
:10DF1000C605FFF735FC012395F87877A74202D8AC
:10DF2000BDE8F04134E4D5F874674FEA840856F848
:10DF300024204AB113B90F48FFF722FC56F8081005
:10DF40000D48FFF771FC00230134E7E741790B48E6
:10DF5000C5E7827941790A48C8E70A48BDE8F04137
:10DF6000DEE400BFF4C80B080AC90B08D83A0B0856
:10DF700021C90B08A7D60B083DD30B0832C90B08E3
:10DF800043C90B085AC90B0838B505460C46FFF7BC
:10DF9000F5FE2A7902F0070302F0E002602A29D197
:10DFA000052B0CD8DFE803F0030B0F0B1B1B6A7962
:10DFB000012393400278DBB214B11343037038BDE0
:10DFC00022EA0303FAE76A790123934002889BB2AD
:10DFD00014B113430380F2E722EA0303FAE76B79F3
:10DFE00001229A40036814B113430360E7E723EA70
:10DFF0000203FAE7052BE2D8DFE803F00303050587
:10E0000007070470DBE70480D9E70460D7E701491C
:10E0100008E500BF72C90B08004903E581C90B0878
:10E0200007B5009313460A460249FFF7FBFC03B00D
:10E030005DF804FB98C90B0808B5202163F095FD35
:10E04000034618461BB102780133202AF9D008BDD7
:10E0500070B50D461446FFF7EFFF0646A0B1FDF779
:10E060001BFE40F6340319229842A8BF1846B0F5AB
:10E07000617FB8BF4FF46170A0F56173B3FBF2F339
:10E080002B702378013323703046FFF7D5FF064607
:10E09000A0B1FDF701FE40F6340319229842A8BF53
:10E0A0001846B0F5617FB8BF4FF46170A0F5617399
:10E0B000B3FBF2F36B70237801332370304670BDED
:10E0C00020B10078B0FA80F0400970470120704715
:10E0D0002DE9F74F81460846FFF7F2FF0E46054649
:10E0E00070B1002401A92046013454F08BF9014697
:10E0F0004846FFF7EDFF122CF4D103B0BDE8F08FD6
:10E100000846FDF7C9FDC4B2112C70D83C4D701CF7
:10E11000FFF792FF3B4E05EB44088346670098F8F3
:10E120006CA3B8B9AAF102014B424B413D4495F8AA
:10E130006C23B25C002B53D095F86D33192040F25C
:10E14000EE2100FB031321462F4803B0BDE8F04F3A
:10E15000FFF7E6BB0178304663F007FD80B1032C82
:10E160002A49A0EB060394BF0022012202EB4202DF
:10E170000A4452FA83F393F844A9BAF1030F04D185
:10E18000484603B0BDE8F04F41E75846FFF754FF5B
:10E19000F0B1BAF1020FF3D1FDF77EFD40F6CA03EC
:10E1A00080B29842A8BF184640F2EE239842B8BF0A
:10E1B00018461923A0F2EE20B0FBF3F088F86D03A7
:10E1C000AAF1020253425341EA1982F86CA3ADE767
:10E1D000BAF1020FF4D1484603B0BDE8F04F1BE797
:10E1E00021460B4803B0BDE8F04FFFF799BB112360
:10E1F0002A460849484603B0BDE8F04F10E700BF83
:10E20000A06A002410020C08B1C90B08D83A0B0808
:10E21000C1C90B08CEC90B082DE9F04F0346A1B0C8
:10E220000846FFF74DFF054620B1184621B0BDE86E
:10E23000F04FF1E6FF23DFF8C09207464FF0FF38BA
:10E240008DF82830D9F890330B9093F83820ADF83A
:10E2500030000D908DF838200F90ADF840001193EC
:10E260000991CDE90500934909A863F03BFB0446F9
:10E2700018BB01460AAC904F0B0190481A57002377
:10E2800010F9016BB24240F0D2804E1C104654F09F
:10E29000A3F8024631463846FFF742FB022E4FF004
:10E2A0000101E9D19DF938A09DF92830534540F08E
:10E2B000C5808348FFF734FB4DE02378002BD2D094
:10E2C000032FD4BF00260126062F00F2A980DFE825
:10E2D00007F00447509104475000042F10D07949AB
:10E2E0002046FDF737FC58B14FF480600DF0D4FEA6
:10E2F000002800F0B48190F90400012306930AE09D
:10E3000071492046FAF776FB70B9D9F8903393F942
:10E310003800042F22D0119B119320AB03EB06167B
:10E3200006F8580C01379EE7204653F04BFF0028B3
:10E33000EFDA01230A2212A92046FDF723FC40B29E
:10E34000002803DB129B1B78002BE2D02246711CB5
:10E350005E48FFF7E5FA21B0BDE8F08F0023DBE768
:10E360002046FDF799FC20AB03EB061646F8540C4B
:10E37000D8E757492046FDF7EDFBB0F1000A5549B3
:10E38000204618BF4FF0010AFDF7E4FB08B14AF040
:10E39000020A3301DFF864C1079320AB03EB0616D2
:10E3A000BCE80F0006F850AC12AE0DF1480A0FC6DB
:10E3B000BCE80F000FC6BCE80F000FC69CE80300C6
:10E3C00086E803000026B346DAF80010204663F022
:10E3D0001BFC10B19AF804301E430BF1010B0AF13B
:10E3E000080ABBF1070FEFD1079B80336B4403F89A
:10E3F0004F6C97E738492046FAF7FCFAA0B1374945
:10E400002046FAF7F7FA00288CD02046FDF744FCA6
:10E410000228804686D901463148FFF781FA9AE7FB
:10E42000224608212F4894E7012305937AE7013318
:10E430000A2B7FF425AF01312B488AE70B9B1BB9D0
:10E44000AAF114025542554100235F1CE368002BDA
:10E4500061D194F900B058460DF0F0FDD4F8049065
:10E4600018B10668002E40F08A80B9F1000F237AB7
:10E4700014BF4E464FF46146666023B91B48FFF750
:10E480004FFA03232372627A2AB139461848079259
:10E49000FFF746FA079A02925846237ACDE90063BD
:10E4A00000231A4619460DF011FEE06040BB3946C4
:10E4B0001048B2E7C6EF0B0858CA0B08E73F0B0835
:10E4C00075CA0B08F1C90B08FCC90B0800CA0B0878
:10E4D0001BCA0B0884E80B081ECA0B08E8DD0B08F2
:10E4E00024CA0B083CCA0B0863CA0B088ECA0B0867
:10E4F000A9CA0B08C4CA0B08A06A002424440B084C
:10E5000058493346584A5948B9F1000F18BF0A46CE
:10E510003946FFF789F9022F04F110044FF0010387
:10E5200093D1119E0D9F4DB15148FFF749F93368C2
:10E530001B6A1BB13A464F4930469847059B002B52
:10E5400050D04D49474BBAF1140F18BF19464B48EC
:10E55000FFF7E6F9BAF1140F09D1059B002B43D060
:10E560003368DB691BB10022454930469847069B5A
:10E57000002B43D100223146384653F03BFEE66083
:10E58000B9F1000F2CD04946304607F0A9FF3D4AAB
:10E59000B36839463C48FFF7C3F994F80890B9F1DD
:10E5A000000F0CD03279914509D04B463946374897
:10E5B000FFF7B6F93368494630469B699847637A56
:10E5C00023B1727939463248FFF7AAF9F36A002B72
:10E5D000A1D039462F48FFF7A3F90023F3629AE749
:10E5E000204AD5E71F49B2E7B8F1000FBFDB336817
:10E5F000DB69002BBBD042462749B6E7DFF89C9089
:10E600000025DFF89CA04FF0030B05F0DDFB052093
:10E61000F8F7AAFB9AF8A035AB42ABD919F8014F2D
:10E62000C4B120460DF08EF9804698B12046F5F72A
:10E630005DF80446EBB210B180F806B0C371204615
:10E640000121F4F731F898F806302046DB0703D5AE
:10E65000F3F75CFE0135DDE7F3F752FEFAE74FF022
:10E66000FF304AE6FDCA0B08D6C90B08E0CA0B0802
:10E6700096CB0B08E1640508E4C90B08BFCB0B0877
:10E680000DA10408DFC90B08FECA0B0823CB0B0839
:10E6900046CB0B087DCB0B08E58C04088F2F00249C
:10E6A000481C00202DE9F04F914687B00C461A46D1
:10E6B000002180464D46FFF7FAFA00270646B9F1D9
:10E6C000000F63D029460622204663F00DFA002889
:10E6D0003246404613BF012100214FF0010A4FF09E
:10E6E000000AFFF7E4FA0646287817F06DFE834625
:10E6F000F8B1687917F068FE4FF461714FF0190CAA
:10E70000AB78EA789BF805E01CFB03131CFB0212B4
:10E7100095F801B0297900B14079CDE90410CDE92F
:10E72000023251463B461A4A4046CDE900EBFFF71C
:10E7300063F8207817F048FE8346F8B1607917F047
:10E7400043FE4FF461714FF0190CA378E2789BF807
:10E7500005E01CFB03131CFB021294F801B02179A5
:10E7600000B14079CDE90410CDE9023251463B4673
:10E77000074A4046CDE900EBFFF70EF801370634B3
:10E780000635142F9BD107B0BDE8F08FCA46D0E7FD
:10E79000E2CB0B082DE9F041054686B008460F464E
:10E7A000FFF78EFC064638B100235B4901201A466C
:10E7B00006B0BDE8F04175E70846FDF76DFA13288D
:10E7C000044600F3A08006258DF81760534E45439C
:10E7D000781CFFF731FC074660B1FDF75DFAC0B267
:10E7E00017F00CFE30B17319027983F888290123E0
:10E7F0008DF817303846FFF71FFC074668B1FDF764
:10E800004BFA0D2809D8062303FB046383F8890912
:10E810009DF8173001338DF81730DFF8FC80A91C04
:10E820000DF1170238464144FFF712FCFFF704FCD4
:10E83000074668B1FDF730FA012809D89DF817306E
:10E840000622013302FB04628DF8173082F88C092E
:10E850003846FFF7F1FB80B1FDF71EFAC0B217F0A2
:10E86000CDFD50B19DF817300622017902FB0462FC
:10E87000013382F88D198DF817309DF81720062383
:10E88000042A2FD103FB04630022A3F88C29062558
:10E8900023F0E4FD05FB046595F8880917F094FD65
:10E8A00095F88B1995F88A7919234FF4617280468F
:10E8B00095F88D0913FB012613FB072717F084FD3C
:10E8C0004379214698F80520039395F88C3914482C
:10E8D0000097CDE9016395F88939FFF721F806B073
:10E8E000BDE8F081052A05D103FB0463002283F80B
:10E8F0008D29CCE7062ACAD0002308EB050248F888
:10E9000005309380C3E7132332460649284606B0F4
:10E91000BDE8F041FFF784BB30630024A859002410
:10E92000E2CB0B08FBCB0B082DE9F04F904689B0EA
:10E930001A460C46002181464546FFF7B8F93A4E83
:10E9400008F178030746DFF8E4B0079394F9040070
:10E950000DF074FB00285CD0B8F1000F61D029469F
:10E960000C22204663F0C0F800283A46484613BF00
:10E97000012100214FF0010A4FF0000AFFF797F93B
:10E98000074695F9040053F027FDEA7903465146FE
:10E9900006EB82024846D2F8842904922A7A06EBD2
:10E9A0008202D2F884290392AA7906EB8202D2F875
:10E9B000842902926A7906EB8202D2F884290192B4
:10E9C0002A6800925A46FEF717FF94F9040053F0A4
:10E9D00003FDE2790346514606EB82024846D2F82F
:10E9E00084290492227A06EB8202D2F884290392C7
:10E9F000A27906EB8202D2F884290292627906EBB0
:10EA00008202D2F884290192226800925A46FEF7C7
:10EA1000C3FE0C35079B0C34AB4297D109B0BDE85F
:10EA2000F08FC246D1E700BFD83A0B0801CC0B08E3
:10EA30002DE9F04780468CB00846FFF741FB0546BC
:10EA400038B10023594901201A460CB0BDE8F047FF
:10EA50006AE7CDE909000B9007A80791544962F0D5
:10EA600041FF064653F0AEFB431C04460CD12B4637
:10EA70000A2208A93046FDF785F8089B1B781BB9C8
:10EA8000C4B2132C0BD944B220460DF083FA0546CC
:10EA900040B94046FFF7BBFA0CB0BDE8F08733340D
:10EAA00064B2F1E7424907A88DF8284062F01AFFE6
:10EAB000B0B3002302260A221946FDF763F8099035
:10EAC0000027DFF8EC90DFF8F0A0494607A862F0D5
:10EAD00009FFF8B1FDF7E0F8364A002352F8041BAD
:10EAE00088421FD1DBB20AEB8302D2F8842990421C
:10EAF00010D1022F20D0032F23D05A1E012FD2B2C3
:10EB000015D00B2A03D88DF829300136F6B201371B
:10EB1000042FDAD1052E1AD84046FFF77DFABBE75D
:10EB20000126CDE70133102BD8D10023DBE7052ADE
:10EB3000EDD88DF82A30E8E7092BE8D88DF82C308D
:10EB4000E3E79A1E0D2AE2D88DF82B30DDE709ABFA
:10EB500003CB286018686960A860204653F03CFC2D
:10EB6000154A9DF82B10034602EB8101D1F8841958
:10EB700004919DF82C1002EB8101D1F884190391C6
:10EB80009DF82A1002EB8101D1F8841902919DF8B9
:10EB9000291002EB81020021D2F884290846019253
:10EBA000099A0092054AFEF7F7FD75E7E86100242F
:10EBB000C6EF0B085C440B08D83A0B0801CC0B08D5
:10EBC0002DE9F04F90468BB000264FF0190A4546CC
:10EBD0004FF461790C461A4600210746FFF767F8A3
:10EBE0000990B8F1000F49D029460A22204662F068
:10EBF0007BFF0028099A384613BF012100214FF0FE
:10EC0000010B4FF0000BFFF752F82A8909903346A9
:10EC100006925946EA88384605922A790492EA789B
:10EC20000392AA781AFB029202926A781AFB029265
:10EC300001922A780092124AFEF7DEFD22893346BD
:10EC40000136594606923846E2880A3505922279FD
:10EC50000492E2780392A2781AFB029202926278FE
:10EC60001AFB0292019214F80A2B0092044AFEF752
:10EC700093FD1E2EB5D10BB0BDE8F08FC346DDE786
:10EC80001ECC0B082DE9F04380468BB008460F469A
:10EC9000FFF716FA044638B100235E4901201A46F0
:10ECA0000BB0BDE8F0438BE70846FCF7F5FF1D28E5
:10ECB000054600F3A5800A268DF827404643781CB8
:10ECC000FFF7BAF910B101238DF82730FFF7B4F937
:10ECD000514C074668B1FCF7DFFF0D2809D80A231D
:10ECE00003FB054383F894039DF8273001338DF827
:10ECF0002730DFF82091711C0DF127023846494476
:10ED0000FFF7A6F9FFF798F9074668B1FCF7C4FFCB
:10ED1000232809D89DF827300A22013302FB054237
:10ED20008DF8273082F897033846FFF785F90746B4
:10ED300068B1FCF7B1FF0D2809D89DF827300A22E9
:10ED4000013302FB05428DF8273082F898039DF8C5
:10ED50002730062B0CD0002309EB0602404649F869
:10ED60000630536013810BB0BDE8F043FFF754B990
:10ED70000A260023384606FB0546A6F89A33A6F86D
:10ED80009C33FFF759F9074618B1FCF785FFA6F841
:10ED90009A033846FFF750F930B1FCF77DFF0A239C
:10EDA00003FB0543A3F89C031C4B4FF0FF324FF4C9
:10EDB00061701A650A2303FB0542B2F89C3306937F
:10EDC000B2F89A33059392F89833049392F89733F4
:10EDD0000393192392F8961313FB0101029192F801
:10EDE000951313FB010300210193084692F8943315
:10EDF0000B4A00932B46FEF7CFFC0BB0BDE8F08327
:10EE00001D232246074940460BB0BDE8F043FFF7FB
:10EE100007B900BF346E0024A06A0024180500243E
:10EE20001ECC0B08FBCB0B082DE9F04F804691461A
:10EE30001E460C4615460027DFF81CA12DED088B59
:10EE400095B094ED008AB5EE408AF1EE10FA7BD0D1
:10EE5000D4ED019A94ED029AD4ED038AB9F1000F32
:10EE600049D0D5ED00BA95ED01BAB4EE6B8AD5ED77
:10EE700002AA95ED03AAF1EE10FA6AD1F4EE4B9ACC
:10EE8000F1EE10FA65D1B4EE6A9AF1EE10FA60D1A3
:10EE9000F4EE4A8AF1EE10FA0CBF0121002132464D
:10EEA0008B46404681F00101FEF701FFB0EE6B0A90
:10EEB000064611A8FBF7A6F8B0EE4B0A07900EA87D
:10EEC000FBF7A0F8B0EE6A0A06900BA8FBF79AF8D9
:10EED000B0EE4A0A059008A8FBF794F80599069A3F
:10EEE000079B039040460291594601925246009377
:10EEF0003B46FEF781FCB0EE480A11A8FBF782F80A
:10EF0000B0EE690A83460EA8FBF77CF8B0EE490A1A
:10EF100006900BA8FBF776F8B0EE680A059008A8F3
:10EF2000FBF770F8069B059A002103904046029279
:10EF3000524610341035CDE900B33B460137FEF799
:10EF40002BFC082F7FF47DAF15B0BDEC088BBDE81E
:10EF5000F08F0021A3E700BF41CC0B082DE9F14F52
:10EF600006460C46DFF894B12046FFF7A9F807469D
:10EF700038B100235A4901201A4601B0BDE8F04FCC
:10EF800052E7052257492046FCF7C0FD60B9544BB3
:10EF900000221A601A611A621A631A641A651A66E4
:10EFA0001A6701B0BDE8F08F042259462046FCF7ED
:10EFB000ADFD05462046002D45D1FFF73DF807463B
:10EFC0000028EED05FF0B0FBDFF834A15FFA80F8E4
:10EFD0005AF8049BB9F1000F07D122464249304646
:10EFE00001B0BDE8F04FFEF71DBD42464946384628
:10EFF0000135FCF78BFD84460028E9D1384A0346E9
:10F0000000211746013342F8101B082BFAD1374B69
:10F0100003EBC505D5F8A8E0BEF1000F05D14946C0
:10F020003348344CFEF77CFC9EE795F8A450AC4581
:10F03000F5DA0EEB0C1307EB0C140CF1010C0FCBF3
:10F0400084E80F00F3E7FCF727FE072805463DD8C4
:10F050002046FEF7F1FF074658B3F9F769FD204B4C
:10F06000012403EB051383ED000A3846FEF7E4FFA5
:10F07000074638B1F9F75CFD194B013403EB051372
:10F0800083ED010A3846FEF7D7FF074638B1F9F796
:10F090004FFD134B013403EB051383ED020A384691
:10F0A000FEF7CAFF38B9304601B0BDE8F04FFEF7B1
:10F0B000B3BF0446D9E7F9F73BFD094B032C03EB3B
:10F0C000051383ED030A3FF454AFECE707233A46F8
:10F0D0000949304601B0BDE8F04FFEF7A1BF00BFBF
:10F0E000586600241ECA0B085ACC0B08D83A0B08E5
:10F0F0006BCC0B08FDCA0B08FBCB0B0855CC0B08DF
:10F100009C440B082DE9F74F92460C461A46002105
:10F1100081465646FEF7CBFD00258046DFF864B0F9
:10F12000BAF1000F2CD031460422204662F0DCFCFC
:10F1300000284246484613BF01210021012700272D
:10F14000FEF7B5FD738880465A46019339463AF872
:10F150002530484600932B46FEF74EFB63885A46FF
:10F16000394648460193043634F8043B00932B4655
:10F170000135FEF711FB042DD2D103B0BDE8F08FAD
:10F180005746EBE775CC0B082DE9F34105460846D9
:10F19000FEF796FF0C46074638B10023334901209D
:10F1A0001A4602B0BDE8F041ACE731492046F9F714
:10F1B00021FC70B904222D4B4FF47A704FF4FA61A0
:10F1C000013A1880598003F10403F9D102B0BDE877
:10F1D000F0812046FCF760FD0328064641D8204612
:10F1E000FEF72AFF074698B1FCF756FD4FF00108DD
:10F1F00004463846FEF720FF20B1FCF74DFDB8F17C
:10F20000000F09D1284602B0BDE8F041FEF704BF67
:10F2100040F2EE248046ECE7A4F2EE2240F2DC530A
:10F220009A4203D8A0F2EE229A420AD940F6CA03C3
:10F2300040F2EE220F49284602B0BDE8F041FEF749
:10F24000EFBE0D4B00210D4A03EB8603A3F8C0442B
:10F25000A3F8C2043346CDE900400846FEF79CFA05
:10F26000B4E703233A460649E5E700BF606F002490
:10F270001ECA0B0886CC0B08A06A002475CC0B08AC
:10F28000CEC90B082DE9F04F8FB0894617460021F3
:10F290001A4606460024FEF70AFD0DF1240B05462A
:10F2A000DFF86CA059F82480594602A8CDF80880F0
:10F2B00053F042F84FB357F824302A463046984569
:10F2C000039313BF012100214FF001084FF0000804
:10F2D000FEF7EDFC04A9054603A853F02DF804A998
:10F2E00023465246009130464146FEF785FA2346B2
:10F2F0000134524641463046CDF800B0FEF74CFA94
:10F30000202CCFD10FB0BDE8F08FB846EFE700BF9B
:10F3100094CC0B08F0B5074689B008460E46FEF7B8
:10F32000CFFE054638B10023194901201A4609B01D
:10F33000BDE8F040A6E70846FCF7AEFC1F280446EF
:10F340001DD83046FEF778FE014620463DF08CF889
:10F3500078B103AE0E48314600EB840052F0ECFF6A
:10F3600023460C4A294628460096FEF715FA09B0AE
:10F37000F0BD384609B0BDE8F040FEF748BE1F2397
:10F380002A460549384609B0BDE8F040FEF748BEB8
:10F39000706F002494CC0B08FBCB0B082DE9F04FC9
:10F3A000924685B00C461A46002181465546FEF726
:10F3B0007EFC00268046DFF86CB0BAF1000F2FD03B
:10F3C00029460422204662F08FFB00284246484628
:10F3D00013BF0121002101270027FEF768FCEB780D
:10F3E00080465A4602933946AB78484601932B88AB
:10F3F00000933346FEF700FAE3785A46394648460A
:10F4000002930435A378019334F8043B0093334608
:10F410000136FEF7C1F9102ECFD105B0BDE8F08F4F
:10F420005746E9E79ECC0B08F0B5074685B008467D
:10F430000E46FEF745FE054638B100231C49012063
:10F440001A4605B0BDE8F040A8E70846FCF724FCE2
:10F450000F28044623DC3046FEF7EEFD0146204629
:10F460003DF0DCF8A8B104F12002124B29462846F1
:10F4700003EB820393F8D324029293F8D2240192EF
:10F48000B3F8D0340C4A00932346FEF785F905B053
:10F49000F0BD384605B0BDE8F040FEF7B8BD0F231B
:10F4A0002A460649384605B0BDE8F040FEF7B8BD2B
:10F4B000F06F0024A06A00249ECC0B08FBCB0B0845
:10F4C0002DE9F04F85B014461A46054602910021F9
:10F4D000FEF7EDFB4FF00008064606234FF000094B
:10F4E00003FB08F7C037029B13F807B0002C7AD053
:10F4F000E35D324628469B45039313BF012100215B
:10F500004FF0010A4FF0000AFEF7D1FB039B0646BD
:10F51000374A51462846CDE900934346FEF76CF939
:10F520004346334A514628460137CDE9009B09F14D
:10F530000109FEF731F9B9F1060FD4D108F101083C
:10F54000B8F1060FC9D1E427029BA7F1E40913F82B
:10F5500007A0002C49D014F807B032462846DA45F7
:10F560000DBF4FF001084FF0000801210021FEF708
:10F570009EFB062306461E4A41462846CDE9009BCF
:10F58000FEF73AF901370623194A41462846CDE9E4
:10F59000009AFEF701F9EF2FD6D1029B93F8EF7096
:10F5A000ACB194F8EF8032462846474513BF01219D
:10F5B000002101240024FEF77AFB00230C4A214697
:10F5C000009328460723CDF80480FEF715F90023A1
:10F5D000074A21462846009307230197FEF7DCF8E7
:10F5E00005B0BDE8F08FA2469AE7A046CAE700BF83
:10F5F000B0CC0B08F0B5054685B008460B46FEF7C3
:10F600005FFD044638B100231B4901201A4605B0AE
:10F61000BDE8F04054E701AE184F6A461749184656
:10F6200062F08DF988B1032C04D12846FEF7F4FC72
:10F6300005B0F0BDFCF730FB6A4646F8040B3946CE
:10F640000020013462F07BF9ECE7032CEDD1039F3D
:10F65000DDE901463A463146E0B23DF019F818B905
:10F660002846FEF7D4FCE3E73B46324621460448F1
:10F67000FEF756F9DCE700BF706F0024C6EF0B08F9
:10F68000B0CC0B082DE9F04F0E46154689B01A464E
:10F6900000210446B046FEF70AFB2F4681464FF094
:10F6A000000B002D7AD039460C22404662F01CFA3D
:10F6B00000284A46204613BF012100214FF0010ACD
:10F6C0004FF0000AFEF7F3FA97F90B2081465B46EC
:10F6D0000492514697F90A2020460392B7F9082070
:10F6E0000292B7F906200192B7F904200092364A37
:10F6F000FEF782F898F90B205B460BF1010B51469F
:10F700000492204698F90A200C3708F10C0803925D
:10F7100038F9042C029238F9062C019238F9082C99
:10F720000092294AFEF738F8BBF1080FB9D14FF023
:10F73000000BDFF898800C2303FB0BF985B300273F
:10F7400055F80900012356F8092003FA07FA424048
:10F750003AEA020214BF1946002110EA0A0F07D044
:10F760005B464246204600970791FEF745F8079909
:10F7700056F809201AEA020F05D05B464246204699
:10F780000097FEF709F801370E2FD9D10BF1010BC5
:10F79000BBF1080FCFD109B0BDE8F08FAA46A9E7A9
:10F7A0002F46012356F8091003FA07F20A4206D041
:10F7B0005B464246012120460097FDF7EDFF0137E9
:10F7C0000E2FEED1E2E700BFC4CC0B08DCCC0B0857
:10F7D000F0B506468BB008460D46FEF771FC0446B0
:10F7E00020B300233D4901201A460BB0BDE8F0408C
:10F7F00048E72D2903D0A1F13003092B49D8052C66
:10F8000005DD30460BB0BDE8F040FEF705BC2846EC
:10F81000FCF742FA0AAB621C03EB440424F80C0C1C
:10F8200015F8013F303B092BFAD9144629780029F5
:10F83000DFD1062CE5D1BDF81C20BDF91C30072A0C
:10F84000DFD8BDF91E50A5F5FA7292B2B2F5FA6F83
:10F8500018D8BDF92070A7F5FA7292B2B2F5FA6F16
:10F8600010D8BDF922C065450CDC67450ADBBDF93F
:10F8700024E00EF1640292B2C82A03D8BDF92640F2
:10F88000112C11DD164930460BB0BDE8F040FEF7F3
:10F89000C9B8202902D101352246C6E730460BB04F
:10F8A000BDE8F040FEF7B3BB0C200E4A64B200FB8B
:10F8B00003220846A2F8C455A2F8C675A2F8C8C526
:10F8C00082F8CAE582F8CB45074A0095CDE903E402
:10F8D000CDE9017CFDF760FF0BB0F0BD6070002446
:10F8E000F1CC0B08A06A0024C4CC0B082DE9F04F22
:10F8F00089468DB0164600211A4607460024FEF7B9
:10F90000D6F9DFF8DCA00546C4EBC40309EB03021B
:10F9100059F80300918840F3074892790890ADF8B0
:10F9200024108DF82620B8F1000F53D0002E54D0AB
:10F93000F218F0589188937907220A9008A8ADF838
:10F940002C100AA98DF82E3062F0CEF800282A4635
:10F95000384613BF012100214FF0010B4FF0000B7F
:10F96000FEF7A5F99DF82E300546524606935946F6
:10F970009DF92D30384605939DF92C3004939DF860
:10F980002B3003939DF92A3002939DF8293001937F
:10F990009DF8283000932346FDF72EFF9DF8263072
:10F9A00052465946384606939DF9253005939DF9F0
:10F9B000243004939DF82330CDE902839DF8213053
:10F9C00001939DF82030009323460134FDF7E4FEB7
:10F9D000102C99D10DB0BDE8F08FB346DEE700BF23
:10F9E00007CD0B082DE9F04F06468BB00D46DFF82A
:10F9F000A08228465EF098FE034630B9024696493A
:10FA000001200BB0BDE8F04F70E70522934928466E
:10FA1000FCF77CF80446C8B9914D0146702205F503
:10FA2000C46062F08BF8C5F8C045C5F8CC45C5F890
:10FA3000D845C5F8E445C5F8F045C5F8FC45C5F816
:10FA40000846C5F814460BB0BDE8F08F04224146C5
:10FA50002846FCF75BF8044630BB2846FEF7ECFA74
:10FA600081460028EFD05EF05FFEDFF828B28246C4
:10FA70005BF8047B3FB92A467A4930460BB0BDE8B3
:10FA8000F04FFDF7CFBF524639464846FCF73EF8E7
:10FA900040B92046744D2BF03FFA39467348FDF7C4
:10FAA0003FFFA6E70134E3E7072271492846FCF748
:10FAB0002DF8074600287AD12021284662F055F813
:10FAC000044670BB6B4D6C48FDF7AEFE2146013419
:10FAD0002846FDF7A9FE0E2CF8D10025DFF8B891D5
:10FAE000664FFDF755FEDFF8B4810C260024DFF8E1
:10FAF000B0A129466E434846FDF796FE0123F25910
:10FB00005F48A340013413420CBF41465146FDF704
:10FB10008BFE0E2CF2D10135FDF73AFE082DE4D113
:10FB200091E702AC574D01AA564961F008FF002841
:10FB300048D0022F11D1029A072A07D8039C0D2C16
:10FB400004D80378722B13D06E2B25D00823002203
:10FB50004D493046FEF764FA75E7FCF79DF801AAB7
:10FB600044F8040B29460020013761F0E8FEDEE787
:10FB70000C233B4903FB02110123D1F8C015A3401C
:10FB80000B4337490C2000FB02123949C2F8C0353B
:10FB90003046FFF727FF56E7314B0C20012100FBD1
:10FBA0000233A140D3F8C03523EA0103E9E7284630
:10FBB000002402AD334F01AA324961F0C0FE80B18A
:10FBC000082C03D13046FEF727FA3CE7FCF764F82F
:10FBD00001AA45F8040B39460020013461F0AFFE5C
:10FBE000EDE7082CEED1029B0F2B30D8DDF80CE0AE
:10FBF000BEF1070F2BD8DDF810C0BCF10D0F26D8D1
:10FC0000059F07F16402C82A21D8069DFF2D1ED842
:10FC1000079864281BD80899642918D8884216DAEE
:10FC2000099C032C13D8C3EBC3020D4B134483F878
:10FC3000251683F820E60C4983F821C683F822763E
:10FC400083F8235683F8240683F82646A0E70F4955
:10FC50003046FDF7E7FEF6E6C07000241ECA0B082A
:10FC6000A06A00245ACC0B08FDCA0B086BCC0B0809
:10FC700024CD0B082CCD0B083ED30B08607000245C
:10FC800031CD0B08C6EF0B0837CD0B08F1CC0B08B4
:10FC900055CC0B089C440B0819F20B084DCD0B08F2
:10FCA000EFCC0B0818B3A0F1800380F080000B2884
:10FCB0001FD80B2B1DD8DFE803F01E06080A0C0E18
:10FCC000101C121416180D4870470D4870470D4847
:10FCD00070470D4870470D4870470D4870470D48F4
:10FCE00070470D4870470D4870470D4870470D48E4
:10FCF00070470D4870470D48704700BFEBEF0B0889
:10FD000073CD0B0804F00B08CAEC0B0879CD0B0877
:10FD10007FCD0B0885CD0B0891CD0B089BCD0B0833
:10FD2000A5CD0B086BCD0B08AFEA0B08B0CD0B08C7
:10FD30000379062B0ED1C9B2C2680D2996BF064BB6
:10FD40000021595601238B40134214BF08464FF03F
:10FD5000FF307047481C704708F40B0838B5074C53
:10FD6000074DAC4203D3074B01221A7038BDA2885D
:10FD7000D4E9021061F0ECFD1C34F2E7E0C30C089A
:10FD800028CE0C08086E0024204BB0F5FA6F1A68D4
:10FD90000346A8BF4FF4FA63B3F57A7FB8BF4FF4B8
:10FDA0007A73D2041DD540F2DC5290421CD040F24E
:10FDB000DB5207EE903A9042F8EE677A96BFDFED9D
:10FDC000146ADFED146A9FED147A77EEE67A92BF3B
:10FDD0009FED120A9FED127A9FED120AA7EE870A95
:10FDE0007047B0F57A7F02D89FED0F0A704707EE93
:10FDF000903ADFED0E6A9FED0E7AF8EE677A9FED8E
:10FE00000D0A77EEE67AA7EE870A7047BC620024F7
:10FE100000007A4400A0BB44D62000C000E0824429
:10FE2000D6200040000083440000000000407A44D7
:10FE30006610004000004042704700BF704700BF9E
:10FE40000020704701207047704700BF704700BF17
:10FE5000704700BF704700BF9FED010A704700BFA9
:10FE60000000000000207047064B1B78834281BFD2
:10FE700000EB4000044B03EBC003586998BF00201F
:10FE8000704700BF000600203C05002000EB40004A
:10FE9000024B03EBC003587C704700BF3C050020B9
:10FEA000024B1878003818BF012070470006002068
:10FEB000C3B25E2B9ABF024B53F820000148704733
:10FEC0005C750B0820380C0838B50B4D0C4605EB5B
:10FED000C00595F97C01FFF7EBFF01460748FDF7E8
:10FEE000A3FC95F8823133B1611C0548C9B2BDE865
:10FEF0003840FDF799BC38BD5C750B083DD30B0845
:10FF000018F20B08194B1B682DE9F0415BB3002573
:10FF1000174FDFF868801748FDF752FCFDF714FC17
:10FF2000F7F742FDF7F780FD044648B113200CF0C7
:10FF3000BFFBFDF72DFC1048BDE8F041FDF740BCCC
:10FF40003B78012BF2D040466E1CFDF76DFC792DFD
:10FF500002D12646FDF71CFCFDF7F6FB6420354672
:10FF6000F6F702FFDEE7BDE8F08100BF4C21002478
:10FF7000A6310024B6CD0B08D0CD0B08A8EF0B0896
:10FF800010B504460848FDF71BFCF7F711FF20B138
:10FF90000648BDE81040FDF713BC20460449BDE803
:10FFA0001040FDF73FBD00BFD6CD0B08E0CD0B08DC
:10FFB000E8CD0B08154B1B682DE9F041044688B0CD
:10FFC000F3B11A6804A91846D56A6A46A8470646D6
:10FFD00088B104AC6D460027DFF83C80013735F866
:10FFE000022B34F8021B4046FDF79AFCBE42F5DCBA
:10FFF00008B0BDE8F08106492046FDF713FDF7E79C
:020000040805ED
:10000000044908B0BDE8F041FDF70CBDEC670024E1
:1000100009CE0B0821CE0B08EFCD0B08034904488D
:1000200001F500610EC9FDF77BBC00BF00E0F11FC8
:1000300028CE0B0810B5114B86B011490446049325
:10004000104B11480393114B114A0293114B01932A
:10005000114B0093114BFDF7E7FBFDF799FB10499E
:100060001048FDF75DFC3CB10F4A1049104806B03E
:10007000BDE81040FDF754BC06B010BD7CCE0B08A7
:1000800046CE0B0881CE0B0851CE0B088BCE0B0849
:100090003CCE0B0894CE0B08A0CE0B089361002435
:1000A000AFCE0B08B7CE0B08C8CE0B08D9CE0B08C5
:1000B000DECE0B080120BDE770B5054608461646A2
:1000C000FBF7EAFD0D4B041E1A780EDB944205DAAD
:1000D00021460B48FDF724FC204670BD2EB1FF2CB5
:1000E00003D10848FDF71CFCF6E7013A064928460B
:1000F0004FF0FF34FDF796FCEEE700BFE82100204B
:100100000BCF0B081CCF0B082FCF0B08F8B50C46F4
:1001100006460846FBF7C0FD20210546204661F053
:1001200024FD044620B93046BDE8F840FDF774BF11
:10013000114F0134114E3B7832789A4201D0F7F7D3
:10014000BFFD0F4B20461D605EF0EEFA0122014616
:100150002046F7F753FD3B7832789A4201D0F7F703
:10016000AFFD20465EF0E0FA2A4601460548BDE8AC
:10017000F840FDF7D5BB00BF48210024A73100247B
:100180004421002455CF0B082DE9F0410D4688B0DD
:1001900006460846FBF780FD20210446284661F00C
:1001A000E4FC28B9304608B0BDE8F041FDF734BFA3
:1001B000FBF772FD2246054601461048FDF7B0FBED
:1001C00085B1202D2A466946204628BF2022E846D0
:1001D000F7F7BEFD00270646B74208DBAD1B3444E7
:1001E000002EEDD1FDF7D4FA08B0BDE8F08118F883
:1001F000010B0137FDF7F6FAEEE700BF6BCF0B08F6
:100200002DE9F04F9246002689B04FF01909554666
:10021000B3464FF461780C461A4600210746FDF7B5
:1002200046FD0790BAF1000F27D029460622204646
:1002300061F05AFC0028079A384613BF01210021BB
:100240004FF0010B4FF0000BFDF731FD6A7907907D
:10025000334619FB02825946384605922A7919FB22
:1002600002820492EA780392AA7802926A78019252
:100270002A780092104AFDF7BFFA627933460136B8
:10028000594619FB0282384606350592227919FB38
:1002900002820492E2780392A2780292627801923A
:1002A00014F8062B0092044AFDF776FA0A2EB9D10B
:1002B00009B0BDE8F08F00BF83CF0B082DE9F04FE8
:1002C000074689B008468B46FDF7FAFE054638B169
:1002D00000234C4901201A4609B0BDE8F04F8FE7D2
:1002E000494B584693F800A093F8019093F8EA80A0
:1002F000FBF7D2FC092804467BDC06268DF81F504C
:10030000404D46430BF10100FDF796FE834638B1A0
:10031000FBF7C2FC0D289EBF0123A8558DF81F30A6
:100320005846FDF789FE834660B1FBF7B5FC5045A2
:1003300008D8062303FB045358709DF81F3001337F
:100340008DF81F305846FDF777FE824660B1FBF707
:10035000A3FC484508D8062303FB045398709DF876
:100360001F3001338DF81F305046FDF765FE814682
:1003700060B1FBF791FC804508D3062303FB0453CF
:10038000D8709DF81F3001338DF81F30311D0DF1ED
:100390001F0248462944FDF75BFE9DF81F30062BDF
:1003A00009D00023AA193846AB51938009B0BDE8A3
:1003B000F04FFDF731BE63434FF461761921EA181F
:1003C000507911FB00600590107911FB00610491D8
:1003D000D1780391917802910021527808460192D8
:1003E000EB5C0A4A00932346FDF7D6F909B0BDE855
:1003F000F08F09232A460649384609B0BDE8F04F78
:10040000FDF70EBE046800245864002483CF0B0857
:10041000FBCB0B08F7B500230F4E0C461546337087
:100420000E4904EB45050E4B0E4F002818BF194628
:10043000304661F08BFBAC4202D1074803B0F0BDFF
:10044000394634F8022B6846FBF7EEFA6946304627
:1004500061F07CFBEFE700BFEC9E0024A5CF0B080A
:100460009CCF0B08AECF0B08F7B500230B4E04460C
:1004700000EB41050A4F06F8313FAC4202D1094872
:1004800003B0F0BD394634F8022B6846FBF7CCFACE
:100490006946304661F05AFBEFE700BFEC9E00244E
:1004A00018F20B081D9F0024F8B54E1E054601F1F9
:1004B0001F04054F16F8012F284639460235FBF771
:1004C000B3FAA642F6D1F8BDB3CF0B0802460846F0
:1004D000531C05D1044B1A681B790A600B717047D5
:1004E0000249FBF7A1BA00BF02D90B0819F20B08A9
:1004F0002DE9F3410023124D044600EB8106114F14
:1005000005F85A3FB44203D10F4802B0BDE8F0816C
:10051000394628464FF0000861F018FB214668462E
:1005200061F09AFB2021684661F01FFB28B96946FB
:100530002846043461F00AFBE4E780F80080F1E724
:10054000EC9E0024C6EF0B08469F00242DE9F04FD7
:1005500014468BB00F461A4600210646FDF7A7FB4E
:100560000546002C00F0D78022783B789A4202465C
:1005700030460DBF4FF001084FF000080121002167
:10058000FDF795FB237805469C4A41463046FDF72A
:1005900033F93B784146994A3046FDF7FDF8002C87
:1005A00000F0BB80627830467B789A422A460DBFC5
:1005B0004FF001084FF0000801210021FDF777FB03
:1005C000637805468E4A41463046FDF715F97B783B
:1005D00041468B4A3046FDF7DFF807F1C90307F1C2
:1005E000020A04F1CA0B0593A31C4FF000090693FD
:1005F000822307933B784B4500F39180002C00F059
:10060000F68097F8EA30304694F8EA209A422A4673
:100610000DBF4FF001084FF0000801210021FDF748
:1006200046FB94F8EA300546764A41463046FDF7E7
:10063000E3F897F8EA304146724A3046FDF7ACF8E5
:10064000002C00F0D68004F1EA0307F1EA0204F17D
:10065000FA014FF0010833F802CF32F8020F844557
:1006600018BF4FF000089942F5D188F001012A46E1
:100670003046C9B2FDF71BFB0821054604F1EC002A
:10068000FFF7F2FE604A034641463046FDF7B4F8F4
:1006900097F8EA1007F1EC00FFF7E6FE5A4A034626
:1006A00041463046FDF778F8002C00F0A4804FF06A
:1006B000FC094FF0010807EB090104EB0900F8F70A
:1006C00099F909F10409002818BF4FF00008B9F59D
:1006D0008E7FF0D188F001012A463046C9B2FDF77D
:1006E000E6FA082104F1FC00FFF702FF474A03463F
:1006F00041463046FDF780F897F8EA1007F1FC0014
:10070000FFF7F6FE414A0346414630460BB0BDE8CE
:10071000F04FFDF741B8A0463BE7A04657E7079BDF
:10072000FB180993002C60D0079B0998E318194621
:100730000893F8F75FF9059B0AF10E015A789BF8C8
:1007400000309A42069AAAF102030CBFB0FA80F870
:100750004FF00008A2F1020208BF4FEA581833F820
:1007600002CF32F8020F844518BF4FF000088B42C9
:10077000F5D188F001012A463046C9B2FDF797FA53
:100780006278069905469BF81800FFF743FE029031
:100790009BF8003041461E4A30460193089B009367
:1007A00009F10103FDF728F8059B51467A7809F114
:1007B0000109587E0AF1100AFFF72CFE059A0290F3
:1007C000414612F8013F30460BF1010B0193099BA2
:1007D000059200934B460E4AFCF7DEFF069B103352
:1007E0000693079B0933079304E7A046DCE7A0467E
:1007F0001FE7A0464CE7A0467EE700BFB8CF0B0836
:10080000CACF0B08F8CF0B0810D00B0827D00B0865
:10081000DFCF0B082DE9F743804608460C46FDF76D
:100820004FFC054628B14046FDF7F6FB03B0BDE896
:10083000F083204601AA2C492F4661F080F82E460D
:100840000446DFF8A4907CB9022DECD1A7F57A73A9
:10085000B3F57A7F21D94FF4FA634FF47A722349C2
:100860004046FDF7DDFBE1E74DB1012D10D001AAB7
:1008700049460020013561F062F80446E3E70122B1
:1008800021464046FFF718FC431C0646EFD1CDE752
:100890002046FBF701FA0746E9E7154BB8B21B689B
:1008A0005B689847FCEEC07AFF2E17EE902A0BD1BA
:1008B000104BB6EEC00A19780F4BA14210DC11465E
:1008C0000E48FDF72DF8B1E70D4B31460D48B6EE59
:1008D000C00A03EB860383ED1F0AFDF721F8A5E7A5
:1008E0000134A3EC010AE8E7C6EF0B08DAE30B08D2
:1008F000A0230020E8210020689F00244BD00B0893
:10090000EC9E00243ED00B0870B50A4C00250A4E20
:1009100094F8913013B12046FCF7C8FD204601350C
:10092000FCF7A2FE3046FCF7D1FE042D04F1EA04E8
:10093000EED170BDB85D00246061002438B50C466E
:10094000054616492046F8F755F830B9FFF7DCFFA1
:100950001348BDE83840FCF733BF12492046F8F78A
:1009600049F8A8B9104B83F8910083F8990083F8EF
:100970007B0183F8830183F8650283F86D0283F8B5
:100980004F0383F85703094B83F821000848E0E739
:100990002846BDE83840FDF73ABB00BF5AD00B08E7
:1009A00060D00B087BD00B08B85D00246061002488
:1009B00083D00B0870B5054608460C465DF0B4FEC2
:1009C000024670B1102804D12146094861F0EBF8C5
:1009D00038B12846064B074A0749BDE87040FDF785
:1009E00021B803490548BDE87040FCF799BF00BF36
:1009F000C8CE0B089FD00B08AAD00B08D4D00B0888
:100A000070B5054608460C465DF08EFE024670B194
:100A1000042804D12146094861F0C5F838B12846B8
:100A2000064B074A0749BDE87040FCF7FBBF034986
:100A30000548BDE87040FCF773BF00BFD9CE0B0876
:100A4000E2D00B08AAD00B08F2D00B082DE9F04336
:100A500007469BB008460C465DF066FE064620221F
:100A6000002101A861F06AF836B3402E08D0402377
:100A700032463A4938461BB0BDE8F043FCF7D2BFD6
:100A800001AD04F140084FF00009022221466846FA
:100A900061F09BF80023102209A968468DF80290A6
:100AA000FBF770F8099B0DF10202934223D1023447
:100AB00005F8010BA045E8D109AC41220021284DE1
:100AC000204661F03BF8002E3CD095F89C60D6B1F2
:100AD000202205F19D0101A861F006F898B105F109
:100AE0009D012046FFF7E0FC23461E4A38461E497A
:100AF000FCF798FF04E01A7838461C49FCF792FF8F
:100B00001BB0BDE8F0831A4B1B78DBB9D6B901AB3B
:100B1000184E1A46083603CAA24246F8080C46F890
:100B2000041C1346F5D101232046124985F8BD3037
:100B3000FFF7BAFC1048FCF749FE21460F48FCF7C6
:100B4000EFFEDDE795F8BD301BB995F89C30002B22
:100B5000F3D008492046FFF7A7FCEEE705D10B08C4
:100B6000EC9E002443D10B08AAD00B0827D10B0818
:100B7000086E0024899F00244DD10B085CD10B081E
:100B800073B50E4610490546F7F734FF18B93070B3
:100B9000012002B070BD2C78602C8CBF613C413CC0
:100BA000082C0FD8013501230A2201A92846FAF79B
:100BB000E9FF019BAB4205D00F2803D8013440EA7E
:100BC0000410E4E70020E4E702D90B082DE9F04F18
:100BD0000F46904689B0002187EA08080646139A16
:100BE00000250393FDF763F8DFF884906FEA0803AC
:100BF0000446069328460BF079F9129B184230D030
:100C0000069BDFF870B0034014BF4FF0010A4FF0AD
:100C1000000A049310EA070328460CBF4A465A46C6
:100C2000059307920BF074F9039B8046079A51468F
:100C300000903046FCF7E0FD049B22463046B3FAB4
:100C400083F14909FDF733F8059A0446039B002A0E
:100C50000CBF5A464A4651463046CDF80080FCF754
:100C60009BFD0135172DC5D109B0BDE8F08F00BF40
:100C700069D10B084FCC0B0810B5044601202CF0AD
:100C8000F5F828B920460549BDE81040FCF7CABE72
:100C90000348BDE81040FCF743BE00BF70D10B080D
:100CA0007FD10B08064B10B5044618683BF0D4F909
:100CB00028B920460349BDE81040FCF7B3BE10BD7B
:100CC000306E00248AD10B0870B500242B4E96F8A4
:100CD0002330651C2341DB0734D529462848FCF71F
:100CE0001FFE284BE4B2D3F8843393F8E030153B71
:100CF000012B2CD8722120462FF0E2FF014622481A
:100D0000FCF70EFE102120462FF0DAFF01461F48A7
:100D1000FCF706FE1C2120462FF0D2FF01461C489E
:100D2000FCF7FEFD1B2120462FF0CAFF01461948A3
:100D3000FCF7F6FD192120462FF0C2FF01461648A8
:100D4000FCF7EEFD022D4FF00104C0D170BD7521FE
:100D500020462FF0B5FF01461048FCF7E1FD1A21AF
:100D600020462FF0ADFF01460D48FCF7D9FD1B21B1
:100D700020462FF0A5FF01460A48E1E76061002404
:100D8000A0D10B08481C0020ACD10B08C8D10B081F
:100D9000E4D10B0800D20B081CD20B0838D20B0888
:100DA0004BD20B085ED20B08F8B5074608460C4636
:100DB000FDF786F9C8B11F4B1E6801363046344630
:100DC0000BF0A6F80546F0B90134182CA8BF002492
:100DD00020460BF09DF80546A8B9B442F4D1384638
:100DE0001549BDE8F840FCF71DBE2046FAF754FF50
:100DF00004460BF08DF8054628B921460F48BDE89A
:100E0000F840FCF78DBD0B4B1C600BF019FC2A461B
:100E10000B482146FCF784FD172C9BBF094B0C2285
:100E2000002002FB043398BF93F82403BDE8F84088
:100E30000BF03EBC6806002471D20B0885D20B086B
:100E40009BD20B085C750B0870B505460C46114E1D
:100E50002046FDF735F960B10F4B104893F90010AB
:100E60004B1C0ABF0E4BC9B21978BDE87040FCF7A5
:100E700057BD2046FAF710FF032804D8C0B2344605
:100E8000FCF74AF9E4E7284603220649BDE870402A
:100E9000FCF7C8BDFDCA0B0830060024B4D20B080D
:100EA0008C610024C4D20B0870B505460C46114E67
:100EB0002046FDF705F960B10F4B104893F900107B
:100EC0004B1C0ABF0E4BC9B25978BDE87040FCF705
:100ED00027BD2046FAF7E0FE032804D8C0B2344606
:100EE00015F0FEFFE4E7284603220649BDE87040FE
:100EF000FCF798BDFDCA0B0831060024B0D20B08E0
:100F00008C610024BFD20B080329F0B5054685B0DB
:100F10000C46164614D80B4F3970FCF739FC0A49B9
:100F20002846FFF791FF2246084901A8FAF77CFD01
:100F300001AB324608212846FCF736FFFF233B7001
:100F400005B0F0BD30060024FDCA0B08B4D20B0872
:100F50000329F0B5054685B00C46164614D80B4F4C
:100F60003970FCF715FC0A492846FFF79DFF224619
:100F700008496846FAF758FD6B4632461021284664
:100F8000FCF712FFFF233B7005B0F0BD31060024D3
:100F9000FDCA0B08B0D20B0870B5174E0446337863
:100FA0006BB1164D2B7853B11549FCF73BFD20462C
:100FB0001449FCF737FD00203070287070BD124BCB
:100FC00093F8BD20B2B193F89C209AB903F19D0229
:100FD00003F1C00503F1BD061068083252F8041C85
:100FE0002C46B24203C42546F6D1012283F8FB20E9
:100FF0000AF002FE0120E1E7305D0024315D0024AB
:10100000DFD20B0816D30B08EC9E00242DE9F84F15
:10101000002607460C461D4DB046DFF87890DFF8F5
:1010200078A02046FDF74CF8D5F800B048B9214625
:101030005846FAF78FFD20B921466868FAF78AFD0D
:1010400080B15846FCF79CFB696811B15046FCF72B
:10105000EBFBA96811B14846FCF7E6FB4FF001082D
:10106000FCF796FB013610353C2EDAD12046FDF711
:1010700027F848B9B8F1000F06D12246384604498E
:10108000BDE8F84FFCF7CEBCBDE8F88FA0790B089F
:1010900040D30B083AD30B0834D30B08424B2DE94D
:1010A000F74F1A780546009140495B780A70404A2C
:1010B0001370404B1B780BB9FEF750FE3E4C0026D8
:1010C0004CF058FAB046A3460D23009973435BF8E1
:1010D00003904846FAF73EFD002840D0B8F1000FD3
:1010E00001DDFCF755FB49463448FCF79DFB002227
:1010F00021462846FCF7CAFEFCF74AFB237903F099
:101100001803082B43D0102B46D02046FCF7CCFE0A
:101110000D2303FB06B3B3F809004CF0F1F9824646
:10112000D8B12046FCF7F2FD0746DAE90221024475
:1011300001442046FCF774FD78B9494601902048E7
:10114000FCF772FBDAF80810019A28461346CA1910
:101150002146FCF77FFCFCF71BFB08F10108013678
:101160000D34B6F52C7FAFD10020FCF7ADFDFF2389
:101170000E4A13700E4A1370B8F1000F11D1009A85
:101180002846104903B0BDE8F04FFCF74BBC0E49B0
:101190002846FFF759FEB8E70B492846FFF784FEBB
:1011A000B3E703B0BDE8F08F8C6100243006002463
:1011B00031060024086E00246C520B08EEC80B08A0
:1011C00054D30B085ACC0B08FDCA0B082DE9F04F7D
:1011D0003B4C89B00A4600210546FCF768FD0590A6
:1011E00094F90000FEF764FE814660884CF088F9AF
:1011F000344BD0F808B01F7817B15F46D0F80CB068
:10120000A3790026012B38BF012306932279637945
:1012100006FB02331BF80380002F3AD0FB5C4345EA
:10122000059A2846079313BF012100214FF0010AB8
:101230004FF0000AFCF73BFD079B0136059053B3C6
:1012400003F00F021B0951462846403302921E4A02
:10125000CDE900634B46FCF7CFFAB8F1000F24D07C
:1012600008F00F034FEA1818174A5146029308F185
:1012700040032846CDE900634B46FCF78DFA069BF8
:10128000B342C3DC0834114BA342A9D109B0BDE875
:10129000F08F3B46C3E7002FDFD04B460C4A514648
:1012A00028460096FCF7A8FAD7E76B06E7D44B462A
:1012B000074A514628460096FCF76EFADFE700BF62
:1012C000D8760B08086E002464D30B0880780B08CE
:1012D0007AD30B08234870B5FCF752FA224B93F8E7
:1012E000FC30002B38D0214B93ED010A5FF032FA2D
:1012F00001461F48FCF714FB1E4C1F48FCF740FA40
:101300001E4B94F821001E4A00280CBF10461846B8
:10131000FCF756FA94F8213013B31A4C1A48B4F873
:101320009210FCF781FA194E94F89000184D00289D
:101330000CBF30462846FCF743FAB4F89410154821
:10134000FCF772FA94F8910000280CBF304628464A
:10135000BDE87040FCF734BA0F48FCF731FACBE730
:1013600070BD00BF9ED30B08EC9E002468060024CD
:10137000B8D30B08B4610024C7D30B086FC90B089E
:101380004DF10B0840350020D8D30B0897D30B083C
:101390008ED30B08FFD30B08BDD30B086B4B1B7808
:1013A0002DE9F04F87B0002B00F0CA80684D4FF058
:1013B00000086848A968FCF7B3FA69686648FCF752
:1013C000AFFA664B6648D3E90031C91A654B1A6813
:1013D000B1FBF2F2FCF7A4FAFCF7DAF96248FCF789
:1013E000EFF96248FCF7ECF9614B5FFA88F41B787F
:1013F000A34221D85F4D00245F4EFCF7C9F90134A8
:1014000055F8041F3046FCF70FFA162CF7D15B4D48
:101410000124594EFCF7BCF92B466968013430466B
:101420001B680435C91AFCF7FFF9162CF4D107B074
:10143000BDE8F04FFCF7ACB9514B14264FF03C0B14
:10144000671C03EB840306FB045693ED280A5FF048
:1014500081F996F81EA081B2B6F80E901AF0010F2D
:1014600080B20CBF2D2252221AF0020F0490454880
:101470000CBF2D2354231AF0040FB1FBFBF10CBF5A
:101480004FF02D0C4FF0560C1AF0080F05914FF04D
:1014900064010CBF4FF02D0E4FF0430E1AF0800F79
:1014A00001FB09F10CBF4FF02D0A4FF0530ACDE9B3
:1014B00000CECDE902A13946FCF7B6F9B37FDB07D0
:1014C0003AD55C23304A6343D118D05891ED010AD4
:1014D00070B1B8EE400ADFED2D7A20EE270A07EE54
:1014E000900AF8EE677A80EE270A5FF033F900B2CF
:1014F000642290FBF2F102FB11022548FCF794F9FB
:101500001421244808F1010801FB075701FB04548A
:10151000F988628A0491218B02F0030392080391F7
:10152000E18A0291A18B0191A18A009119214B437B
:10153000218AFCF7F5F957E71748FCF721F9DFE7AF
:10154000164807B0BDE8F04FFCF73AB90400002098
:10155000101B00201FD40B082FD40B083C1C0020AC
:1015600046D40B08AC1E002473D40B08CFD40B0850
:10157000E8210020B81B00207FD50B08BC1B0020F1
:10158000403500202BD50B083018002000401C46A9
:1015900048D50B085DD50B0854D50B0883D50B082F
:1015A00008B5294B1B68DB041ED5B5EE400AF1EEE9
:1015B00010FA26D0DFED257AB4EEE70AF1EE10FA44
:1015C0001FD49FED237AB4EEC70AF1EE10FA2AD8A1
:1015D00070EE677A9FED1F7A9FED1F0AA7EE870ACC
:1015E0005FF0B8F880B208BDDFED187AB4EEE70A14
:1015F000F1EE10FA0BDA9FED190A5FF0ABF880B24A
:1016000008BD9FED170A5FF0A5F880B208BD70EE27
:10161000677A9FED147A9FED140AA7EE870A5FF0B0
:1016200099F880B208BDDFED117ADFED116A70EE36
:10163000677A9FED107AA7EEA67AB0EE470A5FF0C0
:1016400089F880B208BD00BFBC620024000040429F
:1016500000E0824466BEFFBE0060BB4400007A44E6
:101660000080BB4438DFFF3E00407A4400008344E2
:1016700066BEFF3E00A0BB44B94B42F201011A68AE
:10168000B1EB124F4FEA12432DE9F04F804691B073
:1016900000F0FC8142F20302934200F0F98141F232
:1016A0000302981A43424341AE4A0024AE4E1168E9
:1016B00006EBC303AD4AAE4DAE48AF4FDFF888939B
:1016C000BA46DFF888B3B1FBF2F2D3F80818FCF79A
:1016D000ABF8B5F8FE204FF47A730A20B2FBF3F1B1
:1016E00003FB1122B5F9003192B2B2FBF0F2A3482C
:1016F000FCF716F9A24AA349A348FCF795F8FCF7B2
:1017000047F8A24BA24A997BA24B06EB8101A24863
:10171000D31AA24AD1F824181288FCF701F9FCF771
:1017200037F89F48FCF72CF895F802119D48FCF714
:101730007BF89D48FCF724F89C4B95F803111A8818
:101740009B4892B2FCF770F8FCF722F899499A4846
:10175000FCF76AF8234699F81F202241D1072CD5BF
:1017600013B19648FCF70CF8611C9548FCF75CF83F
:10177000944B9548E35C5BF82310FCF755F89AF816
:101780007A352341DA0702D59048FCF74DF897F8EF
:101790002031032B09D08E48FCF746F897F820310A
:1017A000012B02D18B48FCF73FF8FB6C5B7B012BD4
:1017B00002D98948FCF738F8012307F5D277002CC5
:1017C00000F06881002B40F067818448FBF7F8FF48
:1017D000834FD5F80891DFF878A207F1180B0123A1
:1017E000A34013EA090F15D01AF8042057F8243043
:1017F0005BF8241053F822207A48FCF715F8012CE6
:1018000006D1794B93F8DD1011B17848FCF70CF84C
:10181000FBF7BEFF0134062CE1D17548FBF7B0FFA2
:10182000744B1B681B0640F1678195F82831724F95
:10183000032B8CBF71487248FBF7A2FF3B78022B49
:1018400040F02D816F48FBF79BFF95F82831042B62
:1018500000F24A816C48FBF793FF95F83831002B72
:1018600000F0488106EBC303D3F860186748FBF724
:10187000DBFFFBF78DFF664B66481C68664B1A78EA
:10188000664B53F82210FBF7CFFF24B1227A617A1E
:101890006348FBF7C9FFFBF77BFF62494046FBF754
:1018A000D0FFF6F771F8016921B182685E48120D28
:1018B000FCF736F8FBF76CFF5C4B5D4819684FF49A
:1018C0007A73B1FBF3F1FBF7AFFF05A8FAF7B0FAB3
:1018D00038B105A908A85CF037FB08A95548FBF703
:1018E000A3FFFBF755FFD5F8C471002F00F0088166
:1018F00007EE907ADFED506AB8EEE77AC6EE877AA7
:10190000FDEEE77A17EE903A95F8FC0030B14B4ABD
:10191000039392ED010A5EF01DFF039BD5F844414D
:101920005CB107EE904ADFED446AF8EEE77A86EEA6
:10193000A77AFDEEC77A17EE904A2B4AB2F82C111F
:101940003A466429CDE90004A8BF64213C48FBF76E
:10195000E7FFB5F87C2A64233A48B2FBF3F179E05B
